:020000040800F2
:100000000000022025C1000821C1000821C100080C
:1000100021C1000821C1000821C100080000000022
:1000200000000000000000000000000021C10008E6
:1000300021C100080000000021C1000821C1000802
:1000400021C1000821C1000821C1000821C1000808
:1000500021C1000821C1000821C1000821C10008F8
:1000600021C1000821C1000821C1000821C10008E8
:1000700021C1000821C1000821C1000821C10008D8
:1000800021C1000821C1000821C1000821C10008C8
:1000900021C1000821C1000821C1000821C10008B8
:1000A00021C1000821C1000821C1000821C10008A8
:1000B000FD5E000821C1000821C1000821C100081F
:1000C00021C1000821C1000821C1000821C1000888
:1000D00021C10008AD97000821C1000821C1000816
:1000E00021C1000821C1000821C1000821C1000868
:1000F00021C1000821C1000821C1000821C1000858
:1001000021C1000821C1000821C1000821C1000847
:1001100021C10008819A000821C1000821C10008FE
:1001200021C1000821C1000821C1000821C1000827
:1001300021C1000821C1000821C1000821C1000817
:1001400021C1000821C1000821C1000821C1000807
:1001500021C1000821C1000821C1000821C10008F7
:1001600021C1000821C1000821C1000821C10008E7
:1001700021C1000821C1000821C1000821C10008D7
:1001800021C1000821C10008044B05481B1A062B99
:1001900002D9044B03B11847704700BF9F060020E7
:1001A0009C0600200000000005490648091A891035
:1001B00001EBD171491002D0034B03B118477047CE
:1001C0009C0600209C0600200000000010B5064C94
:1001D000237843B9FFF7D8FF044B13B10448AFF3BA
:1001E00000800123237010BDA00600200000000045
:1001F000786C040808B5084B1BB108490848AFF3F0
:1002000000800848036813B9BDE80840CCE7064BF6
:10021000002BF9D09847F7E700000000A406002063
:10022000786C04089806002000000000134B002B97
:1002300008BF114B9D46A3F5803A00218B460F461F
:100240001148124A121A0CF097FD0D4B002B00D0EA
:1002500098470C4B002B00D0984700200021040049
:100260000D000B480CF088FC0CF0B4FC20002900B9
:1002700004F0A4FA0CF086FC000008000000000066
:100280000000000000000000A006002090BD00203B
:10029000ADCB000838B54FF4B971044604F11C0524
:1002A00006F006F9002222616261A26104F13C01BC
:1002B0002B4623F8022B8B42FBD104F2EC420020A8
:1002C00003F8010B9A424FF00001F9D1F023C4F872
:1002D000F034A4F8EC14A4F8EE14202228460CF014
:1002E0004BFD0523237409236382024B6361A561DF
:1002F000204638BD04000020222A70B506460C4670
:100300000ED106F0E7F820280CD904F1210514F8E5
:10031000011F304606F020F9AC42F8D1002070BD34
:10032000042070BD052070BDF0B500238FB04FF4E0
:10033000E37540F252564FF6AE274FF63A6E01F093
:10034000C002802A02AC0BD0C02A06D0002A0CBF03
:1003500072463A4624F8132004E024F8136001E0C2
:1003600024F8135001338A00042BD1B2E7D104AA38
:10037000214610300BF03AFF0023009304AA142307
:100380000221024803F068F80FB0F0BD00650020BC
:10039000B0F8EC3470B5044623B12A4803F0BCF839
:1003A00005460DE006F0B8F828BB04E0A4F8EC140C
:1003B0000023A4F8EE34B4F8EC34002B41D0ECE781
:1003C000142D3ED9B4F8EE345A1C2344A4F8EE247C
:1003D00093F83C102046FFF7A7FFB4F8EE24B4F8DA
:1003E000EC34143D9A42ADB2EAD30023A4F8EE34C3
:1003F000A4F8EC3470BD144B1B785BB9D4F8F0143E
:100400005F209AB2914203F10103CFD9224482F8CE
:100410003C00F6E704F13B0604F15C05204606F0DB
:10042000C1F806F8010FB542F8D1084900235A5C1B
:1004300005F8012F0133272BF9D14823A4F8EC3418
:10044000B6E770BD00650020FC640020D8D300082A
:1004500008B506F03FF82323B0FBF3F0C0B208BDA7
:100460000C234FF4167203FB0121B1F5966F8ABF7E
:100470004FF49663C0F8F014C0F8F034704730B50C
:10048000002200240025C0E900458260C26002828B
:1004900042618261027730BDF0B500240025C0E9D9
:1004A00000450C4E2501AF5D8F4206D109490D4430
:1004B000D5E90245C0E9004502E00134322CF1D112
:1004C000D0E9004554EA05011DBF8260C3600020E9
:1004D0000420F0BD20D400082DE9F743044601EBC9
:1004E0006101636965682768D4F818E0007FA3613B
:1004F0004FEAE37903FB05F207FB0922A3FB078917
:1005000091444FEAD87242EA490202F31E02CEEB4E
:1005100042021144228A6161013292B241F2707E3C
:1005200000F0FE0672452677228250D181FB0189B8
:100530004FEAD87E4EEA490E83FB03894FEAD87C06
:100540004CEA490C83FB01894FEAD87848EA49080C
:1005500008F31E034FEAE3795D4307FB0955A3FB4C
:10056000078900F00203002BA944A3680EF31E0EB6
:100570000CF31E0C4FEAD872E64418BFE36842EA57
:10058000490202F31E02AEEB420214BF0125002510
:100590009342C8BF20F0030046F00101CCBF40F0F9
:1005A000010046F003062177D4BF26772077217F0C
:1005B000C1F340018D4206D000911BB212B2064930
:1005C000064801F00AFE002323826361A361207FB5
:1005D00003B0BDE8F08300BFFFD30008283000203F
:1005E0000023436183610377038270470022027016
:1005F0007047000008B5037853B1064802F08CFF3D
:10060000A52805D9AA210448BDE8084000F066B82D
:1006100008BD00BF006500203C310020012A06D142
:100620000B785A1E53425341037000207047042038
:100630007047000038B54FF47A61044604F11C0598
:1006400005F036FF002222826261A26104F5B871D2
:100650002B4623F8022B8B42FBD104F50E720020AF
:1006600003F8010B9A424FF00001F9D14823A4F896
:100670003C32A4F83812A4F83A124FF4AA72284671
:100680000CF07AFB06232382024B6561A3612046AE
:1006900038BD00BF5E00002008B5B0F8383213B98D
:1006A00005F03AFF00B1012008BD442A70B50646A6
:1006B0000C460ED105F00EFF43280CD9651E4334BD
:1006C00015F8011F304605F047FFA542F8D100207C
:1006D00070BD042070BD052070BD000070B50646D9
:1006E000ADF5227D0D4600242B0602AB4CBF0F4911
:1006F0000F491819282228340CF0A4FA6D00B4F51B
:10070000A07FEDB2F0D152AA02A906F11000A023F9
:100710000BF068FF0023009352AAA023062105488E
:1007200002F09AFE0DF5227D70BD00BF68D700086B
:1007300040D700080065002038B5044605F0ECFEFF
:10074000B4F8383208B903B938BD3BBB254A127832
:100750009AB9B4F83C52AA219AB2954203D8002320
:10076000A4F83A321AE0B4F83822501C2244A4F813
:100770003802013382F87011EEE74425204605F077
:1007800011FFB4F83832013D5A1C234415F0FF051F
:10079000A4F8382283F87001F0D1E0E7B4F83832D9
:1007A000F3B1114802F0B8FE0546A02D18D9B4F8EF
:1007B0003A325A1C2344A4F83A2293F87011204686
:1007C000FFF78CFFB4F83A22B4F83832A03D9A42D1
:1007D000ADB2EAD30023A4F83A32A4F8383238BDD7
:1007E00038BD00BFFC6400200065002001EB410122
:1007F0004908483189B296298ABF9623A0F83C124D
:10080000A0F83C32704708B505F064FE4423B0FB05
:10081000F3F0C0B208BD10B5044604F079FC002323
:10082000237563752361204610BD38B5457D0446A8
:10083000EDB9037D93B1012B12D103691943016115
:10084000C1F3072104F0B4FCA17C204604F0B0FC05
:10085000E17C204604F0ACFC256101E00903016164
:10086000237D0133DBB2012B88BF00232375637D19
:100870000133DBB2022B88BF0023637538BD002231
:1008800002608280C28070472DE9F8431446214AF5
:100890000546002312F833001E4F884204D1DBB214
:1008A00017EBC30704D12EE00133322BF2D12AE03B
:1008B00028687B88AB8008B10CF028F9A888400034
:1008C0000CF022F904EB44060021286004EB8606B4
:1008D0008846AB888CB2A34201F1010916D9404683
:1008E0000CF0F6F82A68C317A0FB060106FB0311FB
:1008F000C30F43EA410303F30F0322F814307B686C
:1009000049469844E5E70420BDE8F8830020BDE8A7
:10091000F88300BF90D70008C3885A1C92B210B564
:100920000468C28034F91330848894429CBF00224A
:10093000C28011B1584200B210BD184610BD024627
:10094000002310B502F8013B00F2E934194602F821
:10095000011BA2424FF00003F9D1A0F8EA33A0F83E
:10096000EC33A0F8EE33A0F8F033C0F8F433A0F87D
:10097000F833A0F8FA33A0F8FC33A0F8FE3310BD2A
:100980002DE9F74F0446DFF80C81DFF80C910020C9
:10099000A4F8EA03C5B211F805E0BEF1000F48D093
:1009A00000260C27F5B27D4308EB050718F8055023
:1009B000002D3CD0AE4506F10106F2D13D7A0195FD
:1009C0004FF0000C4FF0004E019E5FFA8CF5AE42E6
:1009D0002DD97E68B4F8EA533EEA06064FEAE50AE6
:1009E0000CBF04EB0A0604EB0A0605F0070B0BBF6D
:1009F0007678767819F80BB019F80BB0A2440CBFD2
:100A00004BEA060626EA0B068AF8016040F2E23657
:100A1000B5420CF1010C04D90023A4F8EA330420F8
:100A200035E00135A4F8EA534FEA5E0ECCE7013019
:100A3000B0E79DF83010D4F8F403A4F8FC139DF847
:100A40003410A4F8FE1345F6C051B1FBF2F2B1FB2D
:100A5000F3F3A4F8EE23A4F8F83308B10CF056F839
:100A6000B4F8F8030CF050F8B4F8F813C4F8F40331
:100A700003464C08002501261A1A92B2914205D964
:100A800094428CBF1E701D700133F5E7002003B047
:100A9000BDE8F08F20D9000830DB0008037810B5DE
:100AA000002B3ED0B0F8EC231F4C00EBD20302F039
:100AB00007015B78615C0B400CD0B0F8FA33D0F8DA
:100AC000F413CB5C13B1B0F9FC3303E0B0F8FC33A2
:100AD0005B421BB2B0F8FA13B0F8F843013189B2A7
:100AE0008C42A0F8FA139CBF0021A0F8FA13B0F8CA
:100AF000F013B0F8EE43013189B28C42A0F8F01344
:100B00000FD80132B0F8EA4392B200219442A0F823
:100B1000EC23A0F8F0139EBF0170A0F8EC13A0F82E
:100B2000FA13184610BD00BF30DB0008037810B57B
:100B3000002B3ED0B0F8EC231F4C00EBD20302F0A8
:100B400007015B78615C0B400CD0B0F8FA33D0F849
:100B5000F413CB5C13B1B0F9FE3303E0B0F8FE330D
:100B60005B421BB2B0F8FA13B0F8F843013189B216
:100B70008C42A0F8FA139CBF0021A0F8FA13B0F839
:100B8000F013B0F8EE43013189B28C42A0F8F013B3
:100B90000FD80132B0F8EA4392B200219442A0F893
:100BA000EC23A0F8F0139EBF0170A0F8EC13A0F89E
:100BB000FA13184610BD00BF30DB00080023037095
:100BC000A0F8EC33A0F8F033A0F8FA3370470078BF
:100BD0007047B0F8EC3343B9B0F8F0332BB9B0F844
:100BE000FA03003018BF012070470120704708B594
:100BF0000246FFF7EEFF38B901231370A2F8EC03A9
:100C0000A2F8F003A2F8FA0308BD000030B58BB0DB
:100C1000C57A047A8378427801780995857A0895AF
:100C2000457A0795E50904F07F0406950594C47993
:100C30000494847903944479029404790194C078EB
:100C4000009001EB8101024801F0FCFC0BB030BDCB
:100C50007092002010B50246044600F58071002015
:100C600002F8010B8A424FF00003F9D184F80031F9
:100C700084F8013184F802314FF4B97104F58270BF
:100C800005F016FC204610BD1FB570228DF80E2011
:100C900082788DF80F20E02300228DF80C3000922E
:100CA000042303AA01218DF80D3009F024F805B0C2
:100CB0005DF804FB1FB57F228DF80A2082788DF83D
:100CC0000B20E02300228DF808308DF80C1005234E
:100CD0000092012102AA8DF8093009F00CF805B044
:100CE0005DF804FB2DE9F047824688B0774802F0B2
:100CF000F2FE00228DF80F20754AE0238DF80C30AB
:100D000011780D238DF80D3001238DF80E309146AA
:100D100009B18DF80F306F4B1A7898462AB19DF8BB
:100D20000F3043F002038DF80F306B4F3B782BB13F
:100D30009DF80F3043F004038DF80F30674E337881
:100D40002BB19DF80F3043F008038DF80F30644D40
:100D50002B782BB19DF80F3043F010038DF80F3036
:100D6000604C23782BB19DF80F3043F020038DF8B1
:100D70000F305D4B1B782BB19DF80F3043F04003D3
:100D80008DF80F30594B51481B788DF81030584B67
:100D90000DF10B021B788DF811300DF10A0102F0F4
:100DA00082FE9DF80A302BB19DF8113043F002030A
:100DB0008DF81130454802F08BFE28B19DF81130B6
:100DC00043F004038DF81130404802F07EFE28B154
:100DD0009DF8113043F008038DF811303B4802F0C4
:100DE00081FE28B19DF8113043F010038DF81130C9
:100DF0009DF80B302BB19DF8113043F020038DF896
:100E000011303C4A9DF811301278002A14BF40225C
:100E1000002213438DF8113099F800302BB1364879
:100E200003F022FA8DF8120001E08DF8123098F8E4
:100E30000030A3B1314B1B7843B1314809F0F6F8CB
:100E40008DF813002E4809F0F9F805E00A232D4823
:100E50008DF81330FFF7FCFA8DF8140003E08DF8DD
:100E600013308DF814303B782BB1274802F07EFF09
:100E70008DF8150001E08DF8153033782BB123483B
:100E800005F008FB8DF8160001E08DF816302B7880
:100E90002BB11F4808F092F98DF8170001E08DF88A
:100EA000173023782BB11B48FFF7ADFC8DF81800E5
:100EB00001E08DF818300023009303AA0D230121CF
:100EC000504608F018FF08B0BDE8F0870065002024
:100ED0005D0200205C0200205B0200205E02002018
:100EE0005A0200205F0200205902002088330020AF
:100EF000FC64002089330020DC1000205802002010
:100F00008C33002054B00020A89B002078340020AF
:100F1000480B00203C31002010B5A8B0E0238DF82C
:100F20000830002201230D4C8DF80A208DF80B307B
:100F3000D1B2131D615CDBB2013229B10DF1A00EFB
:100F4000734403F8981CF3E7009102AA01218DF87D
:100F5000093008F0D0FE28B010BD00BF3EDF000809
:100F60002DE9F04F072A97B035D989464B7819F803
:100F7000060F0C788D78CE780F7991F805E0A2F104
:100F8000080B5FFA8BFB03EB83030BF1070B00F0FD
:100F9000010CC0F340085B00C0F380000DF1230A90
:100FA000594419F801BF0AF801BF8945F9D1D11F89
:100FB00016AA52FA81F1002201F8342C0690CDF8DD
:100FC0001480CDF810C08DE8E040224609A90448FD
:100FD00001F0D4FA00E0042017B0BDE8F08F00BFA4
:100FE00070920020F0B5052A93B029D9C8784B78C3
:100FF0000E788F7800EB80000C464500901FC0B241
:1010000003EB8303053014F804EF5B000DF1130CC0
:10101000014414F8010F0CF8010F8C42F9D1511F53
:1010200012AA52FA81F1002201F8342C0648CDF8B8
:1010300008E001950097324605A901F0DFFA00E0CB
:10104000042013B0F0BD00BF709200200B2A02D91B
:101050000846FFF7DBBD0420704710B54FF4E132BE
:101060000446012108F01CFE20464FF416520321CD
:10107000BDE8104008F014BEF0B5154B1B78012BED
:1010800091B023D8134B1B7803B3E0238DF80C30B9
:10109000CDB210238DF80E30C5F10307CBB2DC19A9
:1010A0005B1BDBB29A42E4B206D910AB234411F8C1
:1010B000016B03F8346CF1E7D31C0022DBB2009221
:1010C000012103AA8DF80D3008F015FE11B0F0BD16
:1010D000883300205D020020F0B5154B1B78012BF2
:1010E00089B023D8134B1B7803B3E0238DF80C3061
:1010F000CDB211238DF80E30C5F10307CBB2DC1948
:101100005B1BDBB29A42E4B206D908AB234411F868
:10111000016B03F8146CF1E7D31C0022DBB20092E0
:10112000012103AA8DF80D3008F0E5FD09B0F0BDEE
:10113000883300205D0200201FB50C4B1B78012B6B
:1011400011D80B4B1B7873B11222E0238DF80E20BF
:1011500000228DF80C300092032303AA01218DF8A0
:101160000D3008F0C8FD05B05DF804FB88330020A1
:101170005D0200201FB50C4B1B78012B11D80B4BC7
:101180001B7873B11322E0238DF80E2000228DF816
:101190000C300092032303AA01218DF80D3008F0D2
:1011A000AAFD05B05DF804FB883300205D02002035
:1011B000F0B5184C247814F0FD0F8DB027D1164CE3
:1011C000247824B300294FF0E00414BF1A21182119
:1011D000D5B28DF808408DF80A10C5F10307D1B2D9
:1011E000CC19491BC9B28B42E4B206D90CA92144DF
:1011F00012F8016B01F8286CF1E700220333DBB22F
:101200000092012102AA8DF8093008F074FD0DB09A
:10121000F0BD00BF883300205C0200201FB50E4BDC
:101220001B7813F0FD0214D10C4B1B788BB10029F5
:101230004FF0E00314BF1B2119218DF80C308DF8FD
:101240000E1003230092012103AA8DF80D3008F03F
:1012500052FD05B05DF804FB883300205C020020DD
:10126000F0B5164B1B78032BA5B000D01BBB144B5D
:101270001B7803B3E0238DF80C30CDB220238DF81A
:101280000E30C5F10307CBB2DC195B1BDBB29A420F
:10129000E4B206D924AB234411F8016B03F8846C43
:1012A000F1E7D31C0022DBB20092012103AA8DF8E2
:1012B0000D3008F020FD25B0F0BD00BF88330020C0
:1012C0005B0200201FB50D4B1B78032B00D08BB9A0
:1012D0000B4B1B7873B12122E0238DF80E200022E6
:1012E0008DF80C300092032303AA01218DF80D30F4
:1012F00008F001FD05B05DF804FB00BF8833002055
:101300005B020020F0B5164B1B7813F0FB0FA1B069
:1013100023D1144B1B7803B3E0238DF80830CDB2F2
:1013200030238DF80A30C5F10307CBB2DC195B1B03
:10133000DBB29A42E4B206D920AB234411F8016B28
:1013400003F8786CF1E7D31C0022DBB20092012194
:1013500002AA8DF8093008F0CEFC21B0F0BD00BF24
:10136000883300205E020020F0B5164B1B7813F086
:10137000FB0FC3B023D1144B1B7803B3E0238DF8CC
:101380000C30CDB231238DF80E30C5F10307CBB24E
:10139000DC195B1BDBB29A42E4B206D942AB2344B0
:1013A00011F8016B03F8FC6CF1E7D31C0022DBB2EF
:1013B0000092012103AA8DF80D3008F09CFC43B087
:1013C000F0BD00BF883300205E0200201FB50C4B2B
:1013D0001B7813F0FB0210D10A4B1B786BB1E02392
:1013E00032218DF80C308DF80E100323009201216C
:1013F00003AA8DF80D3008F07EFC05B05DF804FB03
:10140000883300205E020020F0B5164B1B78052BB8
:10141000A5B000D01BBB144B1B7803B3E0238DF8A1
:101420000C30CDB240238DF80E30C5F10307CBB29E
:10143000DC195B1BDBB29A42E4B206D924AB23442D
:1014400011F8016B03F8846CF1E7D31C0022DBB2C6
:101450000092012103AA8DF80D3008F04CFC25B054
:10146000F0BD00BF883300205A0200201FB50D4B8D
:101470001B78052B00D08BB90B4B1B7873B1412225
:10148000E0238DF80E2000228DF80C30009203230B
:1014900003AA01218DF80D3008F02DFC05B05DF890
:1014A00004FB00BF883300205A020020F0B5144B23
:1014B0001B78632BA5B020D1E0238DF80C30CDB282
:1014C00008238DF80E30C5F10307CBB2DC195B1B86
:1014D000DBB29A42E4B206D924AB234411F8016B83
:1014E00003F8846CF1E7D31C0022DBB200920121E7
:1014F00003AA8DF80D3008F0FEFB25B0F0BD00BF4B
:1015000088330020F0B5144B1B78602B8BB020D1B2
:10151000E0238DF80830CDB209238DF80A30C5F1EB
:101520000307CBB2DC195B1BDBB29A42E4B206D9EB
:101530000AAB234411F8016B03F8206CF1E7D31CCC
:101540000022DBB20092012102AA8DF8093008F0D6
:10155000D2FB0BB0F0BD00BF8833002010B590F86F
:101560000231A4B0CBB1E0238DF80C30F1238DF81B
:101570000E300022D4B2D31C0C5DDBB201322CB190
:101580000DF1900E734403F8844CF3E701210091B0
:1015900003AA8DF80D3008F0AEFB24B010BD00009A
:1015A0005F2910B50C4650D021D8052945D00FD859
:1015B00002293BD006D8012959D14D494D48FFF7A2
:1015C000CDFF70E0032936D0042950D14A4947E0C5
:1015D0005B2944D005D8062931D00A2947D147498B
:1015E0003EE05C2939D05D2941D1454938E0662982
:1015F00031D00CD8622926D003D8602937D141498F
:101600002EE063291DD0652931D13F4928E06929A1
:101610001FD005D867291AD0682928D13B491FE077
:101620006A2918D06B2922D1394919E03949314842
:10163000FFF794FF21E0384912E0384910E03849BB
:101640000EE038490CE038490AE0384908E03849EA
:1016500006E0384904E0384902E0384900E03849FA
:101660002448FFF77BFF374806F058FC0AE036496C
:101670002048FFF773FF012C15D0324806F04EFCCE
:10168000022C30D0314802F01AFE314805F0DEFF5E
:10169000304807F0DBF8032C0ED12F4803F07DFE15
:1016A000052C13D00DE0294802F009FE284805F06A
:1016B000CDFF284807F0CAF8284805F099FB042C0C
:1016C000EBD1274803F00EFA0A2C02D0254800F08F
:1016D0001FFF254807F0F8FF244B25481C70BDE884
:1016E000104001F02FBF1D4805F082FBD5E700BF79
:1016F00048DB00082830002075DB0008A9DB000863
:10170000C3DC0008EFDB00082DDD000866DC000804
:10171000A4DC000838DB00085BDB000885DB000880
:1017200096DB0008B8DB0008D5DB00080ADC0008FF
:1017300045DC000885DC000826DC0008E5DC000844
:101740000ADD00089C6100204ADD0008F83900200D
:10175000B47B002080130020483F00203468002024
:10176000A8A0002070920020580700208833002095
:10177000006500202DE9F04F142A9FB001D8042005
:1017800021E10D78C5F3001380F802318E78322EF6
:10179000F5D84C7891F803E004F0020204F0040359
:1017A00004F0080A04F0100904F0200804F04007CF
:1017B000BEF1060FD2B2DBB25FFA8AFA5FFA89F99C
:1017C0005FFA88F8FFB210D9BEF10A0F35D0AEF13A
:1017D0005B0C5FFA8CFCBCF1100FD0D8DFF838B28C
:1017E0002BFA0CFC1CF0010F04E0BEF1010F03D139
:1017F00014F0010FC3D022E0BEF1020F02D1002A83
:10180000BDD01CE0BEF1030F02D1002BB7D016E013
:10181000BEF1040F03D1BAF1000FB0D00FE0BEF15A
:10182000050F03D1B9F1000FA9D008E0BEF1060FF2
:1018300005D1B8F1000FA2D001E0002F9FD091F8A0
:1018400006B0BBF10F0F9AD81D930B790D93CB798E
:101850000E934B790F934B7A91F80DC010938B7ABE
:101860001193CB7A1293ACF1800C0B7B13930FFA8C
:101870008CF391F80EC01493ACF1800C0FFA8CF33A
:101880001593CB7B16930B7C17934B7C18938B7C17
:101890001993CB7C1A930B7D1C9271461B93FFF717
:1018A0007FFE4A491C9A1D9B494804F001040032FE
:1018B0000C70484918BF01220A700033464A18BF0D
:1018C000012313701AF1000A444B454A18BF4FF028
:1018D000010A83F800A019F10009424B18BF4FF02C
:1018E000010983F8009018F100083F4B18BF4FF032
:1018F000010883F8008000373C4B18BF01271F7098
:10190000EB43C3F3C0133146137002F09DFC314624
:10191000374802F01BFA3146364804F0ABFD314639
:101920003548FEF79DFD3146344807F037FC314617
:101930003348FEF75BFF5946324808F0E9FC594648
:10194000314806F06BFF0E992F4806F073FF594699
:101950002E4806F03DF859462D4802F069FE179AC8
:101960002348C5F3C00102F009FA1A99214804F08E
:1019700099FD1B99214807F029FCC5F340130B93EF
:10198000159B0A93149B0993199B0893189B079323
:10199000169B0693139B0593129B0493119B039331
:1019A000109B02930F9B01930D9B0093C5F3400284
:1019B000C5F3800305F00101164802F015F815483B
:1019C00001F0FEFD00201FB0BDE8F08F5D02002099
:1019D000DC1000205C0200205B0200205E02002080
:1019E000580200205A0200205F0200205902002005
:1019F000A89B00207834002054B00020480B002021
:101A00003C3100208C33002080130020B47B002068
:101A1000F839002000650020BFFD010008B5002A4C
:101A200032D01A4B09781B788B422BD006290CD95F
:101A30000A2922D0A1F15B03DBB2102B24D8144A6F
:101A400022FA03F3DB071BD41EE0012901D1114B5D
:101A500014E0022901D1104B10E0032901D10F4BF2
:101A60000CE0042901D10E4B08E0052901D10D4BF2
:101A700004E0062904D10C4B00E00C4B1B781BB191
:101A8000FFF78EFD002008BD042008BD883300202C
:101A9000BFFD01005D0200205C0200205B0200200F
:101AA0005E0200205A0200205F020020590200203E
:101AB00070B590F80231A4B023B3E0238DF80C3058
:101AC000F2238DF80E300025ECB2E31C0E5D0DF113
:101AD000900E01355EFA83F316B103F8846CF3E7D8
:101AE000111203F8841C631D24A9043451FA84F4F0
:101AF000012104F8842CDBB2009103AA8DF80D308B
:101B000008F0F9F824B070BD2DE9F043B64DB74F99
:101B100085B004462E460121204608F0CBF88046C9
:101B2000002800F0E1820121204608F0DAF894F85C
:101B3000002152B9E02803BF0123207084F800314E
:101B400084F8002184F80121E5E7012A06D1022367
:101B5000607084F8010184F80031DCE7A05402F1E0
:101B6000010894F801315FFA88F8434584F8008150
:101B7000D1D1A3781C2B00F0CB8129D8082B00F001
:101B8000988010D8022B56D008D8002B4FD0012BAC
:101B900040F06F822046FFF7A5F86EE2032B51D08C
:101BA000042B60D065E2112B00F0088106D80A2BC7
:101BB00000F0D780102B00F0E7805AE2182B00F0DD
:101BC0004C811A2B00F06381132B40F0528231E1DB
:101BD000502B00F0278214D8202B00F0BF8106D8AC
:101BE0001D2B00F071811E2B00F0A58141E2312BED
:101BF00000F0E881402B00F0FC81302B40F039826E
:101C0000C6E1622B27D004D8602B30D0612B3AD0AC
:101C10002FE2802B06D0C0F02C82903B012B40F2AB
:101C20002C8226E24FF0030804F5827913E2204665
:101C3000FFF772F921E2023AD2B2E11C2046FFF727
:101C400099FD05E0023AD2B2E11C2046FFF7E6FE1C
:101C5000014640B10EE2023A0B2A24D9E01CFEF7FD
:101C6000D5FF804608BB2046FFF70EF805E2023A92
:101C7000D2B2E11C2046FFF773F980460028F2D06B
:101C800002B25B490AE0023AD2B2E11C2046FFF7F9
:101C9000A9F980460028E6D0564902B25648FFF717
:101CA00007FF4146E6E14FF004080FFA88F2534976
:101CB000F4E72B78632B07D1023AD2B2E11C5048EB
:101CC00007F014FC804601E04FF0020833785C3BDB
:101CD000DBB2062B0DD84D2222FA03F3DB0708D521
:101CE00094F801214748033AD2B2E11C06F088FF7C
:101CF00080463378663B052B08D894F8012142488A
:101D0000033AD2B2E11C06F0B9F8804633785D2B75
:101D100008D194F801213D48033AD2B2E11C06F003
:101D2000B5FF804633785B2B08D194F80121384801
:101D3000033AD2B2E11C00F06DFB80463378652B8C
:101D400008D194F801213348033AD2B2E11CFEF7DE
:101D500065FC8046B8F1000F85D00FFA88F22E4955
:101D60009CE72B7853B9023AD2B2E11C2B4807F01A
:101D700039FC8046002800F0808101E04FF0050822
:101D80000FFA88F2264989E7264B1B7883B12B7816
:101D9000012B0DD8023AD2B2E11C234802F028F8F8
:101DA000804638B92B78002B40F0678101216AE02A
:101DB0004FF002080FFA88F21C496FE7194B1B78A5
:101DC00063B12B78012B09D8023AD2B2E11C164834
:101DD00002F034F880460028E4D001E04FF0020819
:101DE0000FFA88F2124959E7883300205C0200207C
:101DF0005BDD000878DD00082830002095DD000854
:101E000050B0002024B000208C610020A4A000204D
:101E1000FD640020460B0020B2DD000858070020BA
:101E2000D4DD00085D020020DC100020E7DD0008A2
:101E300006DE0008944B1B784BB12B78012B06D89B
:101E4000924802F021F880460028ABD001E04FF024
:101E500002080FFA88F28E4920E73B7873B32B789B
:101E600013F0FD0F2AD18B4B1B783BB3023AD2B251
:101E7000E11C894807F0DAFF804608BB2B78002B6D
:101E800040F0FB8002212046FFF78AFBF5E03B781B
:101E9000A3B12B7813F0FD0F10D17E4B1B78023AC3
:101EA000E11CD2B21BB17C4807F0EAFF02E07B489C
:101EB000FEF722FA804618B93378E0E74FF00208BF
:101EC0000FFA88F27649E9E63B78E3B1B8F1040FFE
:101ED00040F04281E178012908D12B78022B14D1FE
:101EE000704B1B78002B40F0C88008E069B92B7854
:101EF000022B0AD16B4B1B78002B00F0BE8066488A
:101F000008F03AF8B9E04FF0020842466649C5E6E3
:101F10003B7853B1023AD2B2E11C5F4807F0DEFFD2
:101F20008046002800F0A98001E04FF002080FFA77
:101F300088F25E49B2E63B7853B1023AD2B2E11C74
:101F4000554808F003F88046002800F0968001E02C
:101F50004FF002080FFA88F255499FE6554B1B785F
:101F600083B12B780BB1032B0CD1023AD2B2E11C16
:101F7000514801F0F5FD804630B93378002B7CD113
:101F8000032180E74FF002080FFA88F24B4985E6FB
:101F90004B4B1B7883B12B7813F0FB0F0CD1023A1B
:101FA000D2B2E11C474804F069F9804630B92B7879
:101FB000002B62D1042166E74FF002080FFA88F285
:101FC00041496BE63E4B1B786BB12B7813F0FB0F4E
:101FD00009D1023AD2B2E11C3A4804F04FF98046E6
:101FE0000028E4D001E04FF002080FFA88F23749E8
:101FF00054E6374B1B787BB12B780BB1052B0BD1FB
:10200000023AD2B2E11C334806F0CAFF804628B932
:10201000337893BB052136E74FF002080FFA88F2B8
:102020002D493BE62D4B1B787BB12B780BB1062B52
:102030000BD1023AD2B2E11C2948FEF736FB8046AA
:1020400028B93378CBB906211DE74FF002080FFA03
:1020500088F2244922E694F8013143450DD914F859
:102060000810484608F1010804F076FA5FFA88F88B
:10207000F1E701212046FEF71DFE002384F8003120
:1020800084F8013147E500BF5D020020DC1000202C
:1020900023DE0008580200208C33002054B00020BA
:1020A0003FDE0008FC64002059DE000874DE0008F2
:1020B00092DE00085B020020A89B0020ADDE000835
:1020C0005E02002078340020D1DE0008EDDE00083A
:1020D0005A020020480B002006DF00085F020020A3
:1020E0003C31002021DF00081E4801F0F8FC4BF6CF
:1020F0007F33984204F5827784BF84F8008184F8A6
:102100000181384604F008FA0646D8B1032120467A
:1021100007F0DDFD0025B042B8BF86B2A846ABB2DD
:102120009E420FD9384604F03DFACDF800808DF874
:102130000F0001230DF10F020321204607F0DBFD04
:102140000135ECE70321204607F0B4FD38B1032147
:10215000204607F0C6FDF5E74FF00408D5E605B0C8
:10216000BDE8F08300650020F0B51F4690F802310D
:10217000A5B083B3E0238DF80C30F3238DF80E3037
:102180000026F4B2E51C0B5D0DF1900E01365EFAEF
:1021900085F513B105F8843CF3E7131205F8843C88
:1021A000211D24AB53FA81F101F8842C621D53FAEE
:1021B00082F23B1202F8843CE21DD3B2063424AA18
:1021C00052FA84F4012104F8847C03AA00918DF86A
:1021D0000D3007F090FD25B0F0BDF0B590F802414C
:1021E000A5B0BDF9A860002C3ED0E0248DF80C40CD
:1021F000F4248DF80E400027FCB2E51C11F804E031
:102200000DF1900C01375CFA85F5BEF1000F02D09C
:1022100005F884ECF0E7111205F8841C24AD211DAB
:1022200055FA81F101F8842C621D55FA82F21912D7
:1022300002F8841CA21D55FA82F2012102F8843CA6
:10224000E31D55FA83F3321203F8842C04F10903D9
:10225000083455FA84F4DBB204F8846C03AA0091C4
:102260008DF80D3007F047FD25B0F0BD2DE9F041A8
:1022700090F80241A4B0BDF9A870BDF9AC60002C83
:102280004ED0E0248DF80C40F5248DF80E404FF030
:10229000000E5FFA8EF4E51C11F804C00DF19008F1
:1022A0000EF1010E58FA85F5BCF1000F02D005F8C9
:1022B00084CCEEE7111205F8841C24AD211D55FADB
:1022C00081F101F8842C621D55FA82F2191202F88C
:1022D000841CA21D55FA82F2012102F8843CE31D00
:1022E00055FA83F33A1203F8842C04F1080355FAE3
:1022F00083F3321203F8847C04F1090355FA83F363
:1023000003F8842C04F10B030A3455FA84F4DBB28D
:1023100004F8846C03AA00918DF80D3007F0EBFCF3
:1023200024B0BDE8F08100224FF480410280428059
:1023300081808271826002737047C9010180D2017D
:102340004942418082807047B0F9003030B583B394
:1023500082795AB98B4205DC0123837100238360A3
:10236000037303E0B0F902308B42F5DA837903B3EB
:102370008268B2F5166F13D8037B0F4DB0F90410C5
:102380005C1C55F82330E4B259430B2C4FEAE13181
:10239000047301F30F0109B203D90023037300E0B2
:1023A0000021531C42F6DF629342836084BF002306
:1023B0008371084630BD00BF98DF0008002202701C
:1023C000427082707047000010B504460F4806F056
:1023D00059FE0E4806F0F2FEB0B16378012B10D121
:1023E0000B4BA1780948312202FB013106F0D8FDE0
:1023F000A378013303F00303A370237823B9637038
:1024000010BD00236370A37010BD00BF480B0020F7
:10241000C8DF0008012A0BD10A78012A0CBF01236A
:102420000023037006D1437823B9427018467047E1
:10243000042070470020704700220260426070470D
:1024400018235A4345F6C05303FB0121016070472E
:1024500000681823B0FBF3F0704703680BB1012349
:102460004360704700234360704743681BB10268B4
:102470000AB10B44436070474068003018BF012028
:102480007047026832B1436833B19A422CBF0020D2
:102490000120704710467047184670470346F0B554
:1024A0008768C668056940699C69DA6999607843FC
:1024B00005FB010518681F6000FB045002FB1600B5
:1024C0005C681A6A5E6004FB1200C01300F30E0021
:1024D00000B2D860F0BD00001FB500F624140B4810
:1024E00001F01AF802280FD90DF10E01204606F06E
:1024F0002AFA48B1002300930DF10E0201230A21AC
:10250000024800F0A9FFEAE704B010BD0065002012
:10251000002310B5044680F8343800F63800FFF781
:10252000A1FF04F50460FFF79DFF04F50560FFF7C8
:1025300099FF04F65800FFF795FF04F50660FFF7D2
:1025400091FF04F66800FFF78DFF04F50760FFF7C1
:1025500089FF04F50060FEF743F804F58060FEF79C
:102560002DFB2046FEF72AFB04F6280000F0C2FDF2
:1025700004F62410BDE8104006F00ABA2DE9F74F22
:102580009DF834409DF830509DF83CB0C4EB0414E5
:102590009946A4009DF838300193A4B29DF84830C4
:1025A00080F837380F4690469DF840109DF844203B
:1025B00080F8351800F6480A80F8362806460022CA
:1025C00021465046FFF73CFFC5EB0511890089B253
:1025D000002206F63800FFF733FF14B15046FFF72C
:1025E0003CFF019B0C9342464B4639463046CDF8A2
:1025F00034B003B0BDE8F04FFEF7C2B92DE9F047A3
:10260000BDF824709DF820609DF828500446884647
:10261000914600213A4600F506609A46FFF710FF02
:102620002EB13A46314604F65800FFF709FF0995E6
:10263000089553464A46414604F58060BDE8F04798
:10264000FEF79EB92DE9F74F04469DF844E09DF84A
:10265000480084F8F4E815461E469DF84C209DF885
:102660003830009384F8F5089DF83C30A4F8F6283B
:1026700004F5046000229DF830709DF834800193C9
:102680009DF840B09DF850A09DF85490FFF7D8FEFB
:10269000019B0022194604F50560FFF7D1FE0022D8
:1026A000594604F66800FFF7CBFE294604F62800D9
:1026B00000F0EEFC2A46514604F6E400FFF73DFE2A
:1026C000A4F8109943463A46314604F50060FDF7F8
:1026D000E3FE40B9009A314604F5026003B0BDE85C
:1026E000F04FFEF7D1B803B0BDE8F08F38B504461F
:1026F0000D4600F63800FFF7B8FE294604F50460E1
:10270000FFF7B3FE294604F64800FFF7AEFE294660
:1027100004F50560FFF7A9FE294604F65800FFF707
:10272000A4FE294604F50660FFF79FFE294604F63D
:102730006800FFF79AFE294604F50760BDE83840B7
:10274000FFF793BE38B500F6480504462846FFF764
:1027500093FE78B12846FFF794FEA0B10A490B48D2
:10276000FEF7FCFE2046FEF742FA2846BDE8384058
:10277000FFF773BE05480449FEF7F0FE2046BDE8AA
:102780003840FEF734BA38BD8CE00008283000200D
:1027900070B504460E4600F50565E1B12846FFF721
:1027A00070FEB0B31B491C48FEF7D8FE022384F824
:1027B00034382846FFF756FE94F835384BB394F872
:1027C000373833B32046FFF7BDFF04F63800BDE8C5
:1027D0007040FFF742BE114800F0A2FE31460F489C
:1027E00000F0ACFE0E490C48FEF7B8FE284684F80F
:1027F0003468FFF737FE04F50460FFF733FE04F694
:102800005800FFF72FFE04F63800BDE87040FFF7D0
:1028100029BE70BD9AE00008283000200065002025
:10282000ACE0000838B504460D4651B100F504652A
:102830002846FFF721FEB0B12846FFF722FEE8B98F
:1028400011E01C4800F06CFE29461A4800F076FEA4
:1028500019481A49FEF782FE032384F8343804F538
:102860000660FFF7FAFD04F638052846FFF704FE78
:10287000F8B12846FFF705FE98B938BD10490E4853
:10288000FEF76CFE042384F8343804F65800FFF792
:10289000E9FD2846FFF7E6FD04F6280000F024FCD9
:1028A000E1E72046FFF74EFF2846BDE83840FFF736
:1028B000D4BD38BD0065002028300020BFE00008EE
:1028C000D6E0000870B5044600F5066691B1012116
:1028D0002A4800F025FE0121284800F02FFE284953
:1028E0002848FEF73BFE022384F834383046FFF7D1
:1028F000B9FD23E03046FFF7BFFDF8B13046FFF7E2
:10290000C0FDD8B11F482049FEF728FE04F658053F
:10291000062384F834382846FFF7AEFDC8B12846B0
:10292000FFF7AFFDA8B93046FFF79CFD04F5046042
:10293000FFF798FD04F66800FFF78FFD04F63805F1
:102940002846FFF799FDC0B12846FFF79AFD60B908
:1029500070BD0E490B48FEF701FE04F58060FEF7DE
:1029600046F92846FFF77EFDDDE72046FFF7EAFE41
:102970002846BDE87040FFF770BD70BD00650020BF
:102980009AE0000828300020F0E00008E7E00008A6
:1029900038B504460D4689B9124800F0C1FD2946F4
:1029A000104800F0CBFD10481049FEF7D7FD052375
:1029B00084F8343804F50660FFF74FFD04F6380557
:1029C0002846FFF759FD58B12846FFF75AFD38B1A0
:1029D0002046FFF7B7FE2846BDE83840FFF73DBD6B
:1029E00038BD00BF0065002028300020FEE0000850
:1029F00038B5044600F5066591B10121284800F07C
:102A00008FFD0121264800F099FD26492648FEF752
:102A1000A5FD042384F834382846FFF723FD07E09A
:102A20002846FFF729FD18B12846FFF72AFD50B9BF
:102A300004F638052846FFF71FFD78B32846FFF750
:102A400020FD18BB38BD19491748FEF787FD06233E
:102A500084F8343804F6280000F04CFB144912487E
:102A6000FEF77CFD04F58060FEF7C1F82846FFF70D
:102A7000F9FC04F65800FFF7F5FC04F50460FFF7D5
:102A8000F1FC04F66800FFF7E8FCD1E72046FFF709
:102A900059FE2846BDE83840FFF7DFBC38BD00BF0F
:102AA00000650020D6E0000828300020F0E0000893
:102AB000E7E0000810B5044600F50460FFF7CDFC20
:102AC00004F65800BDE81040FFF7C7BCF8B504464F
:102AD0000F4600F63805D1B10121244800F020FD51
:102AE0000121224800F02AFD21492248FEF736FD47
:102AF000022384F8343820491E48FEF72FFD04F5E0
:102B00008060FEF75BF82046FFF7D4FF1BE000F67D
:102B100068063046FFF7B0FCA8B13046FFF7B1FCBD
:102B200088B116491348FEF719FD84F83478304609
:102B3000FFF798FC94F8363813B12046FFF702FEF1
:102B40002846FFF78FFC2846FFF796FC60B1284621
:102B5000FFF797FC00B9F8BD2046FFF7F3FD2846C4
:102B6000BDE8F840FFF779BCF8BD00BF0065002064
:102B70009AE000082830002014E10008ACE00008CA
:102B800070B518254D43002400F61416AC4205D04C
:102B90000021304605F0B4FE0134F7E770BD0000B7
:102BA000F8B50446FDF7CBFE04F58060FDF7C7FEDF
:102BB00004F50060FDF763FC04F502600025FDF7F5
:102BC0005EFE04F6280000F05BFA84F8345884F8BE
:102BD000355884F8365884F8375804F63800FFF72B
:102BE0002BFC04F50460FFF727FC04F64800FFF710
:102BF00023FC04F50560FFF71FFC04F65800FFF7FF
:102C00001BFC04F50660FFF717FC04F5076704F6E4
:102C10006800FFF711FC3846FFF70EFC4FF43573E0
:102C2000C4F88838C4F890384FF4B562334BC4F810
:102C30008C28C4F89438324AC4F8B42845F2683372
:102C4000C4F898382F4AC4F8B8284FF40043C4F8A1
:102C5000AC38C4F8D038C4F8D83844F66C222A4BC3
:102C6000C4F8BC28C4F8DC38284AC4F8D42847F68D
:102C7000E423C4F8E0380126C4F88058C4F8785832
:102C8000C4F88458C4F87C58C4F8B058C4F8A458A0
:102C9000C4F89C58C4F8A858C4F8A058C4F8C85838
:102CA000C4F8C058C4F8CC58C4F8C45804F6E400BA
:102CB000FFF739FB84F8F46884F8F558A4F8F6684F
:102CC000802104F6F800FDF7A6FDA4F810694FF482
:102CD000965104F6141005F0C3FD4FF4166104F686
:102CE000241005F0BDFD962229463846FFF7A8FBC3
:102CF00020466421FFF744FF2046F8BDF96BFFFF33
:102D00000080FFFF5D3BFFFFB505FFFF0000FFFFF9
:102D100070B518254D43002400F62416AC4205D0AA
:102D20000021304605F0ECFD0134F7E770BD0000EE
:102D300038B50446002942D000F505652846FFF75E
:102D400087FB98B11E491F48FEF708FC012384F851
:102D500034382846FFF781FB94F835388BB194F866
:102D6000373873B92046FFF7EDFC0AE016491548DD
:102D7000FEF7F4FB022384F8343894F83538002B3E
:102D8000F0D132212046FFF7C3FF2046FFF792FE25
:102D900004F63800FFF761FB04F50760FFF762FBFC
:102DA00001210A4800F0BCFB0121084800F0C6FBE5
:102DB00007490448FEF7D2FB064B0A221A7038BDB9
:102DC0001DE10008283000209AE00008006500207E
:102DD0002FE1000888330020F8B590F83438044615
:102DE000062B19D8DFE803F004070A0D10131600AC
:102DF000FFF79EFF10E0FFF7CBFC0DE0FFF712FDA1
:102E00000AE0FFF75FFD07E0FFF7C2FD04E0FFF710
:102E1000EFFD01E0FFF75AFE94F83438002B4ED155
:102E2000274B1A780A2A1D4649D12046FDF7CFFEC6
:102E300050B904F58060FDF7CAFE28B904F50766AD
:102E40003046FFF719FBA0B12046FDF7C0FEB0BB2E
:102E500004F58060FDF7BBFE074680BB04F50766FE
:102E60003046FFF709FB50B33046FFF70AFB20B9A5
:102E7000F8BD3046FFF7F1FAE6E712491248FEF7CF
:102E80006DFB04F638002F70FFF7ECFA04F50460D0
:102E9000FFF7E8FA04F50560FFF7E4FA04F65800D6
:102EA000FFF7E0FA04F50660FFF7DCFA04F66800C5
:102EB000FFF7D8FA3046BDE8F840FFF7D3BAF8BDBF
:102EC0008833002042E10008283000202DE9F04F2F
:102ED000984690F8F53887B004460E4615460BB173
:102EE00081F0010641462046FFF700FC634F05EBE9
:102EF000480804F5806904F6780A454500F0BA8070
:102F000035F9021BB4F91039090291FBF3F194F879
:102F1000F43809B2012BADF8161005D039D3022BC5
:102F200004F500601DD024E004F50060FDF7D4FA3C
:102F300006AB04F6141B33F9021D029058460193A8
:102F4000039305F0DDFC019B5846194605F0FBFC98
:102F5000029AD00702D43B780A2BCED1C2F34001AB
:102F600018E0FDF7B9FAC1070DD43B780A2BC4D19C
:102F700009E0FDF7B1FAC2073B7802D40A2BBCD1B5
:102F800007E00A2B05D010F0020F14BF31460021D4
:102F900000E031462046FFF71FFF3B780A2BACD1FB
:102FA00094F83438013B012B0CD8BDF9161004F607
:102FB000E400FFF7C9F9B4F8F63813FB00F0ADF8F8
:102FC000160002E00023ADF816302046FDF701FEA2
:102FD00038B94846FDF762FDBDF816301844ADF823
:102FE00016004846FDF7F5FD68B994F834382046D8
:102FF00013B9FDF753FD01E0FDF798FDBDF816305C
:103000001844ADF81600BDF916105046FFF746FA01
:10301000014604F69C00FFF741FA014604F50C60F6
:10302000FFF73CFAADF816002046FDF7D2FD18B9BF
:103030004846FDF7CEFD98B104F50760FFF71CFA8E
:10304000014604F50260FDF767FCBDF81610084460
:1030500001B204F62410ADF8161005F051FC4CE74F
:1030600004F6280000F018F8BDF816301844ADF842
:103070001600E1E707B0BDE8F08F00BF88330020FD
:103080004FF48042028000228270426002727047D8
:1030900001EB810101807047837810B50246FBB1D6
:1030A000446842F6DF639C4211D9017A0D4BB0F9B6
:1030B000000033F911304343DB1303F30F0318B25D
:1030C0004B1CDBB23B2B88BF0023137200E00020B7
:1030D000631C45F6BF518B4288BF0023536010BD6F
:1030E000184610BD58E10008012383700023436097
:1030F0000372704700238370704770B5044606253D
:10310000002686F001063146204603F007F83146D6
:10311000204603F013F83146204603F017F83146F5
:10312000204603F01BF83146204603F01FF83146D5
:10313000204603F023F83146204603F027F83146B5
:10314000204603F02BF83146204603F02FF8013DCE
:10315000FA21204603F032F815F0FF05D1D12046C0
:10316000012102F0F3FF2946204602F0F7FF29462D
:10317000204602F0FBFF2946204602F0FFFF2946C9
:10318000204603F003F82946204603F007F82946B5
:10319000204603F00BF82046FA2103F00FF82046F2
:1031A000012102F0DBFF2046FA2103F007F8204658
:1031B000012102F0DBFF2046FA2102F0FFFF20464A
:1031C000012102F0DBFF2046FA2102F0F7FF204642
:1031D000012102F0DBFF2046FA2102F0EFFF20463A
:1031E000012102F0DBFF2046FA2102F0E7FF204632
:1031F000012102F0DBFF2046FA2102F0DFFF294621
:10320000204602F0D3FF2046FA2102F0D7FF2946DC
:10321000204602F0C3FF2046FA2102F0CFFF2946E4
:10322000204602F0B3FF2046FA2102F0C7FF2946EC
:10323000204602F0A3FF2046FA2102F0BFFF2946F4
:10324000204602F093FF2046FA2102F0B7FF2946FC
:10325000204602F083FF2046FA2102F0AFFF294604
:103260002046BDE8704002F071BF00002DE9F74F25
:10327000002504464FF4167100F8045B05F018FDB4
:103280004FF4FA7104F1180005F012FD4FF41671B5
:1032900004F12C0004F0F9F81022294604F13C0056
:1032A00009F06AFD04F1980B04F14C030093E56406
:1032B00025656565A565A4F85C5025666566A4F876
:1032C0006850E5662567A4F87450A567E567A4F81B
:1032D0008050C4F88450C4F88850A4F88C50C4F8C6
:1032E0009050C4F8945004F592795B4623F8025B41
:1032F0004B45FBD104F5BA784B46002223F8022B4C
:103300004345FBD104F5D8774346002223F8022B2E
:10331000BB42FBD104F523763B46002223F8022B67
:10332000B342FBD104F541723346002123F8021B5E
:1033300093424FF00005F9D14FF48043A4F80633CF
:10334000A4F80833A4F80A33A4F80C33A4F80E3315
:10335000A4F81033A4F81233A4F81433A4F81633E5
:103360004FF40063A4F81833A4F81A33012384F847
:103370002433294684F8045384F81C53C4F820539A
:1033800084F82553A4F82653A4F82853C4F82C53E2
:1033900084F830538C225846019309F0EDFC2946FD
:1033A0005022484609F0E8FC29463C22404609F0F4
:1033B000E3FC2946DC22384609F0DEFC2946782267
:1033C000304609F0D9FC10222946009809F0D4FCB7
:1033D000019BE363009B2364194B63642A23A4F8D5
:1033E0005C30184B63660C23A4F86830164B2367D7
:1033F0000623A4F87430154BE3675223A4F88030F9
:10340000134BC4F888302023A4F88C30114BC4F837
:103410009430204684F84850C4F860B0C4F86C90EA
:10342000C4F87880C4F88470C4F8906002F082FC1C
:103430002046FFF762FE204603B0BDE8F08F00BFD4
:10344000680100208C0100206A000020800100201B
:1034500082000020260100202DE9F04799460378DC
:10346000089E04460D469046002B51D090F830330C
:10347000002B4DD1274B1A7832B990F80413012252
:1034800051401A7002F052FE691E09291BD8DFE86C
:1034900001F005080B0E11141A1A1A17B4F90A5381
:1034A00013E0B4F90C5310E0B4F90E530DE0B4F985
:1034B00010530AE0B4F9125307E0B4F9145304E0CE
:1034C000B4F9165301E0B4F908534FF0000A04F1BF
:1034D0001807D1451CD038F91A10B4F81A336943CB
:1034E000C91301F30F01194489B2B1F5805F22BFFE
:1034F000B4F828330133A4F828330EB9324601E07A
:1035000016F80A20384605F028FC0AF1010AE0E71F
:10351000BDE8F087FC640020183005F0DCBB00003B
:1035200038B5054B1A788A420D461C4601D002F088
:1035300005FE257038BD00BF8933002080F82513B3
:103540007047000038B51D4C21784B1E5942594137
:10355000054602F0FBFD21788A1E51425141284662
:1035600002F0FCFD2178C81E41424141284602F08C
:10357000FDFD2178A1F1040EDEF1000141EB0E0109
:10358000284602F0FBFD2178A1F1050CDCF10001D9
:1035900041EB0C01284602F0F9FD21788B1F5942BE
:1035A0005941284602F0FAFD2178A1F10A02514260
:1035B00028465141BDE8384002F0F8BD883300206C
:1035C000037810B5044643B902F0ACFC0123237024
:1035D0002046BDE81040FFF7B5BF10BDF0B5D0F8EC
:1035E0002033027801338DB00446C0F820337AB31B
:1035F000D0F82C234BF67F339A4216D9A74B1A7872
:10360000511E05291D460DD8022A06D1A44B1B7850
:103610001BB10021A34806F0AFFC002320462B700D
:10362000FFF790FF0023C4F82C33D4F8202345F68D
:10363000BF539A421BD994F82413002381F001014F
:10364000C4F8203384F82413204602F067FD0EE00E
:1036500095498B4240F2B38190F82413C0F820239F
:1036600081F0010180F8241302F058FDA7E194F8DD
:103670001C3323B1204602F045FD84F8300304F1E9
:10368000180005F04AFB20B9854B1A78002A40F053
:103690008F81271D384605F040FB012840F28F81BD
:1036A000002502AB5A190AA9384605F07DFB04AB88
:1036B00003EB450104F12C0003F05AFF94F8253385
:1036C0005BB1BDF828301BB140F6FF72934204D1C4
:1036D000B4F826330133A4F82633B4F81823BDF820
:1036E00028309B1AB4F906231BB203AE5343DB13F5
:1036F00003F30F0326F815300135022DD1D194F8CC
:103700003033002B40F05B812A4608A9304608F090
:103710003DFD2B460AAA08A904F13C0009F0BEF8B9
:103720000A9A0B9B1344BDF80C2093FBF5F31B1472
:1037300003F30F039BB2D21AADF81420BDF80E208C
:10374000D31AADF81630554B1B78002B67D1574B69
:103750001B7863B12B4607AA05A904F1680008F09D
:1037600041FF2B4604AA07A9514804F0C7FF514B5B
:103770001B7863B1022307AA05A904F1740008F0BD
:1037800031FF022304AA07A94B4802F073FA4B4BFE
:103790001B789BB1022306AA05A904F1800008F05A
:1037A00021FF022307AA06A904F18C0008F01AFFE2
:1037B000022304AA07A9424801F05CFC414B424F96
:1037C0001A781D460AB93B78FBB1022307AA314695
:1037D00004F15C0008F006FF3B782BB1022304AA39
:1037E00007A93A4803F0FEFD2B7873B1384B1B78DC
:1037F0002BB1022207A9374800F00CFF05E0022395
:1038000004AA07A9344804F099FA344B1B78002B1A
:1038100000F0D580204602F075FC0223ABE0012BBE
:1038200012D1224B1B78002B00F0C9802B4607AA2F
:1038300005A904F1680008F0D5FE2B4604AA07A9E3
:103840001B4804F05BFFBAE0022B4BD11D4B1B78E9
:10385000002B00F0B4802B4607AA314604F15C002F
:1038600008F0C0FE1A4B1B7883B10D4B1B783BB19F
:10387000009502AB04AA07A9194804F097FF9EE03F
:103880002A4607A9134800F0C5FE98E02B4604AA73
:1038900007A9114804F052FA91E000BF88330020D4
:1038A000FC6400208C3300207FA903005D0200200F
:1038B0009C6100205E020020483F00205A02002048
:1038C000A8A000205C0200205B02002034680020D9
:1038D00058020020F8390020B47B00205902002053
:1038E00080130020032B11D1364B1B78002B66D0A0
:1038F0002B4607AA05A904F15C0008F073FE2B46CD
:1039000004AA07A9304803F06DFD58E0042B11D13B
:103910002E4B1B78002B52D02B4607AA05A904F189
:10392000740008F05FFE2B4604AA07A9284802F09D
:10393000A1F944E0052B18D1264B1B78002B3ED073
:103940002B4606AA05A904F1800008F04BFE2B4681
:1039500007AA06A904F18C0008F044FE2B4604AA2D
:1039600007A91D4801F086FB29E00A2B09D1204652
:1039700002F0C8FB2B46014605AA1848FFF7A6FA35
:103980001DE0632B0CD107AA314604F16800022325
:1039900008F028FE022207A9114801F02DF80EE0D8
:1039A000602B0CD1022204A90E4805F01DFC06E094
:1039B000187094F80413204602F0B8FB69E60DB0C5
:1039C000F0BD00BF5B020020346800205E020020D2
:1039D000483F00205A020020A8A00020709200203A
:1039E000747B00207C3300202DE9F0419DF8388065
:1039F00080F804334FEAC818A0F81683BDF9408058
:103A00009DF81C309DF818C09DF820E09DF82470AA
:103A10009DF828609DF82C509DF8304008F500680E
:103A2000DB01A0F81883BDF93C80A0F808339DF8AD
:103A3000343008F500684FEACC1C4FEACE1EFF0177
:103A4000F601ED01E401DB01A0F81A839DF8448042
:103A5000A0F806C3A0F80AE3A0F80C73A0F80E6360
:103A6000A0F81053A0F81243A0F8143380F81C8378
:103A700019B1CCF1000CA0F806C392B1CEF1000E42
:103A80007F4276426D4264425B42A0F80AE3A0F8AE
:103A90000C73A0F80E63A0F81053A0F81243A0F81E
:103AA0001433BDE8F081B0F82633003318BF01238A
:103AB0000B70B0F82833003318BF012313700023B4
:103AC000A0F82633A0F828337047183005F092B9D3
:103AD000043005F08FB90023C0F82C337047D0F8BC
:103AE0002C03704790F830037047000038B54FF44E
:103AF0007A61044604F11C0502F0DAFC002222611E
:103B00006261A26104F13C012B4623F8022B8B4237
:103B1000FBD104F2EC42002003F8010B9A424FF073
:103B20000001F9D1F023A4F8F0344FF49653C4F80F
:103B3000F434A4F8EC14A4F8EE1484F8F214C4F8E5
:103B4000F8142022284609F017F9052323740923C5
:103B50006382024B6361A561204638BDE00100200D
:103B6000792A70B506460C460ED102F0B3FC7728D0
:103B70000CD904F1780514F8011F304602F0ECFC72
:103B8000AC42F8D1002070BD042070BD052070BD8E
:103B90002DE9F043DFF888C0DFF888E0DFF888809F
:103BA000DFF888908FB0002340F2772640F26577E7
:103BB00001F0C005802D90F8F22402AC0DD0C02D8C
:103BC00005D085B9002A14BF42464A460FE0002AB4
:103BD00014BF4FF46D723A4609E0002A14BF4FF447
:103BE0009E72324603E0002A14BF7246624624F8F1
:103BF000132001338900042BC9B2D9D104AA21466C
:103C0000103008F0F3FA0023009304AA14230321D0
:103C10000248FFF721FC0FB0BDE8F08300650020EB
:103C20009BF8FFFF4CFCFFFFC4FEFFFF89FDFFFF79
:103C300010B58EB0002404AA02A904231030029407
:103C4000039408F0D3FA0094142304AA0321024831
:103C5000FFF702FC0EB010BD00650020B0F8EC3498
:103C600070B504462BB13648364EFFF755FC054675
:103C700013E002F051FC60B1334B1B78002B4DD1A7
:103C8000B4F8F05477219AB295423DD80023A4F8B5
:103C9000EE34B4F8EC340BB3E5E7142D4FD9B4F897
:103CA000EE345A1C2344A4F8EE2493F83C1020462A
:103CB000FFF76EFF3378143DADB21BB1D4F8F43486
:103CC000C4F8F834B4F8EE24B4F8EC349A42E4D3EF
:103CD0000023A4F8EE34A4F8EC3470BDD4F8F83422
:103CE0006BB31748FFF718FC0546142D27D920465B
:103CF000FFF79EFFD4F8F834143D013BADB2C4F891
:103D0000F834002BF1D170BDB4F8EC24501C2244DF
:103D1000A4F8EC04013382F83C10B4E7782520467F
:103D200002F040FCB4F8EC34013D5A1C234415F079
:103D3000FF05A4F8EC2483F83C00F0D1A6E770BDA1
:103D40000065002058020020FC64002001EB4101C6
:103D5000890001F5167189B2B1F5966F8ABF4FF4EB
:103D60009663A0F8F014A0F8F034704708B502F09C
:103D7000B1FB7823B0FBF3F0C0B208BD4FF49663FB
:103D80005A4380F8F214C0F8F424704738B54FF461
:103D9000B971044604F11C0502F08AFB002222617D
:103DA0006261A26104F144012B4623F8022B8B428D
:103DB000FBD104F52772002003F8010B9A424FF063
:103DC0000001F9D13C23A4F8A032A4F89C12A4F875
:103DD0009E122822284608F0CFFF052323740323D0
:103DE0006382024B6361A561204638BD3A02002020
:103DF000292A70B506460C4619D102F06BFB29281A
:103E000006D802B20B490C48FDF752FE052070BDE2
:103E10000021304602F0A0FB651E283415F8011F72
:103E2000304602F099FBA542F8D1002070BD042075
:103E300070BD00BFF8E60008283000200C2A70B5DD
:103E400006460C4619D102F045FB0C2806D802B2F2
:103E50000B490C48FDF72CFE052070BD01213046B2
:103E600002F07AFB651E0B3415F8011F304602F094
:103E700073FBA542F8D1002070BD042070BD00BFC7
:103E800018E700082830002010B5044602F022FB95
:103E9000024628B905490648FDF70AFE052010BD6F
:103EA0000221204602F058FB002010BD36E7000832
:103EB000283000202DE9F04F002397B0184601ACC0
:103EC000D05418550133532BF9D10020DFF8C0E14D
:103ED0000139044605464FF0010C11F8018F2346C5
:103EE00006462C4600270CFA07F518EA050F14BF02
:103EF0000125002503EB050923442B44DB0709F0CA
:103F000001090CD506F007031EF803B016AB03EB4E
:103F1000D60313F854AC4BEA0A0A03F854ACB9F1CF
:103F2000000F0ED0731C0DF1580909EBD30903F0F3
:103F300007031EF803A019F8543C4AEA030309F8E2
:103F4000543C0137082F06F10206234601D02C46C7
:103F5000C9E71030B0F5287FBFD14B4F002138465C
:103F6000012407EB41030733B1F5257F7ED216AD5F
:103F700005EBD10515F8545C2E060BD513F8066C2D
:103F800013F807CC04FA06FE12F80C604EEA060697
:103F900002F80C606E060BD513F8046C13F805CC10
:103FA00004FA06FE12F80C604EEA060602F80C60EF
:103FB000AE060BD513F8026C13F803CC04FA06FE18
:103FC00012F80C604EEA060602F80C60EE060AD5FE
:103FD0001E7813F801CC04FA06FE12F80C604EEAC3
:103FE000060602F80C600E1DB6F5257F03F10803E6
:103FF00001D33146B8E72B070BD510F816E000EBDC
:104000004606737804FA03F612F80E30334302F8CA
:104010000E306B070CD54B1D10F813E000EB43037B
:104020005B7804FA03F612F80E30334302F80E30D0
:10403000AE070CD58B1D10F813E000EB43035B7843
:1040400004FA03F612F80E30334302F80E30EB0791
:104050000AD5CB1D10F8136000EB43035B7804FA1C
:1040600003F5935D2B43935508317AE7074C013AEA
:10407000002312F8010F195D01334140532B1170D9
:10408000F7D117B0BDE8F08FD0E1000867E700086E
:1040900053E7000870B500239AB00C46012240F2A5
:1040A00049354FF6B74632EA040102A94FEA420207
:1040B0000CBF21F8136021F813500133082BD2B242
:1040C000F1D106AA103008F091F80023009306AA57
:1040D000282301210248FFF7BFF91AB070BD00BFC5
:1040E0000065002070B5A2B0044602F015FA20B9B0
:1040F000B4F89C32002B00F09E80204602F04DFA6E
:10410000B4F89C5200283BD1002D3CD14B4B1B787E
:104110007BB9B4F8A052AA219AB2AA424BD2B4F801
:104120009C22501C2244A4F89C02013382F84410C3
:10413000F2E7204602F036FA204602F033FA01A9EF
:1041400048550135292DF7D10DF132022046FFF7F0
:10415000B1FEEA238DF83030B4F89C22A6238DF806
:10416000313000230CA8D118185C14FA81F1013306
:10417000552B81F84400F5D15532A4F89C221AE061
:1041800001281CD125B12E48FFF7C6F9054638E0B5
:10419000204602F007FA0C25B4F89C62731CA4F8C0
:1041A0009C32204602F0FEF92644013D15F0FF0541
:1041B00086F84400F0D10023A4F89E321DE00228C6
:1041C0001BD1002DDFD1204602F0ECF9B4F89C326F
:1041D0001C4D03F1120189B200229818565D14FAA1
:1041E00080F00132062A80F84460F6D106339BB293
:1041F0009942F1D1A4F89C12DDE7B4F89C32D3B116
:10420000C1E7282D17D9B4F89E325A1C2344A4F8CC
:104210009E2293F844102046FFF73CFFB4F89E22FC
:10422000B4F89C32283D9A42ADB2EAD30023A4F8F8
:104230009E32A4F89C3222B070BD00BFFC64002006
:10424000006500205BE7000801EB4101490001F532
:10425000967189B2B1F5167F8ABF4FF41673A0F834
:10426000A012A0F8A032704708B502F033F90D2370
:10427000B0FBF3F0C0B208BD30B5034600F1140244
:10428000002143F8041B9342FBD100F23C5400256B
:1042900023F8025B9C424FF00002F9D142F20F7307
:1042A000A0F83C25A0F83E25A0F84035C0F84425EC
:1042B000A0F84825A0F84A2580F84C2530BD0023F9
:1042C000A0F83E35A0F83C35C0F84435A0F84A3592
:1042D000A0F8483542F20F73A0F84035704700004F
:1042E0002DE9F047BDF82060BDF928C0BDF9248054
:1042F00006EB4202B51C741C0232344EADB2A4B2BD
:1043000092B2CCF10009A5F1020EAA421FFA8EFE6C
:1043100059D000EB4107B7F814A0C8EB0A0A0FFA0E
:104320008AFACA454FEAEE070EF0070E0FDA16F8C2
:104330000EA013F807E02EEA0A0E03F807E004F0D7
:10434000070EE71016F80EA013F807E027E0BAF101
:10435000000F0FDA16F80EA013F807E02EEA0A0E87
:1043600003F807E004F0070EE71016F80EA013F8A4
:1043700007E011E0E24516F80EA013F807E04AEA5C
:104380000E0E03F807E004F0070E4FEAE40716F8F4
:104390000EA013F807E002DA2EEA0A0E01E04AEA5C
:1043A0000E0E03F807E001F1050E1FFA8EF7B7F5C0
:1043B000257F24BFA1F28F27BFB202350234ADB2F0
:1043C000A4B239469FE7BDE8F08700BFFCE70008CC
:1043D0002DE9F04FB0F83C2550F8223000294FEA83
:1043E0004303B8BF43F0010340F82230B0F83E3534
:1043F00000EB43030446998250F822307E4823F0B4
:104400007F4391B0584000F01FFF022800F29B80CC
:10441000B4F83E65794FDFF8F4C106F2212189B284
:10442000B1F5257F28BFA6F173024FF0000E2CBF17
:1044300092B20A464FF47A50754604EB42031EF9D5
:104440000C80B3F914309F42B8BF1F469842A8BFF2
:104450001846B8F1010F0AD0B8F1030F05D0B8F132
:10446000FF3F06D003EB430303E003EB4303ED1AE6
:1044700000E01D44531D9BB2B3F5257F28BFA2F277
:104480008F220EF1010E28BF93B2BEF1180F01D09A
:104490001A46D2E7D4F844359D4254DDC3195B1067
:1044A0000FFA83F8FB1A44F63147B1F5257F07FB75
:1044B00003F728BFA6F173014FF0040347F3CF378A
:1044C0000DF11C0A00934FF0180228BF89B2029721
:1044D000CDF8048053462046FFF702FF0026484AE5
:1044E000DFF82CB1B1461AF80600B35C0592034020
:1044F00016F80B00584000F0A1FE01364844072E84
:104500005FFA80F9059AEED1B9F1030F1BD83B464B
:1045100042463C493C48FDF727FEB4F83E35C4F816
:10452000445503F20D1292B2B2F5257F24BF6FF409
:10453000C3729B18A4F84885A4F84A7534BFA4F840
:104540004025A4F84035B4F83E25B4F840359342F0
:104550003CD1991D89B2B1F5257F28BFA3F28E21E8
:10456000B4F94A350293B4F9483501934FF0080382
:1045700028BF89B284220093204607ABFFF7B0FE24
:1045800006A804F03CFC0DF11B030DF11A020DF11D
:104590001D0106A804F060FC94F84C259DF81A3023
:1045A0009A420CD19DF81B30032B08D1C3238DF800
:1045B0001C3007AA222300211348FCF7F9FD42F220
:1045C0000F73A4F840350023C4F84435B4F83E35E1
:1045D00001339BB2B3F5257F28BF0023A4F83E35F5
:1045E000B4F83C3501339BB2042B88BF0023A4F8F8
:1045F0003C3511B0BDE8F08F6E28760080C1FFFF1A
:10460000C2E70008D0E700082830002004E80008CE
:10461000C9E7000870B505460C4601EB4206B442F6
:1046200005D034F9021B2846FFF7D2FEF7E770BD2C
:1046300080F84C15704700000148FCF70EBD00BF24
:104640002830002010B54348434CFDF75DFA43483D
:10465000FEF7C4FF424B1B782BB12378012B02D10C
:104660004048FFF73FFD404B1B7863B12378022B96
:1046700009D13E4B1B781BB13D4805F0F7FD02E028
:104680003C48FBF785FE3C4B1B782BB12378032B72
:1046900002D13A48FFF7E2FA394B1B782BB1237865
:1046A000042B02D1374801F067FE374B1B782BB142
:1046B0002378052B02D1354804F0E4FC344B1B78F9
:1046C0003BB12378062B40D03248FBF7E5FF0028AA
:1046D0003BD1314B1B782BB123780A2B02D12F48C9
:1046E000FDF7FAFE2378632B02D12D4804F0C4FDB8
:1046F00023785C3BDBB2062B07D84D2222FA03F36A
:10470000DB0702D5274804F051FA23785D2B02D14C
:10471000254804F093FA23785B2B02D12348FDF758
:1047200053FE2378652B02D12148FBF763FF2378E2
:10473000663B052B02D81F4803F026FB237843B9BC
:104740001D48BDE8104004F003BF1248FBF7F4FF1A
:10475000BFE710BD2830002088330020006500200E
:104760005D020020DC1000205C02002058020020C6
:104770008C33002054B000205B020020A89B002056
:104780005E020020783400205A020020480B0020EE
:104790005F0200203C31002059020020709200206E
:1047A00050B0002024B00020A4A00020FD64002010
:1047B000460B00208C6100205807002008B5FFF749
:1047C0003BFFFFF73FFFFCE708B5284803F061FB1C
:1047D0002748FFF7DBFA2748FFF74EFD264803F08E
:1047E000D9FF264805F0A2FA254802F0E6FE254842
:1047F000FBF750FD244802F09DFA2448FFF776F9B4
:10480000234800F063FD234801F0E8FC224800F053
:104810001FF9224804F074FB2148FBF70BFF2148E5
:10482000FEF7BEF9204800F055F8204804F020FDBE
:104830001F4804F0B3F81F4804F0FCF91E48FDF7C8
:10484000BDFD1E4803F094FA1D48FBF7CFFE1D483E
:1048500004F0C2FC1C4804F069FE1C48FCF7FAF99D
:104860001B48BDE80840FEF701BD00BF9C61002069
:10487000DC100020F8390020801300208C33002049
:10488000B47B002054B0002034680020A89B002096
:10489000483F002078340020A8A00020480B0020CA
:1048A0003C31002070920020747B002050B000202A
:1048B00024B00020A4A00020FD6400208C61002012
:1048C000460B00207C3300205807002028300020B1
:1048D00000650020002303600371836000F10C0277
:1048E00000F13C0122F8023B8A42FBD14FF0000369
:1048F00080F83C307047000037B5836890F83C2062
:1049000000294FEA4303B8BF43F001038360531CFF
:10491000DBB2172B00EB420280F83C3088BF00234B
:104920009181044688BF80F83C30806820F07F4346
:104930002D48584000F088FC022825D82B4A04F165
:104940000A0104F13A054FF47A5331F9020F824219
:10495000B8BF02468342A8BF03468D42F5D1D11AA3
:10496000052911DD00218DF800108DF802201112AB
:104970001A128DF801108DF80320694605221C4893
:104980008DF80430FCF792FDA06820F07F431948B1
:10499000584000F059FC022824D8144A04F10A01B6
:1049A0004FF47A533A3431F9020F8242B8BF0246CB
:1049B0008342A8BF03468C42F5D1D11A052911DDE7
:1049C00080218DF800108DF8022011121A128DF836
:1049D00001108DF803206946052205488DF8043042
:1049E000FCF764FD03B030BD68B4AA0080C1FFFFCE
:1049F00028300020974B5500F8B504460E46002598
:104A00001746ABB29F4222D936F915102379CA0F47
:104A1000934209D02368B3F5004F2ABF6FF4CC70DE
:104A200003F299131B1823602368227103F54C507D
:104A30003330B0F5803F01D2206006E0A3F54C434F
:104A4000CD3B23602046FFF757FF0135D9E7F8BD7E
:104A50000346002230B503F8022B00F1160123F8BB
:104A6000022B8B42FBD100F61674002523F8025B63
:104A7000A3424FF00002F9D142F20F73A0F8162FB3
:104A8000A0F8182FA0F81A3FA0F81C3FA0F81E3F6E
:104A9000A0F8203FA0F8223FC0F8242FA0F8282F2C
:104AA00080F82A2F00F62C7100F64C7421F8022BA6
:104AB000A1424FF00003F9D1A0F84C3F00F64E712F
:104AC00000F66E7421F8023B8C424FF00002F9D1DF
:104AD0006323A0F86E2F80F8703FC0F8742FA0F801
:104AE000782F30BD6322002380F8702F42F20F72BE
:104AF0000370A0F8183FA0F8163FC0F8243FA0F8B4
:104B00001A2FA0F81C2FA0F81E2FA0F8202FA0F815
:104B1000222FA0F84C3FA0F86E3FA0F8283F80F865
:104B20002A3FC0F8743FA0F8783F7047394BF7B57B
:104B30004FF47A5604464FF0000E30461F461FFAD7
:104B40008EF5AA421FD904EB4105B5F91650002D88
:104B500006DDAF42B8BF2F46A842A8BF284605E0F1
:104B6000AE42A8BF2E46AB42B8BF2B4601F10A05A4
:104B7000ADB2B5F5F06F24BFA1F276718DB20EF132
:104B8000010E2946DBE73A18334452105B10D51862
:104B90006D102EB2551B2DB21BB21F491F48019537
:104BA000009612B2FDF762FB94F8703F632B04F697
:104BB0002A7104F64A7009D10B4623F8026F984215
:104BC0005D84FAD1002384F8703F0BE004EB4302CC
:104BD0000133DBB20F2BA2F82C6FA2F84E5F84F8E2
:104BE000703FEFD80023A4F84C3FA4F86E3F1A465C
:104BF00031F8025F2A444D8C88422B4412B21BB21A
:104C0000F6D112111B11A4F84C2FA4F86E3F03B07B
:104C1000F0BD00BF80C1FFFF29E800082830002058
:104C20002DE9F04FBDF82440BDF92C80BDF9289046
:104C3000334D04F1020E01341FFA8EFEA4B24FF080
:104C4000000CC8F1000A1FFA8CF7AEF10206BA4256
:104C5000B6B252D900EB4107B7F816B0C9EB0B0B4F
:104C60000FFA8BFBD3454FEAE60706F007060CDA8E
:104C700015F806B0DE5D26EA0B06DE5504F00707E0
:104C8000E61015F807B09F5D21E0BBF1000F0CDACC
:104C900015F806B0DE5D26EA0B06DE5504F00707C0
:104CA000E61015F807B09F5D0EE0C34515F806B095
:104CB000DE5D4BEA0606DE5504F007074FEAE40620
:104CC00015F807B09F5D02DA27EA0B0701E04BEA0F
:104CD00007079F5501F10A07BEB2B6F5F06F24BF72
:104CE000A1F27676B6B20EF1020E02340CF1010C8E
:104CF0001FFA8EFEA4B23146A5E7BDE8F08F00BFD3
:104D000097E80008B0F8163F00EB43032DE9F04F99
:104D100004465888C0F3090080F4A67089B080F07A
:104D2000010000F091FA022800F2A480B4F8186F94
:104D30005248DFF850C106F22677BFB2B7F5F06FE0
:104D400028BFA6F15A024FF0000E2CBF92B23A468D
:104D500075464FF47A5104EB42031EF90C80B3F907
:104D600016309842B8BF18469942A8BF1946B8F104
:104D7000010F0AD0B8F1030F05D0B8F1FF3F06D0FC
:104D800003EB430303E003EB4303ED1A00E01D4490
:104D900002F10A039BB2B3F5F06F28BFA2F276725C
:104DA0000EF1010E28BF93B2BEF10A0F01D01A46D0
:104DB000D1E7D4F8243FAB425CDA94F8703F632B20
:104DC0000AD10B185B10A4F84C3FC31A44F63E10EE
:104DD0004343DB13A4F86E3FB7F5F06F28BFA6F18D
:104DE0005A07B4F96E3F029328BFBFB2B4F94C3FE3
:104DF000019300260DF11C094B460A220096394604
:104E00002046FFF70DFF23781D4ADFF87CB0B34240
:104E10000CBF4FF0010A4FF0030AB04619F8060024
:104E2000B35C0592034016F80B00584000F006FAF8
:104E300001364044032E5FFA80F8059AEED1D04542
:104E400018D80623A4F8283FB4F8183FA4F81E3F4A
:104E500003F21B7292B2B2F5F06F28BF653BC4F843
:104E6000245FA4F81A7F34BFA4F81C2FA4F81C3FB9
:104E7000012000E0002009B0BDE8F08F80C1FFFFF5
:104E800026E800081CE8000894E8000810B504466D
:104E9000FFF738FFA0B194F82A3F8BB9C4F8743FEC
:104EA000A4F8783F01211B48FEF73AFB012119487D
:104EB000FEF744FB632384F8703F052384F82A3F00
:104EC00094F82A3F13B1013B84F82A3F94F82A3F13
:104ED000012B1ED1B4F81E3F03F27F7292B2B2F5DD
:104EE000F06F28BF03F1FF32A4F8202F5A1C92B2B2
:104EF000B2F5F06F24BFA3F27F73A4F8223F4FF006
:104F0000010323704FF0000338BFA4F8222F84F868
:104F10002A3F10BD0065002010B50446B0F8780F98
:104F200058B1D4F8743FB3FBF0F3C3F3072081F812
:104F3000310081F83230332200E031220448FCF79E
:104F400063FA0023C4F8743FA4F8783F10BD00BF93
:104F50002830002030B5B0F8201FB0F8222FB0F86C
:104F6000183F914293B0044607D2994208D89A421A
:104F700006D32046FFF7C6FE02E09942F7D8F8E7CD
:104F8000B4F8182FB4F81C3F9A4269D1B4F8283FFE
:104F9000062B16D1B4F81E3F03F27F7292B2B2F51F
:104FA000F06F28BF03F1FF32A4F8202F5A1C92B2F1
:104FB000B2F5F06F2ABFA3F27F73A4F8222FA4F8F2
:104FC000223FC022B4F81A1F2046FFF7AFFDB4F904
:104FD0006E1FB4F94C3FB4F91E2F009121482249AD
:104FE000FDF7FBF8B4F96E3F0293B4F94C3F01931F
:104FF00008230093B4F81A1F05ABC0222046FFF720
:105000000FFEB4F8285F013DADB2A4F8285FDDB90A
:1050100016491448FCF7A2FA29461548FEF780FA0B
:1050200029461348FEF78AFA0E48FCF71FFA42F2A7
:105030000F73A4F81C3F6323257084F8703F84F835
:105040002A5FC4F8245F0BE06B1F5D425D4105A938
:1050500020468DF81450FFF75FFF0023C4F8243F6B
:1050600013B030BD283000204AE8000872E800087C
:10507000006500202DE9F8434FF0000904460F4673
:1050800090461E464D464E4540D038F81930D4F86B
:10509000742F37F919101344C4F8743FB4F8162F5D
:1050A000B4F8783F04EB42020133A4F8783F538808
:1050B0005B009BB20029B8BF43F001035380B4F8F2
:1050C000183F04EB43032046D9822378012B02D1F9
:1050D000FFF740FF01E0FFF7D9FEB4F8183F0133B6
:1050E0009BB2B3F5F06F38BFA4F8183FB4F8163F81
:1050F00028BFA4F8185F01339BB2092B94BFA4F812
:10510000163FA4F8165F09F10109BCE7BDE8F88372
:1051100010B5002303810446438101800373437368
:10512000084607F0F1FC6060204610BD4289038903
:1051300092B29BB29A42028803D1037B93B9104684
:1051400012E04189038989B29BB2994239BF038930
:105150004089438900893ABF12FA80F0C01A181AB0
:1051600080B201E000207047824238BF00207047C3
:105170004289038992B29BB29A4205D1027B02F026
:10518000FF039AB1008870474289038992B29BB2AB
:105190009A4223BF428903890088038935BF408929
:1051A00010FA83F0181A801A80B2704718467047B8
:1051B000037B10B503F0FF021BB1012343730020F2
:1051C00010BD038944689BB2E1540389018801330F
:1051D0009BB2038103899BB2994298BF02810289E5
:1051E000438992B29BB29A424FF0010308BF037306
:1051F000184610BD034600895A8980B292B2904287
:1052000004D11A7B02F0FF0002B970475A8958682E
:1052100092B2825C0A70002119735A89188801328F
:1052200092B25A815A8992B2904200D85981012093
:10523000704703460022407B5A737047014B185C4D
:10524000704700BF9FE80008094AC1B2C0F30723B6
:10525000515CD35C0B44C0F30741000E515C105C01
:1052600051FA83F350FA83F0C0B282B002B07047B3
:105270009FE8000882B0144ACDE90001C0F307237B
:10528000C1B2D35C515C0B44C0F30741000E515CCA
:10529000105C51FA83F39DF8041050FA83F3505CCC
:1052A0009DF8051050FA83F3505C9DF8061050FAF3
:1052B00083F3505C9DF8071050FA83F3505C50FA6A
:1052C00083F0C0B202B070479FE800080346002296
:1052D00030B503F8042B00F1180143F8042B8B427E
:1052E000FBD100F507511831002523F8025B8B42F2
:1052F0004FF00002F9D142F2D81342F2DC11C2524F
:1053000042F2DA1300F50854C25242F20F734352CC
:1053100042F2DE111434435242F2E011435242F29F
:10532000E211435242F2E411435242F2E611435277
:1053300042F2E811435242F2EC13C25042F2F0132F
:10534000C25242F2F213C25400F50753343323F829
:10535000022BA3424FF00001F9D142F2142300F5D1
:105360000854C15200F508531633363423F8021B93
:105370009C424FF00002F9D142F236236321C2521F
:1053800042F23823C15442F23C23C25000F5095383
:105390001A8042F24223C25430BD42F2DA12002394
:1053A0000370835242F2D8126321835242F2EC120C
:1053B000835042F23822815442F2DC1142F20F72E1
:1053C000425242F2DE11425242F2E011425242F2A5
:1053D000E611425242F2E811425242F2E2114252C6
:1053E00042F2E411425242F21422835242F2362235
:1053F000835242F2F012835242F2F212835442F28A
:105400003C22835000F50952138042F24222835419
:10541000704700003F4BF7B54FF47A5604464FF003
:10542000000E30461F461FFA8EF5AA421FD901F121
:105430000C0534F91550002D06DDAF42B8BF2F46DC
:10544000A842A8BF284605E0AE42A8BF2E46AB4200
:10545000B8BF2B464D1DADB2B5F5875F22BFA1F594
:1054600086511B398DB20EF1010E2946DBE73A1841
:10547000334452105B10D5186D102EB2551B2DB24F
:105480001BB212B22449254801950096FCF7EEFEA6
:1054900042F2382104F50752635C04F50850632B8F
:1054A00002F1320200F112000AD1134623F8026F12
:1054B00098425D84FAD142F238230021E1540DE094
:1054C00004EB430742F2F41E013327F80E60DBB20F
:1054D00042F216260F2BBD536354ECD842F214212E
:1054E0000023635242F236216352194632F8025FBA
:1054F0002944558C90422B4409B21BB2F6D142F29A
:1055000014220911A15242F236221B11A35203B0F8
:10551000F0BD00BF80C1FFFFBDE9000828300020BA
:105520002DE9F04FBDF82440BDF92C80BDF928903D
:10553000334F04F1020E01341FFA8EFEA4B24FF075
:10554000000CC8F1000A1FFA8CF6AEF10205B24257
:10555000ADB252D901F10C0630F816B0C9EB0B0B05
:105560000FFA8BFBD3454FEAE50605F007050CDA89
:1055700017F805B09D5D25EA0B059D5504F007065B
:10558000E51017F806B05E5D21E0BBF1000F0CDA04
:1055900017F805B09D5D25EA0B059D5504F007063B
:1055A000E51017F806B05E5D0EE0C34517F805B0CC
:1055B0009D5D4BEA05059D5504F007064FEAE4059D
:1055C00017F806B05E5D02DA26EA0B0601E04BEA48
:1055D00006065E554E1DB5B2B5F5875F22BFA1F533
:1055E00086551B3DADB20EF1020E02340CF1010CDA
:1055F0001FFA8EFEA4B22946A5E7BDE8F08F00BFD2
:1056000015EB000842F2D8132DE9F04FC35A00EB16
:10561000830304465B686B4823F07F4387B05840A0
:10562000FFF712FE022800F2C98042F2DA134FF0AF
:10563000000EE75A6448DFF894C107F583550D352D
:10564000ADB2B5F5875F26BFA7F1730292B22A46C5
:1056500076464FF47A5102F10C031EF90C8034F9AE
:1056600013309842B8BF18469942A8BF1946B8F1FE
:10567000010F0AD0B8F1030F05D0B8F1FF3F06D0F3
:1056800003EB430303E003EB4303F61A00E01E447D
:10569000531D9BB2B3F5875F24BFA2F586521B3A18
:1056A0000EF1010E28BF93B2BEF1180F01D01A46B9
:1056B000D1E742F2EC13E358B3427FDA42F23823E7
:1056C000E35C632B0CD1014442F214234910E152F4
:1056D000411A44F63E10414342F23623C913E152C7
:1056E00042F23623B5F5875FE35E029342F214235C
:1056F00024BFA7F17305ADB2E35E019300270DF15E
:1057000010094B460097182229462046FFF708FF4C
:105710002378DFF8BCB0BB420CBF4FF0020A4FF059
:10572000040AB84619F8070017F80B305840FFF77D
:1057300085FD01374044062F5FFA80F8F2D1D0454D
:105740003CD842F2EC130522E65042F2F01342F24A
:10575000E011E25242F2DA1342F2E812E35AA352A3
:1057600042F2DE12A55203F58352073292B2B2F52D
:10577000875F28BFA3F1790262522278E2B942F230
:10578000E61242F2E211A35242F2DC12A55203F2F7
:10579000BB7292B2B2F5875F28BFA3F625126252A0
:1057A00003F2BD7292B2B2F5875F42F2E4112ABFF2
:1057B000A3F6231362526352012000E0002007B0D9
:1057C000BDE8F08FA030FB0080C1FFFF9FE900081B
:1057D000B7E9000838B50446FFF714FFB8B142F244
:1057E000F215635D9BB942F23C220121A35004F5FE
:1057F00009521D481380FDF793FE01211A48FDF759
:105800009DFE42F238236322E2540A23635542F29A
:10581000F213E25C0AB1013AE254E35C012B21D1BC
:1058200042F2E61342F2E211E35A03F2BB7292B281
:10583000B2F5875F28BFA3F62512625203F2BD724C
:1058400092B2B2F5875F42F2E41124BFA3F62313AC
:1058500063524FF0010338BF6252237042F2F213D9
:105860000022E25438BD00BF0065002042F2DC1384
:10587000F0B5C35A03F1780189B2B1F5875F28BF4B
:10588000A3F5835142F236239FB0C35E029342F2E6
:10589000142328BF0839C35E01934FF0000300931F
:1058A0004FF0080204AB28BF89B20446FFF738FE68
:1058B0009DF8113042F2422203F00F0383540F2B64
:1058C00000F2BA80DFE803F008B8B86BB8B8B846A1
:1058D000B8B8B8B82FB8B89042F2DC174FF4C67217
:1058E000C15B42F23626FFF795FD42F2142542F2E3
:1058F000E612A15F635FA25E009162486249FCF715
:105900006CFCA35F0293635F0193082300934FF441
:10591000C67205ABE15B2046FFF702FE01238DF85E
:105920001430642284E042F2E61542F23627415BED
:10593000B42242F21426FFF76DFDE15FA35F0091F0
:10594000625F52494F48FCF748FCE35F0293615B9A
:10595000A35F17E042F2DC17B422C15B42F23626A5
:10596000FFF758FD42F2142542F2E612A15F635F91
:105970000091A25E46494348FCF72FFCA35F0293C7
:10598000E15B635F019308230093B42205AB2046DB
:10599000FFF7C6FD01238DF814302E2248E042F2B5
:1059A000DC174822C15B42F23626FFF733FD42F294
:1059B000142542F2E612A15F635FA25E00913148B6
:1059C0003449FCF70AFCA35F0293635F0193082349
:1059D0000093482205ABE15B2046FFF7A1FD0123C0
:1059E0008DF81430132223E042F2DC17D822C15B79
:1059F00042F23626FFF70EFD42F2142542F2E6127D
:105A0000A15F635FA25E00911E482349FCF7E5FB9E
:105A1000A35F0293635F019308230093D82205AB31
:105A2000E15B2046FFF77CFD01238DF8143037221F
:105A300005A91448FBF766FC42F2E81342F2E211B2
:105A4000E35A03F586521F3292B2B2F5875F28BF40
:105A500003F1FF3262525A1C92B2B2F5875F28BF3F
:105A6000A3F5865342F2E41124BF1F3B63524FF06B
:105A7000020338BF6252237042F2EC130022E2505C
:105A80001FB0F0BD28300020DDE900080BEA000857
:105A900039EA000868EA000896EA000842F2E213D0
:105AA00042F2DA11C25A415A42F2E41310B5C35A13
:105AB0009A42044607D28A4208D88B4206D320462F
:105AC000FFF7A0FD02E08A42F7D8F8E742F2DA13C6
:105AD000E25A42F2E413E35A9A4204D12046BDE866
:105AE0001040FFF7C3BE10BD38B500F50955044698
:105AF000288860B142F23C23DB22E358B3FBF0F389
:105B0000C3F3072081F8D90081F8DA3000E0D92208
:105B10000448FBF729FC42F23C220023A3502B80CF
:105B200038BD00BF2830002042F2E213F0B5C25A5F
:105B300042F2E41342F2DA11C35A415A9A42BDB01A
:105B4000044607D28A4208D88B4206D32046FFF784
:105B500059FD02E08A42F7D8F8E742F2DA13E25A36
:105B600042F2E013E35A9A4279D142F2F013E35A37
:105B7000052B1AD142F2E81342F2E211E35A03F57F
:105B800086521F3292B2B2F5875F28BF03F1FF320F
:105B900062525A1C92B2B2F5875F42F2E41125BFFD
:105BA000A3F586531F3B6252635242F2DE174FF455
:105BB0005872E15B204642F23626FFF72BFC42F298
:105BC000142542F2E812A15F635FA25E00912548AE
:105BD0002549FCF702FBA35F0293635F019308234F
:105BE0000093E15B05AB4FF458722046FFF798FC39
:105BF00042F2F013E55A013DADB2E55215BB1B4927
:105C00001848FBF7ABFC29461948FDF789FC2946E3
:105C10001748FDF793FC1348FBF7D8FB42F2E0135B
:105C200042F20F722570E25242F238236322E254AC
:105C300042F2F213E55442F2EC13E55042F24223F1
:105C4000E5540CE02B1F5D425D4105A920468DF80F
:105C50001450FFF749FF42F2EC130022E2503DB02E
:105C6000F0BD00BF28300020C6EA0008F4EA0008B2
:105C7000006500202DE9F84F00F5085A00F507559A
:105C800004460F4690461E464FF000090AF13C0AB2
:105C900018354E454BD038F81920DAF8003037F96E
:105CA0001910134404F50952CAF80030138801335F
:105CB00013802A8804EB82020029536804F5075BED
:105CC0004FEA4303B8BF43F001030BF11A0B5360D3
:105CD000BBF800300C3324F813102378012B05D0C7
:105CE000022B07D12046FFF71FFF06E02046FFF7F3
:105CF000D5FE02E02046FFF76DFDBBF80030013312
:105D00009BB2B3F5875F21BF04F509530022ABF8BE
:105D100000209A7038BFABF800302B8801339BB25B
:105D2000042B88BF00232B8009F10109B1E7BDE8EE
:105D3000F88F0000F7B502254C4E684604F0D8FBFA
:105D400000272846012101248DF805508DF80750C1
:105D50008DF8067004F078FE4FF4805369463046A3
:105D600000938DF8044004F081FB2146284604F09E
:105D70006BFE10236946304600938DF8044004F012
:105D800075FB2146284604F05FFE0823694630462D
:105D900000938DF8044004F069FB2146284604F086
:105DA00053FE4FF400536946304600938DF804705B
:105DB00004F05CFB2146284604F046FE4023694679
:105DC000304600938DF8044004F050FB21462846ED
:105DD00004F03AFE20236946304600938DF80440D3
:105DE00004F044FB2146284604F02EFE8023694639
:105DF000304600938DF8044004F038FB21462846D5
:105E000004F022FE4FF480736946304600938DF80B
:105E1000044004F02BFB2146284604F015FE144DE7
:105E20008DF804404FF4007369463046009304F047
:105E30001DFB2146042004F007FE4FF480636946F1
:105E4000284600938DF8044004F010FB21460420FE
:105E500004F0FAFD4FF400636946284600938DF87C
:105E6000044004F003FB03B0F0BD00BF0004024097
:105E70000008024037B54FF4006300240DF105021D
:105E80000DF1060105461830ADF806308DF80540D5
:105E900002F08AFFBDF80610204604F0CDFB022177
:105EA000144806F062F810B9ADF8060007E0114892
:105EB00005F0B5FFADF806000F4805F0B0FF044649
:105EC00002210C4806F057F80A4805F07CFF9DF8BF
:105ED0000520BDF80610281D02F03FFF214605F100
:105EE0002C0001F022FBD5F82C330133C5F82C33FC
:105EF00003B030BD002001400021014008B5012160
:105F00004FF0804005F0C1FD48B14FF080400121C5
:105F100005F0C6FD0248BDE80840FFF7ABBF08BD6D
:105F2000006500202DE9F041022194B0704806F090
:105F30001CF810B16F48FFF79DFF01A804F0D8FAD4
:105F400006A805F0C1FE0EA805F0A0FE0121022062
:105F500004F07AFD01214FF480700024012504F043
:105F6000A3FD032601A9644801958DF808608DF80A
:105F70000B4004F07BFA2946022004F065FD294617
:105F80004FF4007004F090FD4FF0020801A95A4848
:105F9000CDF804808DF808608DF80B4004F066FAA7
:105FA000062306A8069307940894099405F078FE42
:105FB0000EA94F480E948DF83C408DF83D4010944A
:105FC000119412948DF84C5005F03AFE2946484839
:105FD00005F002FF23462A460821454805F0ACFE9D
:105FE0002946434805F076FE0EA9444805F028FEF0
:105FF0002946424805F0F0FE23462A4609213F483B
:1060000005F09AFE29463D4805F064FE01A804F01B
:106010006FFA0AA804F0DEFA2946284604F014FDB7
:1060200029464FF0005004F033FD102701A93448F1
:1060300001978DF808608DF80B4004F017FA0AA953
:1060400020460A940B940D9404F0AEFA294620469B
:1060500004F0C6FA2946284604F01AFD2A460F2104
:10606000274804F081FA4FF4004301A92448019322
:106070008DF8088004F0FAF903A805F07BF9F923FC
:1060800003A94FF08040ADF80C300495ADF80E40F8
:10609000ADF814408DF8164005F02EF9234622463F
:1060A00021464FF0804005F087FD29464FF08040A3
:1060B00005F0B7F92A4629464FF0804005F001FD6A
:1060C0001C2368468DF800308DF801408DF8025091
:1060D0008DF8035004F0D2FD3946074804F037FA32
:1060E0000821054804F031FA14B0BDE8F08100BF82
:1060F0000020014000650020000402400021014012
:106100000000024008B54FF40051034804F00BFAB8
:10611000431E5842584108BD000402400A46024846
:10612000082104F016BA00BF000402400A460248E3
:106130004FF4805104F00DBA000402400A460248B0
:10614000102104F006BA00BF000402400A460248CB
:10615000402104F0FEB900BF000402400A46024894
:10616000202104F0F6B900BF000402400A460248AC
:10617000802104F0EEB900BF000402400A46024844
:106180004FF4807104F0E5B9000402400A46024869
:106190004FF4007104F0DDB9000402400A460248E1
:1061A0004FF4806104F0D5B9000802400A46024865
:1061B0004FF4006104F0CDB900080240064B40F6F0
:1061C000B8321B68B3FBF2F221B11346013BFDD19B
:1061D0000139F9E7704700BF2C060020F8B54FF4ED
:1061E0007A61044604F1280700F062F90023236174
:1061F0006361A361A3832362636204F148063A46A4
:1062000022F8023BB242FBD104F1C0023346002126
:1062100023F8021B9342FBD104F5AE62002103F880
:10622000011B93424FF00005F9D1F023A4F8743517
:1062300041F27073C4F878352946A4F87055A4F873
:106240007255C4F87C552022384606F095FD782218
:106250002946304606F090FD052323740823638207
:10626000044B63612023A383034BA761266263620F
:106270002046F8BDA002002060020020122AF8B5D6
:1062800006460F46144614D900F024F9A04212D352
:10629000013CE1B2304600F05FF90025EBB29C42D0
:1062A00005F1010509D93B443046597800F054F90D
:1062B000F4E70420F8BD0520F8BD0020F8BD00007B
:1062C000F0B54FF4D27299B00546002440F2EC4686
:1062D0004FF614374FF65C6E01F0C003802B02A816
:1062E0000BD0C02B06D0002B0CBF73463B4620F8CA
:1062F000143004E020F8146001E020F81420013488
:106300008B00042CD9B2E7D1234604AA014605F13B
:10631000100005F06BFF0EAA04A905F11C00142360
:1063200006F060F9002300930EAA142321460248C8
:10633000FDF792F819B0F0BD0065002030B599B0B6
:106340000024054604AA02A90423103002940394F1
:1063500005F04CFF0EAA04A905F11C00142306F059
:1063600041F9009414230EAA04210248FDF774F8A1
:1063700019B030BD0065002070B5B0F87055044606
:106380002DB13948394EFDF7C7F805460BE000F04E
:10639000C3F800283FD102E00023A4F87235B4F816
:1063A00070350BB3EDE7142D5CD9B4F872355A1C77
:1063B0002344A4F8722593F8C0102046FFF780FF0D
:1063C0003378143DADB21BB1D4F87835C4F87C35C0
:1063D000B4F87225B4F870359A42E4D30023A4F8D7
:1063E0007235A4F8703570BDD4F87C35002B39D0E7
:1063F0001D48FDF791F80546142D33D92046FFF7C7
:106400009DFFD4F87C35143D013BADB2C4F87C351A
:10641000002BF1D170BD164B1B787BB9B4F87455C5
:1064200077219AB2AA42B7D2B4F87025501C224400
:10643000A4F87005013382F8C010F2E7204600F09E
:10644000B1F80646EBB2B342A6D2204600F0AAF855
:10645000B4F870355A1C2344A4F87025013583F82C
:10646000C000EFE770BD00BF0065002058020020AB
:10647000FC64002001EB4101890001F5167189B22D
:10648000B1F5966F8ABF4FF49663A0F87415A0F823
:106490007435704708B500F01DF8D823B0FBF3F051
:1064A000C0B208BD4FF496635943C0F878157047E1
:1064B00010B500230381044643810180037308461D
:1064C00006F022FB6060204610BD0023038143815B
:1064D000037370474289038992B29BB29A42028841
:1064E00003D1037B93B9104612E04189038989B235
:1064F0009BB2994239BF03894089438900893ABFD9
:1065000012FA80F0C01A181A80B201E00020704719
:10651000824238BF002070474289038992B29BB201
:106520009A4205D1027B02F0FF039AB100887047BE
:106530004289038992B29BB29A4223BF428903895E
:106540000088038935BF408910FA83F0181A801A31
:1065500080B2704718467047037B10B503F0FF0206
:10656000BBB9038944689BB2E154038901880133B4
:106570009BB2038103899BB2994298BF0281028931
:10658000438992B29BB29A424FF0010303D1037345
:1065900001E0002010BD184610BD438942689BB23F
:1065A000D05C704710B54289416892B20346885C5E
:1065B0001C88002119735A89013292B25A815A8972
:1065C00092B29442C0B298BF598110BD034630B513
:1065D00000F1180203F8041B002143F8041B934246
:1065E000FBD11A4600F5E464002522F8025BA242C2
:1065F0004FF00003F9D142F20F72A0F82827A0F85B
:106600002037A0F82237A0F82437A0F82637A0F8C2
:106610002A37C0F82C37A0F83037A0F83237A0F866
:106620003437A0F83637A0F83837A0F83A37A0F852
:106630003C37A0F83E3780F8403780F8413780F883
:10664000423780F84337A0F8443780F8463780F85F
:10665000473780F8483700F24A7200F6526122F854
:10666000023B8A42FBD130BD0023A0F82237A0F8BC
:106670002A37A0F82037C0F82C3780F84137704708
:106680000023A0F82437A0F82237A0F82A37A0F872
:106690002037C0F82C3780F8413780F8423780F82F
:1066A0004637A0F8263742F20F73A0F82837704714
:1066B0002DE9F047BDF82050BDF92880BDF92490A0
:1066C000DFF8B0E005EB4202AF1C6C1C0232BFB237
:1066D000A4B292B2C8F1000ABE1EBA42B6B246D007
:1066E00001F10C0530F815C0C9EB0C0C0FFA8CFC4D
:1066F000D4454FEAE60506F007060CDA1EF806C098
:106700005E5D26EA0C065E5504F00706E5101EF8ED
:1067100006C05E5D21E0BCF1000F0CDA1EF806C079
:106720005E5D26EA0C065E5504F00706E5101EF8CD
:1067300006C05E5D0EE0C4451EF806C05E5D4CEA14
:1067400006065E5504F007064FEAE4051EF806C08B
:106750005E5D02DA26EA0C0601E04CEA0606053127
:10676000023702345E5589B2BFB2A4B2B4E7BDE8C5
:10677000F08700BFCEEC0008B0F820372DE9F04FCD
:1067800000EB830304465B687B4823F07F4358405B
:1067900089B00F46FEF758FDC31EDBB2122B8046B0
:1067A00040F2E680B4F82217744DDFF8DCC1DFF860
:1067B000DC91733989B200228E464FF47A50164626
:1067C0000EF10C0334F913309D42B8BF1D469842B8
:1067D000A8BF1846B8F1020F94BF12F909A012F928
:1067E0000CA0BAF1010F0AD0BAF1030F05D0BAF12B
:1067F000FF3F06D003EB430303E003EB4303F61A2A
:1068000000E01E4401320EF1050E182A1FFA8EFE1A
:10681000D6D1D4F82C379E4240F3AA8028444010A9
:106820000FFA80F9281A44F631454543042345F30D
:10683000CF350DF1180A009302955346CDF8049018
:106840002046FFF735FFB8F1020F4FF00008DFF8E0
:1068500040B143463FD84A491AF808001BF80820BF
:106860000593024018F8010004915040FEF7E6FC41
:10687000059B049908F101081844B8F1070FC3B249
:10688000EAD1032B74D88FB1A4F83E57A4F83C5733
:10689000A4F83A57A4F83857A4F83697A4F83497D0
:1068A000A4F83297A4F8309700230BE094F840370F
:1068B00004EB43020133DBB2032BA2F83857A2F8F2
:1068C000309702D884F8403701E084F84077C4F864
:1068D0002C6740233EE02B491AF808001BF80820DB
:1068E0000593024018F8010004915040FEF7A6FC01
:1068F000059B049908F101081844B8F1070FC3B2C9
:10690000EAD1032B34D88FB1A4F83E57A4F83C57F2
:10691000A4F83A57A4F83857A4F83697A4F834974F
:10692000A4F83297A4F8309700230BE094F840378E
:1069300004EB43020133DBB2032BA2F83857A2F871
:10694000309702D884F8403701E084F84077C4F8E3
:106950002C67202384F84137B4F82237A4F8243771
:10696000A3F5C37203F20D13A4F82627A4F8283761
:1069700009B0BDE8F08F00BF6E28760080C1FFFF30
:106980002BEB000824EB0008B6EC0008D6EC00085E
:106990001DEB000880F843177047A0F844177047B4
:1069A00030B4B0F8264704F13C0304F51674A5B2E0
:1069B0000A469BB20024591C00EB4303B3F84A3744
:1069C0001C448BB2AB42F6D14FF40773B4FBF3F423
:1069D000C4F3072382F8223082F82340017802486A
:1069E000242330BCFAF7E4BB28300020B0F82A3763
:1069F000F0B501339BB20446A0F82A37B0F844073B
:106A000098428FB000F27E81B4F82237B4F828079C
:106A10009842C0F07781B3F5617F80F0738104EB19
:106A200043000029A0F84A270183B4F8200704EBAB
:106A3000800042684FEA4202B8BF42F00102426061
:106A400094F846272AB9A3F5C8735A2B0FD8012109
:106A50000AE0B4F82427511E89B28B4207D30132D1
:106A600092B2934203D800212046FFF785FEB4F886
:106A70002237B4F82817994240F03681B4F93237FA
:106A8000B4F93067B4F938771E44B4F934371E448A
:106A9000B4F936371E44B4F93A371F44B4F93C37D9
:106AA0001F44B4F93E370EAD1F4494F8413705F842
:106AB000243D46F38F06082347F38F07A1F28E216A
:106AC000009302972B460196842289B22046FFF755
:106AD000EFFD94F84137402B40F0A98004A802F064
:106AE0008EF90DF113030DF112020DF1150104A839
:106AF00002F0B2F994F843279DF812309A4240F020
:106B0000F38000239DF8142084F8423784F8473737
:106B10009DF813301A438DF814200A2B6ED8DFE845
:106B200003F044395D6D6D6D061D1D6D1D002378EC
:106B300078497948002B18BF0222B4F9243708BFDE
:106B400001228DE8C000FBF791FB29462046FFF7A4
:106B500027FF022384F84637002318E094F84637CD
:106B6000022B40F0C18023786C496B48002B18BF82
:106B70000222B4F9243708BF01228DE8C000FBF7D8
:106B800075FB29462046FFF70BFF9DF8133084F86C
:106B90004837A9E023786249002B8DE8C000B4F99A
:106BA000243714BF022201220DE094F84637012B4E
:106BB00010D123785B498DE8C000002BB4F924374D
:106BC00014BF022201225448FBF750FB29462046FD
:106BD000FFF7E6FE012384F8463785E094F8463750
:106BE000012B40F0818023784F49002B8DE8C000B5
:106BF000B4F9243714BF0222012209E023784B495B
:106C00008DE8C000002BB4F9243714BF0222012202
:106C10004148FBF72BFB29462046FFF7C1FE002326
:106C200084F8463742F20F73A4F828375CE0202B33
:106C30001AD123783E493848002B18BF0222B4F9F4
:106C4000243708BF01228DE8C000FBF70FFB29465F
:106C50002046FFF7A5FE012384F84637002384F879
:106C6000423784F847373FE094F84637002B3BD053
:106C700094F842370133DBB20C2B84F842370AD93F
:106C800021782548FAF7CAFA002384F8463742F2F9
:106C90000F73A4F8283794F84637012B17D194F8CE
:106CA000473721781C48042B8DBF20230133DBB2EA
:106CB0008DF8143087BF002384F8473784F84737AE
:106CC0008DF814302A462223FAF772FA0CE0022BD0
:106CD0000AD194F848373BB143F040032946204697
:106CE0008DF81430FFF75CFEB4F822370133A4F8B6
:106CF0002237B4F8203701339BB2042B88BF00231E
:106D0000A4F8203794F84607003018BF01200FB0D0
:106D1000F0BD00BF32EB00082830002069EB00080E
:106D2000A1EB0008D9EB000814EC000850EC0008B7
:106D300080EC00080346002230B503F8042B00F174
:106D4000180143F8042B8B42FBD100F59651183102
:106D5000002523F8025B8B424FF00002F9D141F28B
:106D6000D82341F2DC21C25241F2DA2300F59854D3
:106D7000C25242F20F73435241F2DE2110344352A9
:106D800000F597510B8041F2E221435241F2E42198
:106D9000435241F2E823C25041F2EC23C25241F285
:106DA000EE23C25400F59753103323F8022BA3426D
:106DB0004FF00001F9D141F2103300F59954C1525E
:106DC00000F598531233123423F8021B9C424FF003
:106DD0000002F9D141F232336321C25241F234331D
:106DE000C15441F23833C25041F23C33C25230BD3B
:106DF00041F2DA2200230370835241F2D822632148
:106E0000835241F2E822835041F23432815441F2FC
:106E1000DC2142F20F72425241F2DE21425200F571
:106E200097510A8041F2E221425241F2E42142525A
:106E300041F21032835241F23232835241F2EC225B
:106E4000835241F2EE22835441F23832835041F2B0
:106E50003C328352704700003E4BF7B54FF47A56F0
:106E600004464FF0000E30461F461FFA8EF5AA4228
:106E70001ED901F10C0534F91550002D06DDAF4285
:106E8000B8BF2F46A842A8BF284605E0AE42A8BF1B
:106E90002E46AB42B8BF2B464D1DADB2B5F5166FB1
:106EA00024BFA1F65B118DB20EF1010E2946DCE77D
:106EB0003A18334452105B10D5186D102EB2551B82
:106EC0002DB21BB212B22449244801950096FBF75B
:106ED000CDF941F2343104F59752635C04F59850D2
:106EE000632B02F10E0200F10E000AD1134623F8C3
:106EF000026F98425D84FAD141F234330021E154AB
:106F00000DE004EB430741F2F02E013327F80E6049
:106F1000DBB241F212360F2BBD536354ECD841F271
:106F200010310023635241F232316352194632F874
:106F3000025F2944558C90422B4409B21BB2F6D112
:106F400041F210320911A15241F232321B11A35207
:106F500003B0F0BD80C1FFFF02ED00082830002023
:106F60002DE9F04FBDF82440BDF92C80BDF92890E3
:106F7000324D04F1020E01341FFA8EFEA4B24FF01E
:106F8000000CC8F1000A1FFA8CF7AEF10206BA42F3
:106F9000B6B251D901F10C0730F817B0C9EB0B0BA1
:106FA0000FFA8BFBD3454FEAE60706F007060CDA2B
:106FB00015F806B0DE5D26EA0B06DE5504F007077D
:106FC000E61015F807B09F5D21E0BBF1000F0CDA69
:106FD00015F806B0DE5D26EA0B06DE5504F007075D
:106FE000E61015F807B09F5D0EE0C34515F806B032
:106FF000DE5D4BEA0606DE5504F007074FEAE406BD
:1070000015F807B09F5D02DA27EA0B0701E04BEAAB
:1070100007079F554F1DBEB2B6F5166F24BFA1F6E8
:107020005B16B6B20EF1020E02340CF1010C1FFA1F
:107030008EFEA4B23146A6E7BDE8F08F6AED0008E7
:1070400041F2D8232DE9F04FC35A00EB83030446E5
:107050005B685A48C3F3130387B05840FEF7F4F84F
:10706000032800F2A68041F2DA234FF0000EE55A21
:107070005348DFF850C105F60117BFB2B7F5166FD8
:1070800026BFA5F15F0292B23A4676464FF47A5196
:1070900002F10C031EF90C8034F913309842B8BF8A
:1070A00018469942A8BF1946B8F1010F0AD0B8F1A5
:1070B000030F05D0B8F1FF3F06D003EB430303E015
:1070C00003EB4303F61A00E01E44531D9BB2B3F5D5
:1070D000166F28BFA2F65B120EF1010E28BF93B205
:1070E000BEF1140F01D01A46D2E741F2E823E3586B
:1070F000B3425EDA41F23433E35C632B0CD10B18FC
:1071000041F210325B10A352C31A44F63E104343BF
:1071100041F23232DB13A35241F23233B7F5166F2C
:10712000E35E029341F2103324BFA5F15F07BFB2C3
:10713000E35E019300250DF110094B4600951422E2
:1071400039462046FFF70CFF2378DFF87CB0AB42CE
:107150000CBF4FF0020A4FF0040AA84619F80500C8
:1071600015F80B305840FEF769F801354044052DFD
:107170005FFA80F8F2D1D0451BD841F2E82304F53C
:107180009752E65041F2EC2341F2DE21E55241F202
:10719000DA230120E35A138041F2DC22A75203F6DE
:1071A000FB0292B2B2F5166F2ABF653B6252635280
:1071B00000E0002007B0BDE8F08F00BFADB50700CC
:1071C00080C1FFFFEEEC000872ED000838B5044600
:1071D000FFF736FFB8B141F2EE25635D9BB941F28E
:1071E00038320121A35041F23C321C48A352FCF733
:1071F00097F901211948FCF7A1F941F234336322D0
:10720000E2540523635541F2EE23E25C0AB1013AF0
:10721000E254E35C012B20D104F5975341F2E221C3
:107220001B8803F65F1292B2B2F5166F28BF03F106
:10723000FF3262525A1C92B2B2F5166F41F2E4214B
:1072400024BFA3F65F1363524FF0010338BF6252AD
:10725000237041F2EE230022E25438BD0065002085
:1072600041F23C3310B50446C05A60B141F23833A4
:107270007B22E358B3FBF0F3C3F3072081F87900D6
:1072800081F87A3000E079220548F9F7E9FF41F208
:1072900038320023A35041F23C32A35210BD00BF4C
:1072A0002830002041F2E223F0B5C25A41F2E42333
:1072B00041F2DA21C35A415A9A42A5B0044607D294
:1072C0008A4208D88B4206D32046FFF7B9FE02E077
:1072D0008A42F7D8F8E741F2DA23E25A41F2DE2394
:1072E000E35A9A4273D141F2EC2304F59756E35ADC
:1072F000052B16D1338803F65F1292B2B2F5166FE2
:1073000041F2E22128BF03F1FF3262525A1C92B2CD
:10731000B2F5166F41F2E4212ABFA3F65F13625261
:10732000635241F2DC274FF4F072E15B2046FFF735
:1073300093FDB6F90020274841F2323641F210356C
:10734000A15F635F00912449FAF747FFA35F0293AF
:10735000635F019308230093E15B05AB4FF4F07288
:107360002046FFF7FDFD41F2EC23E55A013DADB2A9
:10737000E552FDB919491748FAF7F0F829461848B7
:10738000FCF7CEF829461648FCF7D8F81148F9F76B
:1073900099FF41F2DE2342F20F722570E25241F270
:1073A00034336322E25441F2EE23E55441F2E82300
:1073B000E5500CE02B1F5D425D4105A920468DF88C
:1073C0001450FFF74DFF41F2E8230022E25025B0B0
:1073D000F0BD00BF2830002022ED000849ED000874
:1073E000006500202DE9F84F00F5995A00F59655F3
:1073F00004460F4690461E464FF000090AF1180A4F
:1074000018354E453FD038F81920DAF8003037F9F2
:1074100019101344CAF8003004F5995300299A8BC7
:1074200002F101029A832A8804EB820204F5965B3A
:1074300053684FEA4303B8BF43F001030BF11A0B43
:107440005360BBF800300C33204624F81310237827
:10745000012B02D1FFF726FF01E0FFF7B7FEBBF8D3
:10746000003001339BB2B3F5166F28BF0023ABF891
:1074700000302B8801339BB2042B88BF00232B8064
:1074800009F10109BDE7BDE8F88F10B500230381BC
:1074900004464381018003734373480005F034FBC5
:1074A0006060204610BD4289038992B29BB29A4225
:1074B000028803D1037B93B9104612E04189038906
:1074C00089B29BB2994239BF0389408943890089B7
:1074D0003ABF12FA80F0C01A181A80B201E00020F8
:1074E0007047824238BF002070474289038992B2B8
:1074F0009BB29A4205D1027B02F0FF039AB1008849
:1075000070474289038992B29BB29A4223BF428953
:1075100003890088038935BF408910FA83F0181A5F
:10752000801A80B2704718467047037B10B503F08D
:10753000FF021BB101234373002010BD038944687F
:107540009BB224F813100389018801339BB2038195
:1075500003899BB2994298BF02810289438992B202
:107560009BB29A424FF0010308BF0373184610BD47
:10757000034600895A8980B292B2904204D11A7BA4
:1075800002F0FF0002B970475A89586892B230F889
:1075900012200A80002119735A891888013292B288
:1075A0005A815A8992B2904200D85981012070477D
:1075B00003460022407B5A73704730B5034600F102
:1075C0001402002143F8041B9342FBD11A4600F633
:1075D0005434002522F8025BA2424FF00003F9D197
:1075E00042F20F72A0F85C2B00F5B552A0F8543BA4
:1075F000A0F8563BA0F8583BA0F85A3BC0F8603BB7
:10760000A0F8643BA0F8663BA0F8683BA0F86A3B92
:10761000A0F86C3BA0F86E3BA0F8703BA0F8723B62
:1076200080F8743B80F8753B80F8763B80F8773BB8
:1076300080F8783B80F8793B80F87A3B00F67C3123
:107640001C3221F8023B9142FBD130BD0023A0F84F
:10765000583BC0F8603B80F8753B80F8763B80F87B
:10766000783BA0F85A3B42F20F73A0F85C3B70479E
:107670002DE9F047BDF82060BDF928C0BDF9248090
:1076800006EB4202B51C741C0232344EADB2A4B2F9
:1076900092B2CCF10009A5F1020EAA421FFA8EFEA9
:1076A00059D000EB4107B7F814A0C8EB0A0A0FFA4B
:1076B0008AFACA454FEAEE070EF0070E0FDA16F8FF
:1076C0000EA013F807E02EEA0A0E03F807E004F014
:1076D000070EE71016F80EA013F807E027E0BAF13E
:1076E000000F0FDA16F80EA013F807E02EEA0A0EC4
:1076F00003F807E004F0070EE71016F80EA013F8E1
:1077000007E011E0E24516F80EA013F807E04AEA98
:107710000E0E03F807E004F0070E4FEAE40716F830
:107720000EA013F807E002DA2EEA0A0E01E04AEA98
:107730000E0E03F807E001F1050E1FFA8EF7B7F5FC
:10774000B46F24BFA1F29B57BFB202350234ADB271
:10775000A4B239469FE7BDE8F08700BFFEEE0008FF
:107760002DE9F04FB0F8543B50F8233004469148CF
:1077700023F07F43584089B08846FDF765FDC31E5E
:10778000DBB2122B814640F21281B4F856EB8A4DDF
:10779000DFF830C2DFF830A20EF22D5189B2B1F518
:1077A000B46F28BFAEF173024FF000072CBF92B246
:1077B0000A464FF47A503E4604EB4203B3F91430C4
:1077C0009D42B8BF1D469842A8BF1846B9F1020FA6
:1077D00094BF17F90AB017F90CB0BBF1010F0AD02A
:1077E000BBF1030F05D0BBF1FF3F06D003EB430312
:1077F00003E003EB4303F61A00E01E44531D9BB263
:10780000B3F5B46F28BFA2F29B5207F1010728BF5E
:1078100093B2182F01D01A46CEE7D4F8603B9E42AF
:1078200040F3C5802844401007B22D1A44F6314079
:10783000B1F5B46F00FB05F528BFAEF173014FF051
:10784000040345F3CF350DF1180A28BF89B2009320
:1078500002955346019718222046FFF709FFB9F118
:10786000020F4FF00009DFF864B14B4642D853498C
:107870001AF809001BF809200593024019F80100C5
:1078800004915040FDF7DAFC059B049909F10109C8
:107890001844B9F1070FC3B2EAD1032B00F2878075
:1078A000B8F1000F11D0A4F8725BA4F8705BA4F8D3
:1078B0006E5BA4F86C5BA4F86A7BA4F8687BA4F800
:1078C000667BA4F8647B00230BE094F8743B04EB24
:1078D00043020133DBB2032BA2F86C5BA2F8647B9A
:1078E00002D884F8743B01E084F8748BC4F8606BB0
:1078F000402340E032491AF809001BF8092005939B
:10790000024019F8010004915040FDF797FC059BD7
:10791000049909F101091844B9F1070FC3B2EAD17A
:10792000032B44D8B8F1000F11D0A4F8725BA4F86F
:10793000705BA4F86E5BA4F86C5BA4F86A7BA4F897
:10794000687BA4F8667BA4F8647B00230BE094F8C2
:10795000743B04EB43020133DBB2032BA2F86C5BF4
:10796000A2F8647B02D884F8743B01E084F8748B3D
:10797000C4F8606B202384F8753BB4F8563BA4F838
:10798000583B03F21A4292B2B2F5B46F28BFA3F586
:10799000C372A4F85A2B03F20D1292B2B2F5B46F6F
:1079A0002ABFA3F29343A4F85C2BA4F85C3B09B074
:1079B000BDE8F08F6E28760080C1FFFF85ED0008DE
:1079C0007EED0008E6EE000806EF000877ED0008FF
:1079D00080F8771B70470000B0F85A3B3C3370B416
:1079E0000A469BB24FF40775002400EB43015E1C6E
:1079F000B6B2B6F5B46FB1F87C1B05F1FF3528BF00
:107A0000A3F29F53ADB20C4428BF9EB20DB13346D2
:107A1000EBE74FF40773B4FBF3F4C4F3072382F8E6
:107A2000223082F8234024230121024870BCF9F758
:107A3000BFBB00BF2830002070B50446B0F8560B1D
:107A400004EB400300299982A3F87C2BB4F8542B53
:107A500054F822304FEA4303B8BF43F0010344F81F
:107A6000223094F8783B8EB00BB901211AE0B4F8BB
:107A7000581B01F29F539BB2B3F5B46F01F10102A1
:107A800092B224BF01F1FF339BB2B2F5B46F24BFB1
:107A9000A1F29F5292B2934208D2834209D8824205
:107AA00007D300212046FFF75BFE02E08342F6D8B1
:107AB000F7E7B4F8562BB4F85C3B934240F01381DF
:107AC000B4F9662BB4F9645BB4F96C6B1544B4F982
:107AD000682B1544B4F96A2B1544B4F96E2B16447F
:107AE000B4F9702B03F212311644B4F9722B89B237
:107AF000B1F5B46F164428BFA3F28E2194F8752B0C
:107B00008DF814204FF0080345F38F0546F38F06D8
:107B100028BF89B20093029605AB019584222046C6
:107B2000FFF7A6FD94F8753B402B40F0848004A835
:107B300001F065F90DF113030DF112020DF11501BC
:107B400004A801F089F994F8772B9DF812309A4235
:107B500040F0C48000239DF8142084F8763B84F81C
:107B6000793B9DF813301A438DF814200A2B52D814
:107B7000DFE803F0332D4751515106171751170015
:107B80002B46B4F9582B654965480096FAF725FB52
:107B900005A92046FFF720FF022384F8783B002345
:107BA00012E094F8783B022B40F098802B46B4F911
:107BB000582B5C495A480096FAF70FFB05A9204656
:107BC000FFF70AFF9DF8133084F87A3B86E0B4F99A
:107BD000582B00962B46544908E094F8783B012B2B
:107BE0000BD1B4F9582B514900962B464C48FAF763
:107BF000F4FA05A92046FFF7EFFE012384F8783B4D
:107C00006CE094F8783B012B68D1B4F9582B0096BE
:107C10002B46474904E0B4F9582B464900962B46B9
:107C20003F48FAF7DAFA204605A9FFF7D5FE2046C5
:107C3000FFF70CFD52E0202B14D12B46B4F9582B42
:107C40003D4937480096FAF7C8FA05A92046FFF7DC
:107C5000C3FE012384F8783B002384F8763B84F844
:107C6000793B3BE094F8783B002B37D094F8763B97
:107C70000133DBB20C2B84F8763B06D9284801216E
:107C8000F9F7CCFA2046FFF7E1FC94F8783B012B9A
:107C900017D194F8793B2248042B8DBF2023013360
:107CA000DBB28DF8143087BF002384F8793B84F869
:107CB000793B8DF8143005AA22230121F9F778FACF
:107CC0000CE0022B0AD194F87A3B3BB143F040031D
:107CD00005A920468DF81430FFF77EFE0023C4F876
:107CE000603B84F8753BB4F8563B94F8780B01334D
:107CF0009BB2B3F5B46F28BF0023A4F8563BB4F889
:107D0000543B01339BB2042B88BF0023003018BFC3
:107D10000120A4F8543B0EB070BD00BF8CED0008EC
:107D200028300020BDED0008EFED000821EE00082E
:107D300056EE00088CEE0008B6EE0008F8B50C46CA
:107D400001EB43070646951E0021BC4208D034F9DA
:107D5000021B35F8022F3046FFF76EFE0146F4E7AE
:107D60000248BDE8F840FBF7DBBB00BF0065002020
:107D700000224FF4C0610280428042600181827221
:107D8000C2720273704700002DE9F743384E027B40
:107D900033789A42044654D0663B052B16D8DFE868
:107DA00003F00306090C0F124FF46F730FE040F25B
:107DB0000F430CE040F2DF4309E040F2616306E06C
:107DC00040F61F0303E040F6BF1300E000232380CA
:107DD00022882849002331F83300264F904204D1ED
:107DE000DBB217EBC30704D13FE00133062BF2D11E
:107DF0003BE060687B88638008B104F087FE6088A0
:107E0000400004F081FE002260609046638895B2D5
:107E1000AB4202F1010912D9404604F059FEB4F90F
:107E20000830626883FB0001C30F43EA410303F398
:107E30000F0322F815307B684A469844E6E733780A
:107E40002373A37A8BB10C48FBF766FB002705462A
:107E500063889D4209D93178009762680648FBF72C
:107E6000FBFA6388ED1AADB2F2E703B0BDE8F08328
:107E70008833002020EF000800650020012A06D189
:107E80000B785A1E534253418372002070470420DE
:107E90007047002310B5036003714371836000F1E4
:107EA0000C0100F1700401F8013BA1424FF0000207
:107EB000F9D1026742678267C267C0F88020C0F8C4
:107EC0008420C0F8882000F18C0300F59A7143F8F3
:107ED000042B8B42FBD100F5EE72002143F8041B0A
:107EE0009342FBD100F52172002143F8041B934219
:107EF000FBD100F54B72002143F8041B9342FBD1E8
:107F000000F25631002403F8014B8B424FF000027F
:107F1000F9D1C0F85823A0F85C2310BD00230360FA
:107F200003714371836003674367C0F85833A0F857
:107F30005C33704710B50446B0F85C0358B1D4F810
:107F40005833B3FBF0F3C3F3072081F8290081F81D
:107F50002A302B2200E029220448F9F78DF800236B
:107F6000C4F85833A4F85C3310BD00BF283000209B
:107F700010B50446B0F85C0348B1D4F85833B3FBED
:107F8000F0F3C3F3072008734B730E2200E00C22BA
:107F90000448F9F7A1F80023C4F85833A4F85C3377
:107FA00010BD00BF28300020836870B55B00044618
:107FB00009B143F00103A360A06820F07F43244887
:107FC0005840FDF741F9022811D822492248F9F713
:107FD000C5FA5322002104F10C0004F0CDFE002369
:107FE0002367C4F85833A4F85C3301232DE0A0685C
:107FF00020F07F4319485840FDF726F9054628BB75
:1080000017491548F9F7AAFA01211648FBF788FA2B
:1080100004F10C0601211348FBF790FA0C221249D7
:10802000C4F85853A4F85C53304604F00BFE3146B4
:108030002046FFF79DFF0E222946304604F09CFEA5
:108040004FF41653636725670223637170BD00BF49
:1080500050765500EBF400082830002068B4AA00E0
:108060000DF50008006500207EF7000883682DE903
:10807000F0415B00044609B143F00103226FA360A5
:10808000D00802F0070329B12118464DED5C0B7BA7
:108090002B4304E02118444DED5C0B7B2B40204426
:1080A00001320373A368414822675840FDF7CCF8BA
:1080B000012812D83E493F48F9F750FA00213E48BE
:1080C000FBF72EFA00213C48FBF738FA3948F9F75C
:1080D00051F800236371BDE8F081236F5C2B01D858
:1080E00000260EE0A06820F07F4334485840FDF79A
:1080F000ABF80228F4D8602323674FF41653636764
:108100000126236F602B18D1BEB9DFF8B08001259E
:108110006FF07F47A36827FA05F0034028FA05F0BF
:108120005840FDF791F8022804D8236FEDB25D1B8B
:10813000256702E00135042DECD1656F013D6567CF
:108140008DB91F491B48F9F709FA29461A48FBF768
:10815000E7F929461848FBF7F1F91648F8F7ECFF5C
:108160006571BDE8F081236F602B19D104F10C0516
:1081700056B1552363752D23A3751623E375294640
:108180002046FFF7F5FE04E00C2229460948F8F7DF
:10819000A3FF0E220021284604F0EEFD00232367F2
:1081A000BDE8F08176F50008E3F400085E13AAAAA2
:1081B0002EF50008283000200065002068B4AA00D1
:1081C0004EF500082DE9F0470D68D0F87C90D0F806
:1081D00084800F69846F09EB050C4744BC454FEA66
:1081E000D4034FEA8303E646A8BFBE46BC4504F06D
:1081F0000702B5BF354D364DAE5CAE5C00EB0307F4
:1082000000EB030CB5BFD7F88C50D7F88C50354035
:108210003543C7F88C504E684D694E444544AE42D4
:108220003746A8BF2F46AE42B5BF284D284DAE5C9D
:10823000AE5CB5BFDCF83451DCF834513540354321
:10824000CCF834518E68D0F880C0D0F888900CEB10
:10825000060A8E6909EB0605AA45D046A8BFA846BE
:10826000AA45B5BF194D1A4DAD5CAD5C00EB030AD4
:108270000344B5BFDAF8DC61DAF8DC612E402E4346
:10828000CAF8DC61CD68C969654449448D422E460F
:10829000A8BF0E468D42B5BF0C490D498A5C8A5C69
:1082A000B5BFD3F88412D3F884120A400A43C3F846
:1082B00084220134C0F87CE0C0F88070C0F884806B
:1082C000C0F888608467BDE8F08700BFD3F4000879
:1082D000DBF4000870B512C988B084F0010381F0A6
:1082E00001029E1865180B442244694600950196C8
:1082F000029303920496059506920793FFF762FF97
:1083000008B070BDF0B52E4C2E4F002340F249123C
:108310001946264603294FD8DFE801F002101D3424
:10832000D51000EB850502F0070ED5F88C5014F837
:108330000EE01EEA050F18BF022118E0D11000EB75
:10834000810102F00705D1F83411655D0D420CBFC3
:108350000021022123E0D11000EB810102F007058A
:10836000D1F8DC11655D0D420CBF0121032103F042
:10837000070500EBD30E17F805C09EF82C530CEA46
:10838000050516E0D51000EB850502F0070ED5F8BF
:10839000845214F80EE01EEA050F08BF012103F015
:1083A000070500EBD30E16F805C09EF82C534CEAD7
:1083B00005058EF82C53013312F1FF32AAD2F0BD1D
:1083C000DBF40008D3F4000870B5114E4FF0FF3312
:1083D0004C1E01F1260514F8012F5A40D2B2C3F306
:1083E000072036F81230A54280EA03000346F2D196
:1083F000C04391F82720C3B29A4207D191F82830A0
:10840000C0F30720C31A5842584170BD002070BD08
:108410007EF500082DE9F043904E174699B00446CA
:108420004A1E002312F8015F985D01336840532B08
:108430001070F7D10023184603AA98540133542B27
:10844000FAD1874B00208025B0F5257F0FDB002374
:10845000E367C4F88030C4F88430C4F88830A36778
:108460001D464FF0800801264FF04009ABE0C210D6
:108470008E5CF20710D513F810200DF1600E7244D7
:1084800003EB400E9EF801E025FA0EFC12F854ECC6
:108490004CEA0E0E02F854ECB20712D500F1010EB0
:1084A0000DF1600C13F81E2003EB4E0E62449EF893
:1084B00001E025FA0EFC12F854EC4CEA0E0E02F81C
:1084C00054EC720712D500F1020E0DF1600C13F896
:1084D0001E2003EB4E0E62449EF801E025FA0EFCCE
:1084E00012F854EC4CEA0E0E02F854EC320712D596
:1084F00000F1030E0DF1600C13F81E2003EB4E0E7D
:1085000062449EF801E025FA0EFC12F854EC4CEAA5
:108510000E0E02F854EC021DB2F5257F01DB104669
:1085200092E716F0100F0FD013F812E003EB42029F
:108530000DF1600CE644527825FA02FC1EF8542C2A
:108540004CEA02020EF8542CB20612D500F1050EC8
:108550000DF1600C13F81E2003EB4E0E62449EF8E2
:1085600001E025FA0EFC12F854EC4CEA0E0E02F86B
:1085700054EC720612D500F1060E0DF1600C13F8E2
:108580001E2003EB4E0E62449EF801E025FA0EFC1D
:1085900012F854EC4CEA0E0E02F854EC320610D5E8
:1085A000C61D0DF1600E13F8162003EB460672444B
:1085B000767825FA06FE12F8546C4EEA060602F8A2
:1085C000546C083040E718AB03EBE503204613F882
:1085D000542C05F0070328FA03F1114029FA03F39C
:1085E0000CBF0291029601A9134005F1020514BFC8
:1085F00001960193FFF76EFEB5F5257FE3D1204686
:10860000FFF780FE7B1E07F12802002103F8011FFF
:108610009A42FBD1134D40F24912012604EBE201CC
:1086200002F0070E91F82C0315F80E10C2F5A47392
:10863000084203F1010307D0D80803F00703395CAF
:1086400006FA03F30B433B5412F1FF32E6D23946EC
:108650002046FFF7B9FE19B0BDE8F08378F40008B2
:1086600050EF0008DBF4000830B583688DB0044695
:108670005B0009B143F00103A360236FD80803F046
:10868000070229B121181A4DAD5C0A7B2A4304E088
:108690002118184DAD5C0A7B2A4001332044B3F504
:1086A000257F0273236721D104F10C0501AA294615
:1086B0002046FFF7AFFEC0B101210F48FAF730FFA7
:1086C00001210D48FAF73AFF01A92046FFF732FCD5
:1086D0000E220021284604F04FFB002323670223CB
:1086E00063714FF41653636700E060710DB030BDE5
:1086F00076F50008E3F40008006500202DE9F0415C
:1087000004460D4616464FF000081F461FFA88F330
:108710009F423DD936F81830D4F858231344C4F892
:108720005833B4F85C330133A4F85C3335F81810CF
:108730002379C90B8B4209D02368B3F5004F2ABFB8
:108740006FF4CC7203F299139B1823602368217194
:1087500003F54C523332B2F5803F01D2226014E06F
:10876000A3F54C43CD3B23606379012B0AD005D39D
:10877000022B0AD12046FFF779FC06E02046FFF7DE
:1087800013FC02E02046FFF76FFF08F10108BDE788
:10879000BDE8F08110B500210446FDF717FF012167
:1087A00004F65460FDF712FF204610BD2DE9F84F86
:1087B00006469DF828A0002099468C1E951E1F464F
:1087C000834606F65468C9EB07039BB29A4519D94C
:1087D00017F8013B042B03D0082B04D1304600E0EE
:1087E0004046FDF741FF35F8022F34F9021F3046AD
:1087F000FEF7FCF82A88B4F9001083464046FEF7DD
:10880000F5F8E0E7BBF1000F0CBF0146012102487B
:10881000BDE8F84FFAF784BE0065002038B504467D
:108820000D46FEF7B7F8294604F65460BDE8384017
:10883000FEF7B0B838B504460D46FEF7AEF8294647
:1088400004F65460BDE83840FEF7A7B810B50446FA
:10885000FDF716FF04F65460BDE81040FDF710BFA9
:1088600010B50023038104464381018003734373E1
:10887000480004F049F96060204610BD4289038930
:1088800092B29BB29A42028803D1037B93B91046FD
:1088900012E04189038989B29BB2994239BF0389A9
:1088A0004089438900893ABF12FA80F0C01A181A29
:1088B00080B201E000207047824238BF002070473C
:1088C0004289038992B29BB29A4205D1027B02F09F
:1088D000FF039AB1008870474289038992B29BB224
:1088E0009A4223BF428903890088038935BF4089A2
:1088F00010FA83F0181A801A80B270471846704731
:10890000037B10B503F0FF021BB10123437300206A
:1089100010BD038944689BB224F8131003890188B1
:1089200001339BB2038103899BB2994298BF0281B4
:108930000289438992B29BB29A424FF0010308BF69
:108940000373184610BD034600895A8980B292B25B
:10895000904204D11A7B02F0FF0002B970475A8995
:10896000586892B230F812200A80002119735A898F
:108970001888013292B25A815A8992B2904200D834
:1089800059810120704703460022407B5A7370478B
:10899000002303814373438103737047002310B5A1
:1089A0000446037043704360083004F12A01024614
:1089B00002F8013B8A42FBD1002384F82A302222AC
:1089C000024904F03FF9204610BD00BF6FF80008CF
:1089D00070B50F4E047FC1EBC101731804F00F0492
:1089E0005A78C2759A780276DA7842761A7982765F
:1089F0005A79C276827D9B7922F00F05725C23F052
:108A00000F0302F00F022A4323438275037770BDE0
:108A10008AF7000870B50F4E047FC1EBC1017318CF
:108A200004F00F045A78C2759A780276DA784276A2
:108A30001A7982765A79C276827D9B7922F00F0567
:108A4000725C23F00F0302F00F022A432343827566
:108A5000037770BD01F8000810B504462E4801F0F8
:108A600005FC2D4801F0EAFA002854D06378013B58
:108A7000032B4ED8DFE803F00216303B01212648D5
:108A800001F046FC09222549234801F027FA222259
:108A90002349214801F0F4F901211F4801F06CFA43
:108AA000022337E094F82A102046FFF791FF222294
:108AB00004F10801184801F0E3F994F82A30052B75
:108AC00006D1002384F82A30237823BB032321E036
:108AD000013384F82A3010BD222212490E4801F0D9
:108AE000CFF90D4801F02FFC0423606012E00A4822
:108AF00001F029FC63681E3398420CD90021064816
:108B000001F03AFA044801F01BFC002384F82A30F3
:108B100000E00023637010BD8C330020F8F70008DC
:108B20004DF80008B4F7000810B504461C48F7F7E4
:108B30002FFC1B48F7F78CFC88B36378022B0AD014
:108B4000032B20D0012B26D1222216491448F7F7F7
:108B5000D3FB02231DE094F82A102046FFF75AFFAA
:108B6000222204F108010E48F7F7C6FB94F82A30D8
:108B7000052B06D1002384F82A3023787BB9032300
:108B800007E0013309E0222207490548F7F7B4FB63
:108B90000023637010BD0023637084F82A3010BD79
:108BA00054B00020D6F700082BF8000808B5124B87
:108BB0001B785C3B062B1DD8DFE803F0181C14045F
:108BC0001C1C0400017841B10C48012101F0E2F9BC
:108BD0000A48BDE8084001F049BB0848BDE8084024
:108BE00001F0D8B9BDE80840FFF736BFBDE808403E
:108BF000FFF79ABF08BD00BF883300208C330020E8
:108C0000012A034610D1097801290CBF0122002254
:108C100002700BD1407848B9054A127802F0FD0283
:108C20005C2A04D1597070470420704700207047B7
:108C300088330020002202704270704710B504464D
:108C40000F48FDF799FB0E48FDF724FCB8B1637897
:108C5000012B02D0022B07D00FE0D9220949084886
:108C6000FDF70CFB022309E0D92207490448FDF770
:108C700005FB237813B1012300E00023637010BDCE
:108C800078340020F0020020C9030020012A0BD113
:108C90000A78012A0CBF01230023037006D1437810
:108CA00023B942701846704704207047002070476F
:108CB00038B504460023218083814374C381037443
:108CC00048000D4603F020FF6060284603F01CFFBB
:108CD000A060204638BDC289838992B29BB29A4275
:108CE000028803D1037C93B9104612E0C1898389BD
:108CF00089B29BB2994239BF8389C089C38980896F
:108D00003ABF12FA80F0C01A181A80B201E00020AF
:108D10007047824238BF00207047C289838992B26F
:108D20009BB29A4205D1027C02F0FF039AB10088FF
:108D30007047C289838992B29BB29A4223BFC2898B
:108D400083890088838935BFC08910FA83F0181A97
:108D5000801A80B2704718467047037C30B503F024
:108D6000FF041BB101234374002030BD8389456893
:108D70009BB225F81310838981689BB2CA548389FA
:108D8000028801339BB2838183899BB29A4298BF48
:108D900084818289C38992B29BB29A424FF00103C7
:108DA00008BF0374184630BD10B503468489C089D6
:108DB000A4B280B2844204D11C7C04F0FF0004B948
:108DC00010BDD8895C6880B234F810000880D98959
:108DD000986889B2415C117000211974DA89188889
:108DE000013292B2DA81DA8992B2904200D8D98106
:108DF000012010BD03460022407C5A747047704722
:108E0000B1F5006F10D34FF4802340F6754021F484
:108E1000FF6222F007023AB1194201D15B08FBE779
:108E2000DA0A42435140F2E70846704710B54C78E1
:108E30000B78E40004EBC3238C7803EB5414214635
:108E4000FFF7DEFF034B53F820006040C0F3C7205C
:108E500010BD00BF94FA0008F7B54C7B0D7D164697
:108E60000A7B1F46A30943EA82038DF80430CB7CBA
:108E7000A4009B0003F03C0324F03F041C4344EA9D
:108E80009514AD0025F00F0501A98DF805408DF86A
:108E90000650FFF7CBFF030900F00F003370387066
:108EA00003B0F0BD02F00F0242EA0111C9B2134A49
:108EB00070B51C7B32F811005D7B24F03F04C6B214
:108EC00044EA91041C7305F00F05B40804F0300265
:108ED00045EA81111143DA7C597322F00F0204F044
:108EE0000F0414431A7DDC7402F00302800A42EA84
:108EF000861200F03C001043187570BD92F800080F
:108F0000F8B54FF47A61044604F12807FDF7D0FA6A
:108F1000002323616361A361A3832362636204F17D
:108F200048063A4622F8023BB242FBD104F1D40291
:108F30003346002123F8021B9342FBD104F28452F2
:108F4000002103F8011B93424FF00005F9D1F023F3
:108F5000A4F8883540F6B833C4F88C352946A4F80F
:108F60008455A4F88655C4F890552022384603F05D
:108F700003FF8C222946304603F0FEFE0A232374A9
:108F800009236382044B63611623A383034BA76108
:108F9000266263622046F8BDCE040020A2040020B1
:108FA000312A70B506460C460ED1FDF793FA2F28EC
:108FB0000CD904F1300514F8011F3046FDF7CCFA46
:108FC000AC42F8D1002070BD042070BD052070BDFA
:108FD000F0B50023ADB00446F52540F2DF264FF68C
:108FE00021574FF60B7E01F0C002802A02A80BD059
:108FF000C02A06D0002A0CBF72463A4620F8132039
:1090000004E020F8136001E020F8135001338A00D7
:10901000042BD1B2E7D104AA014604F1100003F0F9
:10902000E5F818AA04A904F11C00282303F0DAFAD1
:109030000023009318AA282305210248FAF70CFA06
:109040002DB0F0BD0065002030B5ADB00024054660
:1090500004AA02A9042310300294039403F0C6F872
:1090600018AA04A905F11C00282303F0BBFA0094F8
:10907000282318AA05210248FAF7EEF92DB030BDD1
:1090800000650020B0F8843570B504462BB1404827
:10909000404EFAF741FA05461EE0FDF73DFA00287A
:1090A00051D115E0E218572182F8D4105A1C14FA55
:1090B00082F2752182F8D410DA1C023314FA83F399
:1090C000A4F88425FD2283F8D4200023A4F8863553
:1090D000B4F884350BB3DAE7282D58D9B4F88635BF
:1090E0005A1C2344A4F8862593F8D4102046FFF791
:1090F0006FFF3378283DADB21BB1D4F88C35C4F87E
:109100009035B4F88625B4F884359A42E4D3002328
:10911000A4F88635A4F8843570BDD4F89035B3B37F
:109120001B48FAF7F9F90546282D30D92046FFF7F4
:109130008BFFD4F89035283D013BADB2C4F8903593
:10914000002BF1D170BD144B1A787AB9B4F8885558
:109150005F2193B2AB42B4F88435A3D2581C2344A8
:10916000A4F88405013283F8D410F2E730252046B4
:10917000FDF718FAB4F88435013D5A1C234415F064
:10918000FF05A4F8842583F8D400F0D19DE770BDD5
:109190000065002058020020FC64002001EB410122
:1091A000490001F5967189B2B1F5966F8ABF4FF407
:1091B0009663A0F88815A0F88835704708B5FDF7C4
:1091C00089F93023B0FBF3F0C0B208BD4FF4167339
:1091D0005943C0F88C15704700224FF6FF710260AA
:1091E00042600181428170472DE9F34104460E46F9
:1091F0000025174645F6BF58ABB29F4233D936F823
:1092000015106368CA18638962608B42238938BF6E
:1092100061818B42236888BF2181013343452360EC
:109220001FD9B2FBF3F362898DF80120110A22895C
:109230008DF800108DF80320110AC3F307228DF872
:1092400002108DF804206946062208488DF8053082
:10925000F8F758F900234FF6FF722360636022810C
:1092600063810135C8E702B0BDE8F08128300020F5
:1092700000220270428070471FB504469948FAF7F1
:1092800031FF2378002B00F02A819648FAF7ECFF93
:10929000042840F224819448002301A91A5C5A54FE
:1092A00001330C2BFAD162881520B2FBF0F300FBDE
:1092B00013239BB2002B00F0E080012A04D130235D
:1092C0008DF80D3002239EE0022A01D1342397E06D
:1092D000032A04D131238DF80D306F2393E0042A43
:1092E00007D11F238DF80D302B238DF80E30F62378
:1092F000C1E0052A04D132238DF80D3022238EE0FF
:10930000062A07D124238DF80D302A238DF80E303C
:10931000E023B0E0072A04D133238DF80D303B233E
:109320007DE0082A77D0012B07D125238DF80D3059
:109330004F238DF80E3093239DE0022B07D170232D
:109340008DF80D300B238DF80E30DA2393E0032BCC
:1093500001D1252310E0042B04D133238DF80D30E7
:109360001B235CE0052B04D125238DF80D306F23E2
:109370003DE0062B04D139238DF80D301D235AE032
:10938000072B07D125238DF80D300C238DF80E30D7
:10939000C72370E0082B04D150238DF80D306F23C4
:1093A00007E0092A77D0092B07D125238DF80D3046
:1093B0001E238DF80E30D0235DE00A2A6ED00A2BD2
:1093C00007D121238DF80D300C238DF80E30C223E8
:1093D00051E00B2A65D00B2B01D125231CE00C2A70
:1093E00062D00C2B07D13D238DF80D3002238DF870
:1093F0000E30D7233FE00D2A59D00D2B07D125235E
:109400008DF80D3019238DF80E30DE2333E00E2A4F
:1094100050D00E2B07D150238DF80D306F238DF8CF
:109420000E30B32327E00F2A56D00F2B07D1252368
:109430008DF80D301B238DF80E30D6231BE0102A3B
:109440000BD0102B07D123238DF80D301B238DF863
:109450000E303A230FE0112A06D0112B04D121231C
:109460008DF80D30252303E016238DF80D302923C8
:109470008DF80E30F5238DF80F300C221948FAF7CD
:10948000DDFC638840F276210133B3FBF1F201FB8E
:109490001233638023E00A2B0FD192E70B2B0FD1FD
:1094A0009BE70C2B9FD00EE00D2B0FD1A7E70E2BC7
:1094B000B1D00EE00F2B0FD1B9E70B2B8DD090E779
:1094C0000C2B90D099E70D2B99D0A2E70E2BACD1A5
:1094D000A1E70F2BB5D1AAE7102BBED1B3E704B09B
:1094E00010BD00BFDC100020BD1A0108012A38B5EC
:1094F000044615D10B78012B0CBF012500250378FC
:1095000007D153B94380292206490748FAF770FC6E
:1095100003E013B10448FAF7B7FC2570002038BD0A
:10952000042038BD941A0108DC10002010B5024652
:1095300000F57A71002402F8014B8A424FF00003D3
:10954000F9D1A0F8E833A0F8EA3380F8EC3310BD85
:10955000B0F8E83373B50446002B38D01D481E4ED2
:10956000F9F7DAFF0546182D31D9B4F8EA3319486E
:10957000D91003F00702635CB25C13401BBF0023E9
:109580000093009318230ABF1823144A144A612138
:10959000F9F762FF94F8EC330133DBB2183D312B5D
:1095A000ADB284F8EC3307D9B4F8EA330133A4F848
:1095B000EA33002384F8EC33B4F8EA23B4F8E83350
:1095C0009A42D0D30023A4F8EA33A4F8E83302B0D7
:1095D00070BD00BF00650020F81C01088205002056
:1095E00048B500202DE9F84F04460E4617460021E5
:1095F0004FF47A7203F0C0FB0823A4F8E833DFF8D5
:10960000C0C0DFF8C0800023A4F8EA3384F8EC334C
:10961000DDB2BD423FD200210C20CAB242430CEB66
:1096200002001CF80220A2B316F805E0964501F1ED
:109630000101F1D190F808904FF0000E4FF0004575
:109640005FFA8EF2914524D9B4F8E82341684FEAD5
:10965000E20A35EA010102F007010EF1010E18F8E5
:1096600001B014F80A100CBF4BEA010121EA0B010A
:1096700004F80A1040F2E2318A4205D90023A4F826
:10968000E8330420BDE8F88F0132A4F8E8236D0820
:10969000D6E70133BCE7B4F8E823082AEED0053258
:1096A00092B2A4F8E8230449044812B2F8F700FA89
:1096B0000020BDE8F88F00BFC91A0108283000203B
:1096C000E81A0108F81C01080023A0F8E833A0F804
:1096D000EA3380F8EC337047024A00231380024AD1
:1096E0001380704778B500207EB90020024A00231D
:1096F0001380024A1380704786BD00207CB9002089
:10970000064B1888064B1A8880B293B2984286BFDF
:1097100003F50072101A181A80B270477EB9002043
:1097200078B50020064B1888064B1A8880B293B291
:10973000984286BF03F50072101A181A80B270475B
:109740007CB9002086BD002008B58021024801F0C8
:10975000BFFC0028F9D108BD0010014010B5044637
:10976000FFF7CEFFB0F5007F17D20D4B0D491A88D9
:109770000D4892B28C541A88013292B21A801A881B
:1097800092B2B2F5007F24BF00221A8040F2277106
:10979000012201F07BFC012010BD002010BD00BFA4
:1097A00078B5002084B900200010014008B540F2CF
:1097B00025512A4801F08CFCF0B1284801F0D6FB75
:1097C0000146FFF7AFFFB0F5007F10D2244B2548CC
:1097D0001A8892B2C9B281541A88013292B21A80A0
:1097E0001A8892B2B2F5007F24BF00221A8040F29C
:1097F00025511A4801F08CFC40F22771174801F0FE
:1098000067FC48B3184B1988184B1A8889B292B272
:10981000914214D01A881649104892B2895C1A886D
:10982000013292B21A801A8892B2B2F5007F28BF34
:109830000022C9B228BF1A8001F094FB05E0002283
:1098400040F22771054801F021FC40F227710348DE
:10985000BDE8084001F05CBC08BD00BF001001403D
:1098600086BD00207AB5002078B500207EB90020A2
:1098700084B90020F0B5012189B02D4E0746084675
:1098800001F0E2F80121102001F00EF93046072224
:10989000092100F069FE07220A21304600F064FE2B
:1098A0000124252301A88DF804308DF807408DF898
:1098B00005408DF8064001F0E1F902A800F018FE1D
:1098C00000254FF4C062022302A9304602928DF8AF
:1098D0000C308DF80D308DF80E508DF80F4000F0E3
:1098E000C5FD04A801F0F0FAADF81450ADF816501B
:1098F000ADF81850ADF81C5005F1804505F58835D8
:109900000C2304A92846ADF81A30049701F084FA14
:109910002146284601F0F9FA224640F22551284610
:1099200001F0B4FBFFF7D8FEFFF7E0FE09B0F0BD91
:109930000000024008B5FFF7F5FE003018BF012017
:1099400008BD08B5FFF7DCFEC0F5007008BD0000DB
:10995000094B0A491A8892B2885C1A88013292B27D
:109960001A801A8892B2B2F5007F28BF0022C0B2D6
:1099700028BF1A80704700BF7CB900207AB500204C
:10998000013938B5441E4518AC4204D014F8010F13
:10999000FFF7E4FEF8E7012240F227710248BDE834
:1099A000384001F073BB00BF00100140024A0023A1
:1099B0001380024A138070477AB7002080B90020D4
:1099C000024A00231380024A1380704784BD00209E
:1099D00082B90020064B1888064B1A8880B293B2D1
:1099E000984286BF03F50072101A181A80B27047A9
:1099F00080B900207AB70020064B1888064B1A88D9
:109A000080B293B2984286BF03F50072101A181AFA
:109A100080B2704782B9002084BD002008B5802143
:109A2000024801F055FB0028F9D108BD0050004064
:109A300010B50446FFF7CEFFB0F5007F17D20D4BEF
:109A40000D491A880D4892B28C541A88013292B28C
:109A50001A801A8892B2B2F5007F24BF00221A80C1
:109A600040F22771012201F011FB012010BD0020FE
:109A700010BD00BF7AB7002084BB0020005000401A
:109A800008B540F225512A4801F022FBF0B12848E0
:109A900001F06CFA0146FFF7AFFFB0F5007F10D27E
:109AA000244B25481A8892B2C9B281541A880132CF
:109AB00092B21A801A8892B2B2F5007F24BF0022B7
:109AC0001A8040F225511A4801F022FB40F227711A
:109AD000174801F0FDFA48B3184B1988184B1A883B
:109AE00089B292B2914214D01A881649104892B2A3
:109AF000895C1A88013292B21A801A8892B2B2F541
:109B0000007F28BF0022C9B228BF1A8001F02AFABC
:109B100005E0002240F22771054801F0B7FA40F253
:109B200027710348BDE8084001F0F2BA08BD00BF44
:109B30000050004084BD00207CB700207AB7002090
:109B400080B9002084BB00202DE9F041012188B0BC
:109B50008046042000F078FF304F314E012108206C
:109B600000F072FF01214FF4801000F091FF3846A1
:109B700008220C2100F0F8FC08220221304600F0F7
:109B8000F3FC0124352301A88DF804308DF807403B
:109B90008DF805408DF8064001F070F802A800F03D
:109BA000A7FC00254FF48052022302A938460292F6
:109BB0008DF80E508DF80C308DF80D308DF80F406B
:109BC00000F054FC042302A93046029300F04EFC3E
:109BD00004A801F079F9ADF81450ADF81650ADF8BD
:109BE0001850ADF81C500F4DCDF810800C2304A96F
:109BF0002846ADF81A3001F00FF92146284601F049
:109C000084F9224640F22551284601F03FFAFFF739
:109C1000CDFEFFF7D5FE08B0BDE8F0810008024098
:109C2000000C02400050004008B5FFF7E5FE003090
:109C300018BF012008BD08B5FFF7CCFEC0F50070C5
:109C400008BD0000094B0A491A8892B2885C1A883C
:109C5000013292B21A801A8892B2B2F5007F28BF00
:109C60000022C0B228BF1A80704700BF82B900200E
:109C70007CB70020013938B5441E4518AC4204D0E9
:109C800014F8010FFFF7D4FEF8E7012240F2277124
:109C90000248BDE8384001F0F9B900BF005000406B
:109CA0000129104602D0032902D07047FFF7E2BD18
:109CB000FFF74ABF012908B504D0032905D1FFF7F2
:109CC000B3FF08BDFFF736FE08BD002008BD01291F
:109CD00003D0032903D1FFF7AEBFFFF732BE002048
:109CE0007047012903D0032903D1FFF7ABBFFFF76A
:109CF0002FBE0020704710B5012910469DF808407E
:109D000002D0032908D010BD1946FFF739FE5CB117
:109D1000BDE81040FFF718BD1946FFF7ABFF1CB1B7
:109D2000BDE81040FFF77ABE10BD00002DE9F041FC
:109D30004FF4B9710446FCF7BBFB4FF4B97104F161
:109D40001000FCF7B5FB04F12C06002323626362CC
:109D5000A36204F14C01324622F8023B8A42FBD155
:109D60004FF0000384F84C3004F14D0204F16E0111
:109D7000002002F8010B8A424FF00003F9D104F1F0
:109D80006F0884F86E3004F17B07424602F8013B0D
:109D9000BA42FBD104F187023B46002103F8011BC4
:109DA0009342FBD104F1AF02002103F8011B93425F
:109DB000FBD104F1D702002103F8011B9A424FF0B6
:109DC0000005F9D12946A4F8D850A4F8DA50C4F80F
:109DD000DC50C4F8E050C4F8E45084F8E85084F84B
:109DE000E9502022304602F0C7FF052384F82030D6
:109DF000092363840B4B6362A6620C220A4938462E
:109E000002F020FF0C220849404602F01BFF84F8B4
:109E1000E85084F8E950C4F8E050C4F8E450204613
:109E2000BDE8F081B2050020441D0108222A70B56A
:109E300005460C461CD1FCF74DFB20281AD995F895
:109E4000E8302BB12846FCF740FB002385F8E830CA
:109E500004F1210614F8011F2846FCF77DFBB442EB
:109E6000F8D1064B187838B9012385F84C3070BD0D
:109E7000042070BD052070BD002070BDFC64002072
:109E8000222AF8B505460C461FD100F110063046CF
:109E9000FCF720FB20281AD995F8E9302BB1304681
:109EA000FCF713FB002385F8E93004F1210714F8CF
:109EB000011F3046FCF750FBBC42F8D1064B187826
:109EC00038B9012385F84C30F8BD0420F8BD0520D1
:109ED000F8BD0020F8BD00BFFC640020092AF8B5D9
:109EE00004460D462CD10C2200217B3002F044FFA9
:109EF000144F1548002202F0070ED110D35D6E5C9E
:109F000010F80E100E424FEAE30103F0070317BFEB
:109F10006618C65C10F803E096F87B3008BF63183B
:109F200002F1010208BF93F87B30214414BF4EEACE
:109F30000303B343442A81F87B30DCD10020F8BD11
:109F40000420F8BD001D0108711D0108012A11D16E
:109F50000978012907D002290CD10023C0F8E43088
:109F600080F8E92004E00023C0F8E03080F8E81031
:109F70001846704704207047002380F84C10C0F842
:109F8000DC30C0F8E030C0F8E43080F8E83080F829
:109F9000E9307047002914BF0523002380F84C30B6
:109FA000704700002DE9F0414FF63A6C064617461F
:109FB00094B000244FF4E37240F252504FF6AE2EAC
:109FC00001F0C003802B03AD0BD0C02B06D0002BBB
:109FD0000CBF6346734625F8143004E025F81400DE
:109FE00001E025F8142001348900042CC9B2E7D11E
:109FF0000DF1140814220021404602F0BDFE234654
:10A000000AAA294606F120008DF81E7002F0EEF82B
:10A01000CDF8008014230AAA02210348F9F71CFA9C
:10A0200014B0BDE8F08100BF0065002008B5FCF762
:10A0300051FA2323B0FBF3F0C0B208BD08B51030CD
:10A04000FCF748FA2323B0FBF3F0C0B208BD2DE9BA
:10A05000F04100EB0116044630460D46FCF75CFA71
:10A06000202820D9D4F8DC30132B1CD905F1380373
:10A0700054F82330052B16D904F1AE0504F1CF07AF
:10A080004FF000083046FCF78DFA05F8010FBD428D
:10A0900005F8288CF6D12123A4F8D8300023A4F8A1
:10A0A000DA30BDE8F0812544002285F8E82004F18B
:10A0B0004C0304F16D0113F8010F83F862008B4229
:10A0C00083F83A20F7D1E6E71A4B1B78622B10B5DC
:10A0D0000DD100F1AE0300F1CF025F24002103F89F
:10A0E000014F9A4203F8281CF9D121231CE05F2B71
:10A0F0001CD100F1AE0300F1B5025524002103F894
:10A10000014F934203F8281CF9D103465F2203F85C
:10A11000B62FFF2400F1BD02002103F8014F9A423F
:10A1200003F8281CF9D10F23A0F8D8300023A0F899
:10A13000DA3010BD88330020D0F8DC3001332DE94F
:10A14000F041C0F8DC30D0F8E0300133C0F8E03046
:10A15000D0F8E4300133C0F8E43090F86E300B2BC7
:10A1600084BF002380F86E3090F86E300446884635
:10A17000164600F16F0583B9FCF7CEF938B904F142
:10A180001000FCF7C9F910B90C22374902E00C2283
:10A1900004F17B01284602F055FD94F86E1003226D
:10A1A000294404F1AF0002F04DFD012E0CBF08233D
:10A1B000042384F88930D4F8DC300020132B84F891
:10A1C000870084F8880006D904EB0610FCF7A4F990
:10A1D000003018BF012008F1FF3394F86E105E4282
:10A1E0005E4129B1B1F1090518BF0125012701E040
:10A1F0000F46012594F8AF3094F8B020B8F1010F64
:10A2000080EA060E43EAC0100CBF08230023002F8B
:10A2100040EA030014BF802300231A4342EAC50228
:10A22000774514BF0223002313437E4084F8B030E7
:10A2300094F8B13084F8AF00B54214BF2026002650
:10A240001E43754514BF0225002503233543033102
:10A25000A4F8D83084F8B150002384F86E10A4F824
:10A26000DA30BDE8F08100BF441D010838B590F830
:10A270004C300446002B47D0B0F8D8200ABB013B35
:10A28000042B17D8DFE803F003160E081300002193
:10A29000FFF7DDFE042312E000220121FFF74CFF4F
:10A2A00003230CE00121FFF7D2FE022307E0FFF7B2
:10A2B0000BFF06E001220021FFF73EFF012384F897
:10A2C0004C30B4F8D830FBB11048F9F725F9054601
:10A2D000142D19D9B4F8DA30E218013392F8AF101E
:10A2E00092F88720A4F8DA302046FFF75BFEB4F836
:10A2F000DA20B4F8D830143D9A42ADB2E8D3002346
:10A30000A4F8DA30A4F8D83038BD00BF00650020CA
:10A3100037B500F14D040D4621220749204602F0D1
:10A3200091FC01A8FEF76BFD23460922294601A8EE
:10A33000FEF7B8FD03B030BD501D0108FCF7C5B8ED
:10A340001030FCF7C2B8D0F8DC00704708B53C4BC1
:10A35000984206D10121084600F0B2FB00210120FD
:10A3600068E0384B984206D10121022000F0A8FB9A
:10A37000002102205EE0344B984206D101210420E6
:10A3800000F09EFB0021042054E0304B984206D19F
:10A390000121082000F094FB002108204AE02C4B0A
:10A3A000984206D10121102000F08AFB00211020E4
:10A3B00040E0284B984206D10121202000F080FB8C
:10A3C0000021202036E0244B984206D10121402074
:10A3D00000F076FB002140202CE0204B984206D173
:10A3E0000121802000F06CFB0021802022E01C4B2A
:10A3F000984208D101214FF4807000F061FB0021E8
:10A400004FF4807016E0174B984208D101214FF4A9
:10A41000007000F055FB00214FF400700AE0124B71
:10A4200098420BD101214FF4806000F049FB0021DC
:10A430004FF48060BDE8084000F042BB08BD00BF9B
:10A44000000002400004024000080240000C0240EC
:10A45000001002400014024000180240001C02409C
:10A460000020024000240240002802402DE9F04371
:10A470000F6800234FF0010E03260EFA03FC3CEA9E
:10A48000070230D15A00056806FA02F4E443254079
:10A4900005600D79D0F8008005FA02F9013D49EA1E
:10A4A0000808012DC0F8008011D885682C40846010
:10A4B0004C798568944025438560446824EA0C04FF
:10A4C00044608C7945689C40A4B22C434460C468C5
:10A4D00006FA02F524EA0504C460CD79C46805FAD9
:10A4E00002F22243C2600133102BC6D1BDE8F083D3
:10A4F0004FF6FF7303600023037143718371C371CF
:10A50000704782B04FF480330193019B0B4301935A
:10A51000019BC361C161019BC361C3690193C369AD
:10A52000019302B070470369194214BF0120002053
:10A530007047006980B270474369194214BF012017
:10A5400000207047406980B27047018370474183A3
:10A5500070470AB10183704741837047416170477A
:10A56000436959404161704701F00703C90800EB96
:10A57000810010B59B00046A0F21994024EA010173
:10A580000162016A9A400A43026210BD08B50121C6
:10A590004FF0005000F0B8FA00214FF00050BDE835
:10A5A000084000F0B1BA000030B5094D40F6FE7326
:10A5B0002A68834022EA030391E8140014438A685E
:10A5C0001443CA68224302FA00F01843286030BDE1
:10A5D000007400400023036043608360C3607047E1
:10A5E000064A012319B1116883400B4303E0116847
:10A5F000834021EA03031360704700BF00740040EA
:10A60000064A0009012319B1516883400B4303E056
:10A610005168834021EA030353607047007400408F
:10A62000044B5A6810B142F0030201E022F0030229
:10A630005A6070470074004082B000230193054BBC
:10A640000193019B083318440190019B196002B0EB
:10A65000704700BF0074004082B000230193054B97
:10A660000193019B143318440190019B196002B0BF
:10A67000704700BF007400400828044B0CBF42EA3A
:10A68000012242EA0142C250704700BF20740040DC
:10A6900082B000230193064B0193019B2C3303EB03
:10A6A00090000190019B186880B202B0704700BF13
:10A6B00000740040064A4FF4805319B1116883407A
:10A6C0000B4303E01168834021EA030313607047E2
:10A6D00000740040054B814012B11A68114302E03A
:10A6E0001A6822EA01011960704700BF0074004037
:10A6F000FFF7F0BF034B5B6B8140194214BF012091
:10A700000020704700740040014B8140596370473E
:10A7100000740040054B1A685B6B814011EA03002E
:10A7200003D00A4214BF012000207047007400408B
:10A73000014B814059637047007400400E4B1A680A
:10A74000002142F001021A6099601A6822F0A852B2
:10A7500022F410221A60094A5A60094AC3F8842078
:10A7600002F18062C3F888201A6822F480221A60FD
:10A77000D960C3F88C1070470038024010300024B4
:10A7800000300020024B00221A701870704700BF82
:10A7900002380240034A136823F0F80343EAC0007A
:10A7A0001060704700380240014B1860704700BFCE
:10A7B00000004742064B002201281A701A7002D08E
:10A7C000042802D070471870704705221A7070472D
:10A7D00070380240014B1860704700BF800E47423E
:10A7E00010B5029C40EA046001435B08013B41EA6A
:10A7F000821242EA0340014B586010BD003802400B
:10A80000014B1860704700BF600047420907034BC7
:10A8100041EA8010C3F88400704700BF003802404E
:10A82000014B1860704700BF68004742120742EAB8
:10A830000161034B41EA8010C3F88800704700BFF4
:10A8400000380240014B1860704700BF700047425B
:10A85000014B1860704700BF4C004742034A9368A1
:10A8600023F0EC63194308439060704700380240BE
:10A87000034A936823F07843194308439060704774
:10A8800000380240034A936823F0030318439060A2
:10A89000704700BF00380240024B986800F00C007F
:10A8A000704700BF00380240034A936823F0F0036A
:10A8B00018439060704700BF00380240034A936815
:10A8C00023F4E05318439060704700BF0038024003
:10A8D000034A936823F4604343EAC00090607047E2
:10A8E000003802401D4A936803F00C03042B10B596
:10A8F00003D0082B03D01A4B18E01A4B16E051680E
:10A90000536811F4800F03F03F03516814BF154AD8
:10A91000134AB2FBF3F3114A5268C2F30142C1F386
:10A92000881101324B435200B3FBF2F30B4A036030
:10A9300093680D49C3F30313CC5C0368E3404360A1
:10A940009468C4F382240C5D23FA04F48460926852
:10A95000C2F342328A5CD340C36010BD003802406B
:10A960000024F40000127A000C06002000F440736A
:10A97000B3F5407F084A08D1936820F0704123F472
:10A98000F81321F440710B439360136FC0F30B0075
:10A9900018431067704700BF00380240014B186031
:10A9A000704700BF3C0E4742014B1860704700BF24
:10A9B000400E4742014B1860704700BF5C014742A0
:10A9C000044AD2F88C3023F440131843C2F88C00A8
:10A9D000704700BF00380240044AD2F88C3023F49C
:10A9E00040031843C2F88C00704700BF0038024093
:10A9F000044AD2F88C30013823F01F030343C2F815
:10AA00008C30704700380240054AD2F88C3001384B
:10AA100023F4F85343EA0023C2F88C30704700BF98
:10AA200000380240044AD2F88C3023F440331843F3
:10AA3000C2F88C00704700BF00380240014B18601C
:10AA4000704700BFE0114742044B1A6B09B1104335
:10AA500001E022EA00001863704700BF003802409E
:10AA6000044B5A6B09B1104301E022EA000058631D
:10AA7000704700BF00380240044B9A6B09B1104385
:10AA800001E022EA00009863704700BF00380240EE
:10AA9000044B1A6C09B1104301E022EA000018646B
:10AAA000704700BF00380240044B5A6C09B1104394
:10AAB00001E022EA00005864704700BF00380240FD
:10AAC000044B1A6909B1104301E022EA0000186141
:10AAD000704700BF00380240044B5A6909B1104367
:10AAE00001E022EA00005861704700BF00380240D0
:10AAF000044B9A6909B1104301E022EA0000986111
:10AB0000704700BF00380240044B1A6A09B1104375
:10AB100001E022EA00001862704700BF00380240DE
:10AB2000044B5A6A09B1104301E022EA000058625E
:10AB3000704700BF00380240044B1A6D09B1104342
:10AB400001E022EA00001865704700BF00380240AB
:10AB5000044B5A6D09B1104301E022EA0000586528
:10AB6000704700BF00380240044B9A6D09B1104392
:10AB700001E022EA00009865704700BF00380240FB
:10AB8000044B1A6E09B1104301E022EA0000186676
:10AB9000704700BF00380240044B5A6E09B11043A1
:10ABA00001E022EA00005866704700BF003802400A
:10ABB000044B1A6F01280CBF42F0080222F0080271
:10ABC0001A67704700380240044B1A7809B11043E5
:10ABD00001E022EA00001870704700BF0D38024003
:10ABE0004209012A074B01D11B6803E0022A0CBF6E
:10ABF0001B6F5B6F00F01F0023FA00F000F00100F4
:10AC0000704700BF0038024007B500230193312090
:10AC1000FFF7E6FF019B01330193019BB3F5A04FC2
:10AC200001D00028F3D03120FFF7DAFF003018BF41
:10AC3000012003B05DF804FB024A536F43F08073B8
:10AC40005367704700380240034BDB68184214BF5B
:10AC500001200020704700BF00380240014B1870EF
:10AC6000704700BF0E38024040F0BF60024B40F416
:10AC70000030D860704700BF00ED00E0C278037874
:10AC800030B51AB3174A4578D168C943C1F30221D8
:10AC9000C1F10402D2B205FA02F2D4B20F220A4183
:10ACA00081780A40224303F1604303F561431201B6
:10ACB000D2B283F8002303780122590903F01F035D
:10ACC00002FA03F3084A42F8213030BD5A09012143
:10ACD00003F01F0301FA03F32032034941F8223045
:10ACE00030BD00BF00ED00E000E100E021F0604178
:10ACF00021F07F01014B08439860704700ED00E0B0
:10AD0000044B1A6909B1104301E022EA00001861FE
:10AD1000704700BF00ED00E0044B1A6804280CBF28
:10AD200042F0040222F004021A60704710E000E0D2
:10AD300008B5314B984206D101211020FFF7F0FEF3
:10AD40000021102038E02D4B984208D101214FF40A
:10AD50000030FFF7D9FE00214FF4003047E0284BC8
:10AD6000984208D101214FF48020FFF7CDFE002149
:10AD70004FF480203BE0234B984208D101214FF44F
:10AD80000020FFF7C1FE00214FF400202FE01E4BF2
:10AD9000984208D101214FF48010FFF7B5FE002141
:10ADA0004FF4801023E0194B984209D10121202053
:10ADB000FFF7B6FE00212020BDE80840FFF7B0BE37
:10ADC000134B984208D101214FF08040FFF79CFEC1
:10ADD00000214FF080400AE00E4B98420BD1012138
:10ADE0004FF00040FFF790FE00214FF00040BDE81B
:10ADF0000840FFF789BE08BD001001400044004034
:10AE000000480040004C0040005000400014014049
:10AE100000780040007C00407FB5038ACA889BB25E
:10AE200023F440531343038283890E469BB223F4D9
:10AE3000B053898823F00C0233890B4371890B438B
:10AE40009BB213438381838AB2899BB223F44073FC
:10AE50001343838204466846FFF744FD194B9C4226
:10AE600003D003F580639C4201D1039D00E0029D65
:10AE7000A389316813F4004F4FF0190202FB05F269
:10AE800014BF4D008D00B2FBF5F5A2896426B5FB19
:10AE9000F6F000010109120406FB115307D5D90091
:10AEA0003231B1FBF6F202F00702104306E01A015C
:10AEB0003232B2FBF6F303F00F03184380B2208165
:10AEC00004B070BD001001404FF4165303600C2213
:10AED00000238380C3800381428183817047038A7A
:10AEE0009BB223F4706210B54B880C8823438C8886
:10AEF000C98823430B439BB21343038210BD002335
:10AF0000038043808380C3807047838919B19BB2DB
:10AF100043F4005303E023F400531B041B0C838110
:10AF20007047038B03F47F430383038B9BB2194366
:10AF300001837047838929B16FEA43436FEA534322
:10AF40009BB201E0C3F30E0383817047838A19B17A
:10AF50009BB243F4006303E023F400631B041B0C67
:10AF600083827047C1F30801818070478088C0F3F5
:10AF700008007047038A23F00F031B041B0C038295
:10AF8000038A9BB2194301827047838919B19BB22E
:10AF900043F0020303E023F002031B041B0C838134
:10AFA0007047838923F400631B041B0C838183890E
:10AFB0009BB2194381817047038A23F020031B044D
:10AFC0001B0C0382038A9BB2194301827047038AD8
:10AFD00019B19BB243F4804303E023F480431B0484
:10AFE0001B0C0382704783899BB243F0010383816A
:10AFF0007047838A19B19BB243F0080303E023F042
:10B0000008031B041B0C83827047038BDBB2038392
:10B01000038B9BB243EA012101837047838A19B1F4
:10B020009BB243F0200303E023F020031B041B0C1E
:10B0300083827047838A19B19BB243F0100303E007
:10B0400023F010031B041B0C83827047838A23F0B8
:10B0500004031B041B0C8382838A9BB219438182E5
:10B060007047838A19B19BB243F0020303E023F0D7
:10B0700002031B041B0C83827047838A9BB20AB1B4
:10B08000194301E023EA010181827047012310B5D1
:10B09000C1F342149C4201F01F0103FA01F101D1F6
:10B0A0000C3003E0022C0CBF1030143003680AB1DE
:10B0B000194301E023EA0101016010BD0388194230
:10B0C00014BF012000207047C94389B20180704736
:10B0D000012310B5C1F3421401F01F029C4203FA90
:10B0E00002F201D1838903E0022C0CBF038A838A18
:10B0F0009BB21340028892B243B10123090A03FABA
:10B1000001F10A4214BF1846002010BD184610BDB8
:10B11000090A012303FA01F1C94389B2018070478A
:10B1200030B5048C24F001042404240C0484048B22
:10B13000058CA4B2ADB224F0F304224325F00A0535
:10B1400042EA031345F001059AB2294302830184C0
:10B1500030BD30B5048C24F010042404240C048485
:10B16000058B048C25F44075A4B22D052D0D24F01B
:10B17000A00444F0100445EA022242EA033344EA00
:10B1800001119BB28CB20383048430BD08B54D4BD2
:10B19000984206D101210846FFF7C2FC0021012098
:10B1A00044E0B0F1804F06D101210846FFF7ACFC26
:10B1B0000021012081E0444B984206D10121022068
:10B1C000FFF7A2FC0021022077E0404B984206D115
:10B1D00001210420FFF798FC002104206DE03C4B86
:10B1E000984206D101210820FFF78EFC002108209B
:10B1F00063E0384B984206D101211020FFF784FC10
:10B200000021102059E0344B984206D10121202022
:10B21000FFF77AFC002120204FE0304B984209D103
:10B2200001210220FFF77CFC00210220BDE808403C
:10B23000FFF776BC2A4B984208D101214FF48030A9
:10B24000FFF76EFC00214FF48030EFE7254B98426A
:10B2500008D101214FF40030FFF762FC00214FF4C8
:10B260000030E3E7204B984208D101214FF48020C1
:10B27000FFF756FC00214FF48020D7E71B4B984284
:10B2800006D101214020FFF73FFC0021402014E0BF
:10B29000174B984206D101218020FFF735FC002191
:10B2A00080200AE0134B98420BD101214FF48070AB
:10B2B000FFF72AFC00214FF48070BDE80840FFF73B
:10B2C00023BC08BD0000014000040040000800400D
:10B2D000000C004000100040001400400004014039
:10B2E0000040014000440140004801400018004077
:10B2F000001C0040002000401C4A038890429BB282
:10B3000012D002F5806290420ED0B0F1804F0BD087
:10B31000A2F58032904207D002F58062904203D0BD
:10B3200002F58062904203D14A8823F070031343F0
:10B330000F4A904208D002F5806290421FBF23F46A
:10B3400040730A899BB2134303804B68C3620B8826
:10B350000385064B984203D003F58063984201D1E0
:10B360008B7A038601238382704700BF000001406F
:10B37000001000404FF0FF3343600023038003813F
:10B38000438083727047018582827047038823F06F
:10B3900070031B041B0C1943018070474162704706
:10B3A000C1627047406A7047008D80B27047038861
:10B3B00019B19BB243F0020303E023F002031B0424
:10B3C0001B0C03807047038819B19BB243F0040340
:10B3D00003E023F004031B041B0C03807047038865
:10B3E00019B19BB243F0800303E023F080031B04F8
:10B3F0001B0C03807047038823F008031B041B0CFD
:10B40000038003889BB2194301807047038823F4AB
:10B4100040731B041B0C038003889BB219430180FB
:10B420007047038819B19BB243F0010303E023F096
:10B4300001031B041B0C038070470000038C23F0E6
:10B4400001031B041B0C0384038C70B58488028BDE
:10B450000E8822F073021204120C23F00205164328
:10B460008B894A882D0413430F4A2D0C2B4390429D
:10B47000A4B29BB203D002F5806290420ED1CA8979
:10B480000D8A23F0080313438A8823F0040313432F
:10B490004A8A24F4407415432C43A4B28A688480F9
:10B4A00006834263038470BD00000140038C23F0D7
:10B4B00010031B041B0C0384038C30B58588028B9E
:10B4C0000C8822F4E6421204120C42EA042223F011
:10B4D000200394B21B048A891B0C43EA02134A8896
:10B4E00043EA0213124A9042ADB29BB203D002F576
:10B4F0008062904215D123F08003CA899BB243EA4F
:10B5000002124FF6BF7313408A8843EA02130A8A75
:10B5100025F4406545EA82054A8A45EA82059BB2E0
:10B52000ADB28A68858004838263038430BD00BF26
:10B5300000000140038C23F480731B041B0C038464
:10B54000038C30B58488828B0D8822F0730212043C
:10B55000120C23F4007315431B048A891B0C43EA65
:10B5600002234A8843EA0223124A9042A4B29BB2C1
:10B5700003D002F58062904215D123F40063CA899A
:10B580009BB243EA02224FF6FF3313408A8843EA14
:10B5900002230A8A24F4405444EA02144A8A44EA00
:10B5A00002149BB2A4B28A6884808583C263038438
:10B5B00030BD00BF00000140038C23F480531B0406
:10B5C0001B0C0384038C30B58488828B0D8822F495
:10B5D000E6421204120C23F4005342EA05221B0433
:10B5E0008D891B0C43EA05334D8843EA05330B4D27
:10B5F000A842A4B292B29BB203D005F58065A842DE
:10B6000005D10D8A24F4804444EA8514A4B28480D0
:10B6100082838A680264038430BD00BF0000014059
:10B62000002303804380838083608381C3810382FE
:10B630004382704730B5048CA5B201248C4025EAC2
:10B64000040400F11803048421F0080038B9490803
:10B650004FF68F70CC582040C850C8580AE00439C3
:10B66000C1F34E0148F6FF70CC582040C85012027A
:10B67000C85892B20243CA5030BD416370478163DB
:10B680007047C163704701647047038B23F07003F8
:10B690001B041B0C194301837047038B23F4E04305
:10B6A0001B041B0C43EA012189B201837047838B81
:10B6B00023F070031B041B0C194381837047838B99
:10B6C00023F4E0431B041B0C43EA012189B281836C
:10B6D0007047038B23F008031B041B0C19430183E1
:10B6E0007047038B23F400631B041B0C43EA012106
:10B6F00089B201837047838B23F008031B041B0C62
:10B70000194381837047838B23F400631B041B0C54
:10B7100043EA012189B281837047038B23F004033C
:10B720001B041B0C194301837047038B23F48063B4
:10B730001B041B0C43EA012189B201837047838BF0
:10B7400023F004031B041B0C194381837047838B74
:10B7500023F480631B041B0C43EA012189B281831B
:10B760007047038B23F080031B041B0C19430183D8
:10B770007047038BC3F30E0343EA012189B20183AF
:10B780007047838B23F080031B041B0C19438183B8
:10B790007047838BC3F30E0343EA012189B281838F
:10B7A0007047038C23F002031B041B0C1943018414
:10B7B0007047038C23F008031B041B0C19430184FE
:10B7C0007047038C23F020031B041B0C43EA011178
:10B7D00089B201847047038C23F080031B041B0C87
:10B7E00043EA011189B201847047038C23F400738A
:10B7F0001B041B0C43EA012189B201847047038CAE
:10B8000023F400631B041B0C43EA012189B2018469
:10B810007047038C23F400531B041B0C43EA0131D3
:10B8200089B20184704730B5048CA5B201248C40E4
:10B8300025EA04040484038C8A4013439BB20384E6
:10B8400030BD30B5048CA5B204248C4025EA040434
:10B850000484038C8A4013439BB2038430BD0023CD
:10B860000122038043808280C38003817047406B44
:10B870007047806B7047C06B7047006C7047038BDC
:10B8800023F00C031B041B0C0383038B9BB2194393
:10B8900001837047038B23F440631B041B0C038359
:10B8A000038B9BB243EA012189B201837047F8B54B
:10B8B0000C464988A288B4F800E0238900290CBF0F
:10B8C00002260026012A0CBF02270127BEF1000F25
:10B8D0000ED1FFF725FCE188FFF7D1FF3146238920
:10B8E0003A46FFF736FCE188BDE8F840FFF7D2BFE3
:10B8F000FFF72FFCE188FFF7CDFF314623893A4659
:10B90000FFF70EFCE188BDE8F840FFF7B8BF838B76
:10B9100023F00C031B041B0C8383838B9BB2194302
:10B9200081837047838B23F440631B041B0C838348
:10B93000838B9BB243EA012189B281837047F8B5BA
:10B940000E880B898A880D46498836B9FFF7E8FBCF
:10B95000E988BDE8F840FFF792BF042E06D1FFF753
:10B96000F8FBE988BDE8F840FFF794BF082EB5F86A
:10B9700006C0058C1CD125F480752D042D0C058482
:10B98000858B068CADB2B6B225F0F30526F42066A1
:10B9900045EA031346EA01259BB2ADB21A4345F4CA
:10B9A0008075828361460584BDE8F840FFF7AFBF2C
:10B9B00025F480552D042D0C0584B0F81CE0068C70
:10B9C0002EF4407726F400553F056D043F0D6D0CB5
:10B9D00047EA022745EA013547EA0333ADB29BB295
:10B9E00045F48055838361460584BDE8F840FFF740
:10B9F00099BF0A884B8813438A881343CA88134324
:10BA00000A8913434A8913438A8913439BB2A0F8D6
:10BA1000443070470023038043808380C3800381C8
:10BA2000438183817047B0F8443029B16FEA4343C2
:10BA30006FEA53439BB201E0C3F30E03A0F8443016
:10BA40007047838819B19BB243F0040303E023F0ED
:10BA500004031B041B0C83807047838819B19BB2BD
:10BA600043F0010303E023F001031B041B0C83805C
:10BA7000704781827047038A194214BF0120002059
:10BA80007047C94389B201827047038A828911EAEB
:10BA9000030092B203D0114214BF0120002070476E
:10BAA000C94389B2018270470A43A0F84820704711
:10BAB00083899BB20AB1194301E023EA0101818124
:10BAC0007047FFF7F5BF838819B19BB243F00803B5
:10BAD00003E023F008031B041B0C838070470389D9
:10BAE00023F007031B041B0C03817047038923F019
:10BAF00070031B041B0C1943018103899BB243F0A3
:10BB000007030381704738B50D46602D1146044682
:10BB10004FF0010202D1FFF71CFB01E0FFF700FB31
:10BB2000218921F070010904090C2943218123890D
:10BB30009BB243F00703238138BD038923F07003D0
:10BB40001B041B0C194301817047838823F0700389
:10BB50001B041B0C838083889BB219438180704730
:10BB6000038923F007031B041B0C038103899BB289
:10BB7000194301817047038923F080031B041B0CC8
:10BB8000038103899BB219430181704710B5048971
:10BB9000E4B221430A4342EA032399B2018110BD72
:10BBA00010B5FFF7F3FF038923F077031B041B0C89
:10BBB00043F07703038110BD10B5FFF7E7FF03895A
:10BBC0009BB243F48043038110BD70B50689048B9A
:10BBD000058C24F44074ADB224F0030425F0220552
:10BBE00026F0070624042A433604240C360C44F4B9
:10BBF000807442EA0313314344F001049DB2018191
:10BC00000483058470BD838819B19BB243F080031F
:10BC100003E023F080031B041B0C83807047A0F813
:10BC20005010704708B501214FF48070FEF778FF7F
:10BC300000214FF48070BDE80840FEF771BF00009E
:10BC4000436823F040720B6822F4807213430A7930
:10BC500043EA022343600A69CB681A438B6810B534
:10BC60001A438468084B234013434A7943EA42034A
:10BC70008360C36A23F470020B7D013BDBB242EAAE
:10BC80000353C36210BD00BFFDF7FFC00023036074
:10BC9000037143718360C3600361012303757047BF
:10BCA00010B5074C074B6268134090E8060011433B
:10BCB00082681143C2680A431343636010BD00BF2A
:10BCC00000230140E030FCFF0023036043608360F9
:10BCD000C3607047836811B143F0010301E023F0B2
:10BCE000010383607047436823F4400323F4007327
:10BCF000194341607047416282627047436823F094
:10BD00001F03194341607047044B5A6810B142F455
:10BD1000000201E022F400025A6070470023014053
:10BD2000044B5A6810B142F4800201E022F4800210
:10BD30005A60704700230140092970B50DD9A1F15F
:10BD40000A04C66804EB44040725A54026EA050555
:10BD500003FA04F42C43C4600AE0066901EB4104D1
:10BD60000725A54026EA050503FA04F42C430461DF
:10BD7000062A0CD8013A446B02EB82021F2393403F
:10BD800024EA030301FA02F21A43426370BD0C2A4B
:10BD90000CD8073A046B02EB82021F23934024EA7B
:10BDA000030301FA02F21A43026370BD0D3AC46A3A
:10BDB00002EB82021F23934024EA030301FA02F2FA
:10BDC0001A43C26270BD836843F08043836070474A
:10BDD0008068C0F380707047836811B143F480635A
:10BDE00001E023F4806383607047836811B143F0FE
:10BDF000020301E023F002038360704743680139C6
:10BE000023F4604343EA413343607047436811B110
:10BE100043F4006301E023F4006343607047C06CA7
:10BE200080B27047014B1868704700BF082301407B
:10BE3000836811B143F4807301E023F4807383605D
:10BE40007047836811B143F4007301E023F4007379
:10BE500083607047044B5A6810B142F4005201E00D
:10BE600022F400525A60704700230140092970B53E
:10BE70000DD9A1F10A04C66804EB44040725A540C6
:10BE800026EA050503FA04F42C43C4600AE00669B7
:10BE900001EB41040725A54026EA050503FA04F451
:10BEA0002C430461836B0232C3F30154121BD2B2E0
:10BEB00002EB82021F24944023EA040391401943B9
:10BEC000816370BD836B013923F4401343EA01534E
:10BED0008363704782B0002301930190019B194452
:10BEE0000191019B1A6002B07047836823F47023AC
:10BEF000194381607047836823F4401319438160BC
:10BF00007047836843F48003836070478068C0F3A0
:10BF100080507047436811B143F4806301E023F41B
:10BF2000806343607047436811B143F4805301E07C
:10BF300023F480534360704782B000230193019043
:10BF4000019B283319440191019B186880B202B00B
:10BF500070470123C9B203FA01F143680AB11943DA
:10BF600001E023EA0101416070470368194214BFF0
:10BF7000012000207047C943016070474268006893
:10BF800010EA112007D00123C9B203FA01F11142CE
:10BF900014BF1846002070476FEA112101607047F6
:10BFA000374AD2F8883043F47003C2F88830354BF2
:10BFB0001A68002142F001021A6099601A6822F0A2
:10BFC000847222F480321A602F4A5A601A6882B052
:10BFD00022F480221A60D960009101911A6842F41B
:10BFE00080321A601A6802F400320192009A01321B
:10BFF0000092019A1AB9009AB2F5A04FF2D1214BE2
:10C000001B6813F4003318BF01230193019B012B1C
:10C0100005D01B4B4FF000629A6002B07047194B7D
:10C020001A491A6C42F080521A640A6842F440427B
:10C030000A609A689A609A6842F400429A609A6824
:10C0400042F4A0529A60124A5A601A6842F0807212
:10C050001A6019680B4A8901FBD50E4B40F2057135
:10C060001960936823F003039360936843F002031D
:10C070009360936803F00C03082BFAD1C9E700BF63
:10C0800000ED00E000380240103000240070004055
:10C0900008544007003C0240174A1849936803F0CF
:10C0A0000C03042B03D0082B03D0154B18E0154BC1
:10C0B00016E05068536810F4800F03F03F03506897
:10C0C00014BF104A0E4AB2FBF3F30B4A5268C2F394
:10C0D0000142C0F38810013243435200B3FBF2F334
:10C0E0000B60054B084A9B68C3F30313D25C0B68D3
:10C0F000D3400B60704700BF003802402C06002080
:10C100000024F40000127A001C06002038B5044612
:10C110000D46AC4203D254F8043B9847F9E738BDCA
:10C12000FEE7000008B5104A104B11498B4204D2BB
:10C1300052F8040F43F8040BF8E7124812494FF085
:10C1400000028842B8BF40F8042BFADBFFF728FF53
:10C1500008490948FFF7DAFF08490948FFF7D6FF01
:10C16000BDE80840F8F72ABB806C040800000020F6
:10C17000980600206C6C04086C6C0408746C04084D
:10C180006C6C0408A006002090BD00202DE9F0038F
:10C190005FEA92098446884619D000F108040B46EC
:10C1A0004F4614E90300060C0D0C360400042D0460
:10C1B0000904013F83E84100DD60996004F108044F
:10C1C00003F11003EDD10CEBC90C08EB091812F0C8
:10C1D000030207D03CF9023B013A4FEA034348F817
:10C1E000043BF7D1BDE8F003704700BF2DE9F00F25
:10C1F000A0B00E901A910E99408889681B910E9CF0
:10C200001B9E1D9000F10041013903F0010064689C
:10C21000119406EB41015B08149219911E901F9333
:10C2200000F0E2800C461D991D9B30461A9E89083D
:10C23000CA0004360C9103F00303043402301F9942
:10C240001C920F93169417960D9018913246169CD7
:10C2500032F8043C24F8043C32F8023C0E9E24F8E8
:10C26000023C36781596002E00F0A6810D9A1C9996
:10C27000149C08941144B146701C0126139112902D
:10C280000996CDF81C9049463246881A119C0D9E9D
:10C290000C9A36F8021C04EB4000002A78D0079B69
:10C2A00010901446DB004FF0000A4FF0000B019491
:10C2B000079C0693D046D9463246034615881E8809
:10C2C00033F81400B2F802C033F82470C6FB85AB13
:10C2D000C1FB86894FF0060616FB0431C5FB808939
:10C2E00096880D88D188C0FB8CABCCFB8789C7FBB7
:10C2F00086ABC6FB8589019E0698013E0344C5FBBB
:10C3000081AB02F108020196D8D103460C9A10982D
:10C31000139D03FB02000F9C74B1079A234656003D
:10C3200000E0A1B2028835F8024B013B3044C2FB69
:10C3300084ABC1FB8289F4D14FEAD83343EA494444
:10C340000899029420464FEAE9364FEADA320E9C09
:10C3500000F30F0303960B8042EA4B4609982378BB
:10C3600004964FEAEB3134460591089E129904F386
:10C370000F02013026F81320884206F102060990C8
:10C3800008960DD00E9A127807921146099A7CE70A
:10C390004FF0000A4FF0000B3546D046D946BAE7B9
:10C3A000149C159B0E9E04EB430433781494204692
:10C3B00000EB43001699179A0D9B189C14900431BA
:10C3C00004320433013C169117920D9318947FF4B4
:10C3D0003EAF1F9E19981A991B9CB300184419442C
:10C3E0001C4419901A911B941E9E002E00F0A080F0
:10C3F0001D981D9A1B9C10968008C10002F0030234
:10C4000002901291079209941A9E199836F8023BED
:10C4100020F8023B0E991A96097819900F9100297D
:10C4200079D0129B099C149E04964A1C0120234437
:10C430000C920D938A4606900246119C029EC2EB16
:10C440000A0104EB4101002E00F0B0804FF0020021
:10C450001AFB00F04FEA400C04466444099A01902C
:10C460004FEA800B0B4630464FF000084FF00009B2
:10C47000089127461D88168833F81A105488C6FB81
:10C4800085893CF803509688C4FB8189D95BD488A0
:10C49000C6FB858901385B44C4FB818902F108022F
:10C4A000E8D1019B0899029C4FF0020212FB0A3B63
:10C4B00012FB0ABB12FB0ABB0D9A04FB0B11079E71
:10C4C00056B14FEA4A0A3346088832F8024B013B1C
:10C4D0005144C4FB8089F7D14FEAD830069A049EB4
:10C4E00040EA49414FEAE9330C980B9301320C467C
:10C4F00004F30F0326F8023B82420A910692049647
:10C5000004D00E9C069A94F800A096E714980F9E0B
:10C5100000EB460014900999109A0231013A0991F2
:10C5200010927FF471AF1B9C1E9E04EB46041B947B
:10C530001D980E9C471EBD08A06829D01B9E00F1C7
:10C54000080206F10803964238BF984234BF002122
:10C550000121022D94BF002101F0010179B346EAC7
:10C56000000189072BD10021013153F8086C53F8E1
:10C57000044C42F8044CA94242F8086C03F1080349
:10C5800002F10802F0D11B99ED00294428441B91C7
:10C5900017F0030706D01B9B33F8022B20F8022B61
:10C5A000013FF9D120B0BDE8F00F7047099A4FF074
:10C5B00000084FF0000982E733461498F8E61B9B09
:10C5C000024629461C8814805C8854809C8894808C
:10C5D000DC88D480013903F1080302F10802F1D1AB
:10C5E000D1E700BF2DE9F00F92B00F9010930F9B91
:10C5F00000885B680A930E9000F100430F9C0A9D2F
:10C600001098A4680994013B05EB43038008079147
:10C6100008920693119000F0A9808B460E99029023
:10C620008908CA009A4614440E9B0D94089C0491F4
:10C6300003F003030B93083453460835DA460C9293
:10C64000019400959B46BAF80030ABF80030BAF878
:10C650000230ABF80230BAF80430ABF80430BAF864
:10C66000063000980499ABF8063010E90C00002958
:10C6700000F0FA8000F10804099803940E460021A6
:10C680002546CDF814A089460F468C4600F10804D3
:10C69000B24654F8086C22FB06CC23FB0699C3EA89
:10C6A000020855F8082C28FB1677C2EA030828FB75
:10C6B000161654F8040C23FB00CC55F8043C22FB5E
:10C6C000009928FB1077C3EA020121FB1061BAF13F
:10C6D000010A05F1080504F10804DAD1009C0C9860
:10C6E000DDF814A020440D9C0B9D6DB1246822FB45
:10C6F00004CC23FB0499C3EA020222FB14770268EC
:10C70000C2EA030323FB14110198029B039A0092CF
:10C710004FEAEC3CFF130CF30F0C07F30F074FEA43
:10C72000E939CCEA074709F30F0940F8087CC91337
:10C73000083001F30F01013BC9EA014140F80C1C2C
:10C740000AF1080A0BF1080B019002937FF47BAF0A
:10C75000119C069D07980899E3000A9C1D44184403
:10C7600019441C440695079008910A94109D15F0F1
:10C770000305009539D009980E9B0A9C00F1040B23
:10C780004FEA530AA8464FF0000C04F10409079D34
:10C79000069835F80C3020F80C305A4609EB0C039B
:10C7A0005146002033F8047C32F8046C33F8025C04
:10C7B00032F8024C17FB0600013903F1040315FBA4
:10C7C000040002F10402EDD10899B8F101084FEA22
:10C7D000E03000F30F0021F80C000CF1020CD6D170
:10C7E0000A9B009C03EB44030A930E9D0F986F1E57
:10C7F000BE0845682AD00A9B0A9C03F1080205F18D
:10C8000008039C4238BF954234BF00210121022E0B
:10C8100094BF002101F0010171B344EA05018907C9
:10C820002AD10021013152F8084C52F8040C43F887
:10C83000040CB14243F8084C02F1080203F108036A
:10C84000F0D10A98F600304435440A9017F00303FB
:10C8500006D00A9A32F8021B25F8021B013BF9D1D7
:10C8600012B0BDE8F00F704700F10805099C039570
:10C8700089460F468C4637E70A9A2B463146108880
:10C8800018805088588090889880D088D880013946
:10C8900002F1080203F10803F1D1D2E72DE9F00F0C
:10C8A0001C469EB0037B4568066880681290A70806
:10C8B0003801C3F11F0C1792024413910133CCF1DC
:10C8C000200104F003041D9205F110021B90119544
:10C8D000159616971C9310911A941492E2461046DE
:10C8E000129B50F8104C5D689E68DF68D3F800809A
:10C8F00004950596D3F810B0119D119B169E0697CE
:10C90000D5F80C905F689B68002E00F0DB80304605
:10C91000A446139E179D09904C46D146C246DDF8A9
:10C9200070803168049A079181FB0A01C2FB0C01F7
:10C93000059AC2FB0701069FC7FB0301CBFB04015D
:10C9400020FA09F001FA08F404432C607068049F8F
:10C95000089000220392079A029180FB0A01C7FB0C
:10C960000201059A069FC2FB0C01C7FB0401CBFB29
:10C9700003010A9120FA09F001FA08F108436860FE
:10C98000B76801900499089800220B9287FB0A234C
:10C99000C1FB002307980599C1FB00230198069964
:10C9A000C1FB0023CBFB042322FA09F203FA08F4AB
:10C9B0001443AC60D6F80CC00C9300200D90049882
:10C9C00008998CFB0A23C0FB07230598C0FB0123B1
:10C9D00006990198C1FB0423CBFB002300210E9391
:10C9E0000F91099922FA09F203FA08F31343013966
:10C9F000EB6006F1100605F11005099191D1139A2B
:10CA00001B9D1D9E2A44D0461392CA46A1466446E9
:10CA10001A98002851D0CDF81C80CDF820B0099785
:10CA2000984601968446DDF84CB003E0C14609946F
:10CA300090462C465BF8045B079E049F85FB06012D
:10CA4000C7FB0401099E059FC7FB0601069E109FB8
:10CA5000C6FB0801089EC6FB090101FA07F920FA86
:10CA60000AF2BAF1200742EA090258BF41FA07F771
:10CA7000019858BF3A4340F8042BBCF1010C41FA2D
:10CA80000AF301901146D1D1CDE918234346149AF7
:10CA9000119E42F8105C159F129D7460B160F360A6
:10CAA000143510321036013F1295149211961597D5
:10CAB0000AD017981390149812E7194625464B464A
:10CAC0003C46E4E7179EA3E71EB0BDE8F00F7047B1
:10CAD000F0B40C49860DC0F3150051F82640400211
:10CAE000C0F100470136A7FB0423E51707FB053714
:10CAF00051F826103B460022C1FB00235800F0BC31
:10CB0000704700BF30B8020800F002B800F02AB841
:10CB100010B5002814BF04460124204600F082F816
:10CB200030B900F017F808B900F01EF88047F4E7B4
:10CB300010BD0000064BBFF35F8F024653E8000FA5
:10CB400043E800210029F9D1BFF35F8F704700BF90
:10CB500088BD0020024B1868BFF35F8F704700BF8D
:10CB600088BD002000F066B808B5062000F08CFAF9
:10CB7000012000F02FFC00BF002301461A46184692
:10CB800000F0B6BA08B5074B044613B1002100F017
:10CB900017FB054B1868836A03B19847204600F0DD
:10CBA00019FC00BFC1D100084C6C040838B5074D12
:10CBB000074C2C1BA41005D0013C55F8043D9847A8
:10CBC000002CF9D1BDE838403AF04AB8786C040836
:10CBD000746C040870B50F4E0F4D761BB61018BF5D
:10CBE000002405D0013455F8043B9847A642F9D1FA
:10CBF0000A4E0B4D761B3AF02DF8B61018BF0024E4
:10CC000006D0013455F8043B9847A642F9D170BDCF
:10CC100070BD00BF6C6C04086C6C0408746C040874
:10CC20006C6C0408024B0146186800F039B900BF6B
:10CC300030060020024B0146186800F0EBB800BF38
:10CC400030060020844641EA000313F003036DD14F
:10CC5000403A41D351F8043B40F8043B51F8043BBF
:10CC600040F8043B51F8043B40F8043B51F8043BC6
:10CC700040F8043B51F8043B40F8043B51F8043BB6
:10CC800040F8043B51F8043B40F8043B51F8043BA6
:10CC900040F8043B51F8043B40F8043B51F8043B96
:10CCA00040F8043B51F8043B40F8043B51F8043B86
:10CCB00040F8043B51F8043B40F8043B51F8043B76
:10CCC00040F8043B51F8043B40F8043B51F8043B66
:10CCD00040F8043B403ABDD2303211D351F8043B06
:10CCE00040F8043B51F8043B40F8043B51F8043B46
:10CCF00040F8043B51F8043B40F8043B103AEDD2B5
:10CD00000C3205D351F8043B40F8043B043AF9D205
:10CD1000043208D0D2071CBF11F8013B00F8013BD8
:10CD200001D30B8803806046704700BF082A13D3E5
:10CD30008B078DD010F003038AD0C3F10403D21AFD
:10CD4000DB071CBF11F8013B00F8013B80D331F831
:10CD5000023B20F8023B7BE7043AD9D3013A11F8B1
:10CD6000013B00F8013BF9D20B7803704B7843701C
:10CD70008B7883706046704770B4840746D0541E29
:10CD8000002A41D0CDB2034602E0621EE4B314464D
:10CD900003F8015B9A07F8D1032C2ED9CDB245EAEE
:10CDA00005250F2C45EA054519D903F11002264641
:10CDB000103E0F2E42F8105C42F80C5C42F8085C02
:10CDC00042F8045C02F11002F2D8A4F1100222F041
:10CDD0000F0204F00F041032032C13440DD91E4629
:10CDE0002246043A032A46F8045BFAD8221F22F0AE
:10CDF00003020432134404F003042CB1C9B21C44EE
:10CE000003F8011BA342FBD170BC704714460346D4
:10CE1000C2E700BF30B481B151F8043C0439002BA3
:10CE2000B8BFC9181D4B1A682AB18A420AD90868C6
:10CE30000C18A24225D04A60196030BC70478B4262
:10CE400003D81A465368002BF9D1146815198D427E
:10CE50000CD007D808680C189C4218D04B6030BC26
:10CE6000516070470C23036030BC704709680C4464
:10CE7000111999421460E0D10ACB0C44536014603C
:10CE8000DBE7146852684A6020440860D4E71C68F5
:10CE90005B684B60204408605160CEE7BC06002010
:10CEA00070B5CD1C25F0030508350C2D38BF0C25B9
:10CEB000002D06463BDBA94239D827490A6852B102
:10CEC00013685B1B04D436E023685B1B1AD522462B
:10CED0005468002CF8D149681F4C002936D02946E7
:10CEE000304600F03BF8431C21D0C41C24F003045E
:10CEF000A04205D0211A304600F030F8013016D09B
:10CF0000256004E00B2B0DD923601C44256004F13F
:10CF10000B0020F00700231DC31A02D05A42E25032
:10CF200070BD70BD94420ED063685360EFE70C2370
:10CF30003360002070BD0B2B03D8536814460B6080
:10CF4000E5E71446E0E713461446F8E7304600F0FC
:10CF500005F86060C3E700BFBC06002038B5074C89
:10CF6000002305460846236000F026FA431C00D043
:10CF700038BD2368002BFBD02B6038BD8CBD002052
:10CF800038B5446C0CB1002038BD80210546FFF750
:10CF900087FF686448B12346224600E0686CC250AF
:10CFA0000433802BFAD1002038BD4FF0FF3038BD5C
:10CFB0001F29F8B509D8446C074616460D464CB1F2
:10CFC00054F8250044F82560F8BD162202604FF0A1
:10CFD000FF30F8BDFFF7D4FF08B97C6CF0E74FF0E5
:10CFE000FF30F8BD1F2938B521D8426C05460C46E4
:10CFF0009AB152F8213083B1012B0CD0591C06D0C4
:10D000000025204642F824509847284638BD16236C
:10D010000360012038BD002038BD284600F066F8C6
:10D02000224601462846BDE8384000F04BB816239A
:10D0300003604FF0FF3038BD1F291ED838B5436C50
:10D0400005460C46A3B153F8242003EB84036AB1D0
:10D05000511C09D0012A05D0002520461D609047AB
:10D06000284638BD032038BD022038BD012038BD18
:10D07000FFF786FF20B96B6CE5E74FF0FF30704794
:10D080004FF0FF3038BD00BF024B01461868FFF774
:10D09000A9BF00BF30060020024B0A4601461868AF
:10D0A000FFF786BF30060020014B1868FFF768BF06
:10D0B00030060020024B01461868FFF7BDBF00BFD5
:10D0C0003006002038B50B46074C05461146184679
:10D0D0000023236000F068F9431C00D038BD2368AA
:10D0E000002BFBD02B6038BD8CBD002000F054B964
:10D0F0002DE9F0472E4E34680746884691469A46F9
:10D10000002C37D065681F2D13DD2A4B002B4AD029
:10D110008C20FFF787FD0446002844D03368036065
:10D12000002330604360C0F8883077BB3D46012360
:10D1300013E08FB1D4F8880028B3D0F8001140F87C
:10D1400025900126AE4000EB85033143022FC0F845
:10D150000011C3F880A007D06B1C0235636000206B
:10D1600044F82580BDE8F087D0F804311E43C0F8AC
:10D170000461F1E7104B114C3460002BC2D01B68E6
:10D18000C4F88830BEE70B4B6BB14FF48470FFF7E7
:10D1900049FD40B100216568C0F80011C0F80411D4
:10D1A000C4F88800CBE74FF0FF30BDE8F08700BF40
:10D1B0005007002025CC000800000000C406002015
:10D1C0002DE9F04F83B00F460190394BD3F8009012
:10D1D000B9F1000F32D09B46D9F80450D9F88880B5
:10D1E0006C1E11D4AD002E1D4E4445444FB3B8F112
:10D1F000000F02D0EB6F9F4223D0013C631CA5F1CE
:10D200000405A6F10406F1D12A4BBBB1D9F80430CC
:10D21000002B44D1D9F80030002B42D0CBF800309D
:10D22000B8F1000F02D04046FFF704FD4846FFF773
:10D2300001FDDBF80090B9F1000FCDD103B0BDE8DE
:10D24000F08FD9F804303268013BA34216BF0023A7
:10D25000C9F804403360002ACFD0D9F804A0B8F14F
:10D26000000F16D0D8F800110123A3400B4210D0B4
:10D27000D8F804110B420ED155F8041C01989047C0
:10D28000D9F804309A45A0D1DBF800304B45B4D032
:10D290009BE79047F4E755F8040C9047F0E7D9F87E
:10D2A0000030CB469946B9F1000F95D1C6E700BFD3
:10D2B0005007002035CC000838B50C4609680546F3
:10D2C00009B1FFF7F9FF21462846BDE83840FFF7CE
:10D2D000A1BD00BF2F4B1B68834259D0426A70B575
:10D2E0000546002A50D0D3689BB10026995941B118
:10D2F0000C682846FFF78EFD2146002CF8D16B6A9A
:10D30000DB680436802EF1D119462846FFF782FDEE
:10D310006A6A116811B12846FFF77CFD696911B18D
:10D320002846FFF777FD696A11B12846FFF772FDBD
:10D33000A96B11B12846FFF76DFDE96B11B12846C5
:10D34000FFF768FD296C11B12846FFF763FDE96D11
:10D3500011B12846FFF75EFDA96D11B12846FFF710
:10D3600059FD696B11B12846FFF754FDAB6903B94C
:10D3700070BDAB6A28469847A96C0029F8D02846AA
:10D38000BDE87040FFF798BF41690029C8D1CFE7D9
:10D39000704700BF30060020024B58221A604FF041
:10D3A000FF3070478CBD0020024B58221A604FF0AE
:10D3B000FF3070478CBD0020044A05491368002BDC
:10D3C00008BF0B46184410601846704754070020E9
:10D3D00090BD0020FEE700BF63EA00766C76C45281
:10D3E000C878092DB87927579B31BC3EEA45C33030
:10D3F000491793AE8B6DA4A5ADA2F135B53C1E4384
:10D40000544353532056616C7565202F2054687225
:10D410006573686F6C64202F2056616C696400002E
:10D42000430000000000000092F5FA7F00000000B9
:10D430004500000000000000749BFA7F000000001F
:10D440004700000000000000EC31FA7F00000000FF
:10D450004A00000000000000C9C8F97F0000000079
:10D460004D00000000000000A257F97F00000000FE
:10D470004F0000000000000003DEF87F0000000005
:10D480005200000000000000775BF87F0000000001
:10D49000550000000000000081CFF77F0000000071
:10D4A00058000000000000008B34F77F00000000EF
:10D4B0005B000000000000005299F67F00000000B1
:10D4C0005E000000000000009AE8F57F0000000008
:10D4D0006100000000000000F658F57F0000000029
:10D4E00064000000000000006FC5F47F0000000031
:10D4F0006700000000000000B5F8F37F00000000A6
:10D500006B00000000000000A018F37F0000000086
:10D510006E00000000000000AC30F27F0000000050
:10D520007200000000000000AB33F17F000000003B
:10D5300076000000000000001827F07F00000000C7
:10D540007B000000000000003303EF7F00000000BC
:10D550007F00000000000000D9CDED7F000000003A
:10D560008300000000000000BC7EEC7F0000000093
:10D5700088000000000000004D14EB7F0000000058
:10D580008D000000000000000F95E97F0000000002
:10D5900092000000000000002D00E87F0000000065
:10D5A00097000000000000006B43E67F00000000D1
:10D5B0009C000000000000001F6EE47F00000000DF
:10D5C0009F000000000000002654E37F00000000E0
:10D5D000A2000000000000000E76E27F00000000C4
:10D5E000A500000000000000463FE17F00000000B1
:10D5F000A7000000000000005359E07F0000000079
:10D60000AB00000000000000E50DDF7F000000001F
:10D61000AD00000000000000F615DE7F00000000F5
:10D62000B100000000000000D3B4DC7F0000000067
:10D63000B300000000000000F1A9DB7F0000000043
:10D64000B7000000000000000032DA7F0000000098
:10D65000BA000000000000002813D97F000000007D
:10D66000BD000000000000004883D77F00000000DC
:10D67000C0000000000000005E44D67F00000000F3
:10D68000C4000000000000002C9BD47F00000000BC
:10D69000C7000000000000001A51D37F0000000006
:10D6A000CB00000000000000E981D17F00000000F5
:10D6B000CE000000000000007D20D07F00000000B0
:10D6C000D2000000000000000429CE7F000000000E
:10D6D000DA000000000000004F99CA7F000000003F
:10D6E000E1000000000000003ED0C67F0000000006
:10D6F000E500000000000000FB13C57F00000000F3
:10D70000E900000000000000C9BDC27F0000000069
:10D71000F100000000000000DB5DBE7F00000000A3
:10D72000FA000000000000003BACB97F00000000E0
:10D73000FE00000000000000A185B77F000000008F
:10D740005CF95CF95CF95CF95CF95CF95CF95CF931
:10D750005CF95CF95CF95CF95CF95CF95CF95CF921
:10D760005CF95CF95CF95CF9A406A406A406A406BD
:10D77000A406A406A406A406A406A406A406A40659
:10D78000A406A406A406A406A406A406A406A40649
:10D7900043006601337A5B0045005A011C9E5E001F
:10D7A00047004E01E02A62004A004301B094650040
:10D7B0004D003801742169004F002D012CD16C00FF
:10D7C00052002301D8A37000550019017799740005
:10D7D00058000F01FED478005B00060192ED7C003A
:10D7E0005E00FD00016F81006100F600C5FB840052
:10D7F0006400F000898888006700E800E04F8D0031
:10D800006B00E0001E5D92006E00D8005D6A97001C
:10D810007200D10083BD9C007600CA009D33A20037
:10D820007B00C3009EEFA7007F00BD0094CEAD003B
:10D830008300B60071F3B3008800B000365EBA0012
:10D840008D00AA00EEEBC0009200A4009B9CC700D4
:10D8500097009F0023B6CE009C0099009FF2D50050
:10D860009F009600262EDA00A20094000375DD00CA
:10D87000A500910072F6E100A7008F004E3DE50083
:10D88000AB008C00B1E1E900AD008A00814BED00F6
:10D89000B1008700D812F200B30085009C9FF5000C
:10D8A000B7008300E789FA00BA0081009E39FE00C4
:10D8B000BD007E00DD460301C0007C007C3C07010A
:10D8C000C4007A00AF6C0C01C70078004E621001F2
:10D8D000CB00760068D81501CE007400FCF0190169
:10D8E000D2007200FDAC1F01DA006E007AC7290178
:10D8F000E1006A00DF273401E500690041CC38010E
:10D90000E90067001FF13E01F10063003A234A017C
:10D91000FA00600031BE5501FE005E0064EE5A015F
:10D9200041000000000000B80800000042000000B4
:10D93000000080EA0C000000430000000000A0EBA3
:10D940000E00000044000000000000EA0A00000091
:10D9500045000000000000800400000046000000B8
:10D96000000080AE0C00000047000000000080EEC8
:10D970000C00000048000000000000AA0A0000009F
:10D9800049000000000000A0060000004A0000005E
:10D990000000B8BB100000004B000000000080EB4E
:10D9A0000C0000004C000000000080BA0C000000D9
:10D9B0004D000000000000EE0A0000004E000000D4
:10D9C000000000E8080000004F0000000000E0EE4A
:10D9D0000E000000500000000000A0BB0E00000080
:10D9E000510000000000B8EE1000000052000000DE
:10D9F000000000BA0A00000053000000000000A868
:10DA00000800000054000000000000E006000000D4
:10DA100055000000000000AE0A00000056000000A3
:10DA2000000080AB0C00000057000000000080BB2D
:10DA30000C000000580000000000E0EA0E000000AA
:10DA4000590000000000B8EB100000005A00000070
:10DA50000000A0EE0E000000310000000080BBBB03
:10DA600014000000320000000000EEAE12000000C2
:10DA7000330000000000B8AB1000000034000000CC
:10DA80000000E0AA0E00000035000000000080AA9F
:10DA90000C000000360000000000A0EA0E000000AC
:10DAA000370000000000A8EE100000003800000061
:10DAB0000000EAEE12000000390000000080EEEEE7
:10DAC000140000003000000000E0EEEE1600000040
:10DAD0002F0000000000E8EA100000003F000000F6
:10DAE0000000EAAE120000002C00000000E0AEEEE4
:10DAF000160000002D0000000000AEEA1200000039
:10DB00003D0000000000B8EA100000002E000000F8
:10DB10000080EBBA140000002000000000000000AC
:10DB200004000000000000000000000000000000F1
:10DB300080402010080402014D6F646520736574F5
:10DB400020746F20444D52004D6F646520736574DE
:10DB500020746F20442D53746172004D6F646520F2
:10DB600073657420746F2053797374656D204675E6
:10DB700073696F6E004D6F64652073657420746FF8
:10DB800020503235004D6F64652073657420746FCA
:10DB9000204E58444E004D6F6465207365742074A8
:10DBA0006F20504F43534147004D6F6465207365AC
:10DBB0007420746F20464D004D6F6465207365744A
:10DBC00020746F20442D537461722043616C69622C
:10DBD00072617465004D6F64652073657420746FA5
:10DBE00020444D522043616C696272617465004D3E
:10DBF0006F64652073657420746F205253534920FD
:10DC000043616C696272617465004D6F6465207375
:10DC1000657420746F20383020487A2043616C6925
:10DC20006272617465004D6F646520736574207461
:10DC30006F20464D2031304B687A2043616C696219
:10DC400072617465004D6F64652073657420746F34
:10DC500020464D2031322E354B687A2043616C6965
:10DC60006272617465004D6F646520736574207421
:10DC70006F20464D2031354B687A2043616C6962D4
:10DC800072617465004D6F64652073657420746FF4
:10DC900020464D2032304B687A2043616C696272B5
:10DCA000617465004D6F64652073657420746F2026
:10DCB000464D2033304B687A2043616C6962726153
:10DCC0007465004D6F64652073657420746F205017
:10DCD0003235203130313120487A2043616C69621D
:10DCE00072617465004D6F64652073657420746F94
:10DCF00020444D52204D53203130333120487A207A
:10DD000043616C696272617465004D6F6465207374
:10DD1000657420746F204E58444E203130333120CA
:10DD2000487A2043616C696272617465004D6F646A
:10DD3000652073657420746F20504F435341472012
:10DD400043616C696272617465004D6F6465207334
:10DD5000657420746F2049646C6500526563656961
:10DD600076656420696E76616C696420464D20702A
:10DD70006172616D73203100526563656976656417
:10DD800020696E76616C696420464D207061726115
:10DD90006D73203200526563656976656420696E33
:10DDA00076616C696420464D20706172616D7320EC
:10DDB0003300526563656976656420696E76616CCF
:10DDC00069642063616C6962726174696F6E20645A
:10DDD00061746100496E76616C6964204357204923
:10DDE00064206461746100526563656976656420CE
:10DDF000696E76616C696420442D53746172206889
:10DE00006561646572005265636569766564206961
:10DE10006E76616C696420442D5374617220646174
:10DE2000746100526563656976656420696E766128
:10DE30006C696420442D5374617220454F54005224
:10DE40006563656976656420696E76616C696420D6
:10DE5000444D522064617461005265636569766562
:10DE60006420696E76616C696420444D522073743D
:10DE700061727400526563656976656420696E76C7
:10DE8000616C696420444D522053686F7274204C59
:10DE90004300526563656976656420696E76616CDE
:10DEA000696420444D522041626F72740052656370
:10DEB000656976656420696E76616C696420537962
:10DEC0007374656D20467573696F6E20646174614B
:10DED00000526563656976656420696E76616C6978
:10DEE0006420503235206865616465720052656354
:10DEF000656976656420696E76616C69642050326C
:10DF000035204C4455005265636569766564206927
:10DF10006E76616C6964204E58444E206461746171
:10DF200000526563656976656420696E76616C6927
:10DF30006420504F435341472064617461004D4D4C
:10DF400044564D2032303230303731342028442D81
:10DF5000537461722F444D522F53797374656D2041
:10DF6000467573696F6E2F5032352F4E58444E2FC1
:10DF7000504F435341472F464D292031322E3030E8
:10DF80003030204D487A2047697449442023613657
:10DF900030656362330000000000000000400000B4
:10DFA000DA6E0000FF7F0000DA6E00000040000023
:10DFB0000000000001C0FFFF2791FFFF0180FFFF6D
:10DFC0002791FFFF01C0FFFF00CDF59D5D7CFA0AA0
:10DFD0006E8A2356E84CAADE8B26E4F28288C68A33
:10DFE0007429A4ECD00822CEA2FC018CECDA0AA0A1
:10DFF000EE8A7E2B26CCF88A0800CDF59D5D7C6DDF
:10E00000BB0EB3A426A84CAADE8B26E4F28288C6F7
:10E010008A7429A4ECD00822CEA2FC018CECDA0A86
:10E02000A0EE8A7E2B26CCF88A0800CDF59D5D7681
:10E030003A1B4A81A8E2804CAADE8B26E4F2828851
:10E04000C68A7429A4ECD00822CEA2FC018CECDA9A
:10E050000AA0EE8A7E2B26CCF88A0800CDF59D5DBD
:10E0600074288302B02D07E24CAADE8B26E4F282EC
:10E0700088C68A7429A4ECD00822CEA2FC018CECBC
:10E08000DA0AA0EE8A7E2B26CCF88A0853656E64E5
:10E090002063616C6C7369676E00537461746520F2
:10E0A000746F2052454C4159494E47005374617476
:10E0B0006520746F204C495354454E494E470053D8
:10E0C0007461746520746F2052454C4159494E4724
:10E0D0005F5741495400537461746520746F205434
:10E0E000494D454F55540053656E642061636B0084
:10E0F000537461746520746F2048414E4700537417
:10E1000061746520746F2054494D454F55545F57D5
:10E110004149540053746F702061636B0053746104
:10E12000746520746F204B45524348554E4B004355
:10E1300068616E676520746F2053544154455F4693
:10E140004D004368616E676520746F2053544154DD
:10E15000455F49444C4500000000620D9D1A8E2722
:10E16000103400403D4BA6551F5F8E67DA6EEF748A
:10E17000BC79347D4C7FFF7F4C7F347DBC79EF745C
:10E18000DA6E8E671F5FA6553D4B004010348E2718
:10E190009D1A610D00009FF263E572D8F0CB00C0BC
:10E1A000C3B45AAAE1A072982691118B4486CC82FE
:10E1B000B4800080B480CC824486118B2691729802
:10E1C000E1A05AAAC3B400C0F0CB72D863E59FF2B5
:10E1D0000004040007040B000E04120015041900CB
:10E1E0001C042000230427002A042D0731023405D3
:10E1F00038003B033E064201450448074C024F05E8
:10E200000005040107050B010E0512011505190192
:10E210001C052001230527012A052E0031033406A1
:10E2200038013B043E074202450549004C034F06B6
:10E230000006040207060B020E061202150619025A
:10E240001C062002230627022A062E013104340769
:10E2500038023B053F004203450649014C044F0785
:10E260000007040307070B030E0712031507190322
:10E270001C072003230727032A072E023105350038
:10E2800038033B063F014204450749024C05500054
:10E290000100040408000B040F0012041600190406
:10E2A0001D002004240027042B002E033106350115
:10E2B00038043B073F024205460049034C06500123
:10E2C0000101040508010B050F01120516011905CE
:10E2D0001D012005240127052B012E0431073502DD
:10E2E00038053C003F034206460149044C075002F2
:10E2F0000102040608020B060F0212061602190696
:10E300001D022006240227062B022E0532003503AB
:10E3100038063C013F044207460249054D005003C0
:10E320000103040708030B070F031207160319075D
:10E330001D032007240327072B032E063201350473
:10E3400038073C023F054300460349064D0150048F
:10E350000104050008040C000F04130016041A0041
:10E360001D042100240428002B042E073202350549
:10E3700039003C033F064301460449074D0250055E
:10E380000105050108050C010F05130116051A0109
:10E390001D052101240528012B052F003203350618
:10E3A00039013C043F07430246054A004D0350062D
:10E3B0000106050208060C020F06130216061A02D1
:10E3C0001D062102240628022B062F0132043507E0
:10E3D00039023C054000430346064A014D045007FC
:10E3E0000107050308070C030F07130316071A0399
:10E3F0001D072103240728032B072F0232053600AF
:10E4000039033C064001430446074A024D055100CA
:10E410000200050409000C041000130417001A047C
:10E420001E002104250028042C002F03320636018B
:10E4300039043C074002430547004A034D06510199
:10E440000201050509010C051001130517011A0544
:10E450001E012105250128052C012F043207360253
:10E4600039053D004003430647014A044D07510268
:10E470000202050609020C061002130617021A060C
:10E480001E022106250228062C022F053300360322
:10E4900039063D014004430747024A054E00510337
:10E4A0000203050709030C071003130717031A07D4
:10E4B0001E032107250328072C032F0633013604EA
:10E4C00039073D024005440047034A064E01510406
:10E4D0000204060009040D001004140017041B00B8
:10E4E0001E042200250429002C042F0733023605C0
:10E4F0003A003D034006440147044A074E025105D5
:10E500000205060109050D011005140117051B017F
:10E510001E052201250529012C053000330336068E
:10E520003A013D044007440247054B004E035106A3
:10E530000206060209060D021006140217061B0247
:10E540001E062202250629022C0630013304360756
:10E550003A023D054100440347064B014E04510772
:10E560000207060309070D031007140317071B030F
:10E570001E072203250729032C0730023305370025
:10E580003A033D064101440447074B024E05520041
:10E59000030006040A000D041100140418001B04F3
:10E5A0001F002204260029042D0030033306370102
:10E5B0003A043D074102440548004B034E06520110
:10E5C000030106050A010D051101140518011B05BB
:10E5D0001F012205260129052D01300433073702CA
:10E5E0003A053E004103440648014B044E075202DF
:10E5F000030206060A020D061102140618021B0683
:10E600001F022206260229062D0230053400370398
:10E610003A063E014104440748024B054F005203AD
:10E62000030306070A030D071103140718031B074A
:10E630001F032207260329072D0330063401370460
:10E640003A073E024105450048034B064F0152047C
:10E65000030407000A040E001104150018041C002E
:10E660001F04230026042A002D0430073402370536
:10E670003B003E034106450148044B074F0252054B
:10E68000030507010A050E011105150118051C01F6
:10E690001F05230126052A012D0531003403370605
:10E6A0003B013E044107450248054C004F0352061A
:10E6B000030607020A060E021106150218061C02BE
:10E6C0001F06230226062A022D06310134043707CD
:10E6D0003B023E054200450348064C014F045207E9
:10E6E000030707030A070E031107150318071C0386
:10E6F0001F07230326072A03445374617254583AB0
:10E70000206865616465722073706163652061765D
:10E7100061696C61626C6500445374617254583A6B
:10E720002064617461207370616365206176616942
:10E730006C61626C6500445374617254583A2045B0
:10E740004F5420737061636520617661696C61620A
:10E750006C6500804020100804020155555555C8CD
:10E760007A00000000000000F734094446D706B3E1
:10E7700072DE42F5A5D8F1877B9A0422A36B8359F8
:10E78000396FA1FA52ECF8C33D4D0291D1B5C1AC3D
:10E790009CB7507D2976FCE19E2681C8E8DA605658
:10E7A000CE5BA8BE143BFE704F934064746D302B5B
:10E7B000E72D545F8A1D7FB8A7492032BA36989555
:10E7C000F3060FFFFFFFFFFFF00D5D7F77FD757014
:10E7D000444D5249646C6552583A2064617461201A
:10E7E00073796E6320666F756E642063656E7472F4
:10E7F000652F7468726573686F6C640080402010C8
:10E8000008040201FD030303FD0303FDFDFD03FDF9
:10E8100003FDFDFDFD0303FD030303FDFD01FD03FA
:10E82000FDFD0303FF03FFFFF04E58444E52583ADC
:10E8300020706F732F6E65672F63656E7472652F1E
:10E840007468726573686F6C64004E58444E525819
:10E850003A2073796E6320666F756E6420706F73F3
:10E860002F63656E7472652F7468726573686F6C60
:10E8700064004E58444E52583A2073796E632074A7
:10E88000696D6564206F75742C206C6F7374206CD7
:10E890006F636B00CDF590804020100804020100EA
:10E8A0000101020102020301020203020303040147
:10E8B0000202030203030402030304030404050128
:10E8C0000202030203030402030304030404050217
:10E8D00003030403040405030404050405050601F9
:10E8E00002020302030304020303040304040502F7
:10E8F00003030403040405030404050405050602D8
:10E9000003030403040405030404050405050603C6
:10E9100004040504050506040505060506060701A9
:10E9200002020302030304020303040304040502B6
:10E930000303040304040503040405040505060297
:10E940000303040304040503040405040505060386
:10E950000404050405050604050506050606070268
:10E960000303040304040503040405040505060366
:10E970000404050405050604050506050606070347
:10E980000404050405050604050506050606070436
:10E990000505060506060705060607060707080318
:10E9A00003030303FD0303FDFD0303FDFDFDFD0361
:10E9B000FD03FDFDFDFDFD5575F5FF77FF5032357B
:10E9C00052583A20706F732F6E65672F63656E74AF
:10E9D00072652F7468726573686F6C6400503235AD
:10E9E00052583A2073796E6320666F756E642069A1
:10E9F0006E2048647220706F732F63656E74726549
:10EA00002F7468726573686F6C64005032355258A9
:10EA10003A2073796E6320666F756E6420696E208C
:10EA200050445520706F732F63656E7472652F7438
:10EA300068726573686F6C640050323552583A20C2
:10EA400073796E6320666F756E6420696E2054530F
:10EA5000445520706F732F63656E7472652F7468F0
:10EA6000726573686F6C640050323552583A207387
:10EA7000796E6320666F756E6420696E205444550C
:10EA800020706F732F63656E7472652F7468726582
:10EA900073686F6C640050323552583A2073796E47
:10EAA0006320666F756E6420696E205444554C4334
:10EAB00020706F732F63656E7472652F7468726552
:10EAC00073686F6C640050323552583A2073796E17
:10EAD0006320666F756E6420696E204C64752070CB
:10EAE0006F732F63656E7472652F746872657368D7
:10EAF0006F6C640050323552583A2073796E63203F
:10EB000074696D6564206F75742C206C6F7374204C
:10EB10006C6F636B0080402010080402010FFFFF40
:10EB2000FFFFFFF007F7D5DD57DFD00D5D7F77FDE5
:10EB30007570444D52536C6F7452583A206461742E
:10EB4000612068656164657220666F756E6420730C
:10EB50006C6F742F706F732F63656E7472652F7492
:10EB600068726573686F6C6400444D52536C6F74C7
:10EB700052583A2064617461207061796C6F6164ED
:10EB800020666F756E6420736C6F742F706F732FB7
:10EB900063656E7472652F7468726573686F6C64F8
:10EBA00000444D52536C6F7452583A20766F69632B
:10EBB000652068656164657220666F756E64207398
:10EBC0006C6F742F706F732F63656E7472652F7422
:10EBD00068726573686F6C6400444D52536C6F7457
:10EBE00052583A20766F69636520706920686561C4
:10EBF00064657220666F756E6420736C6F742F701D
:10EC00006F732F63656E7472652F746872657368B5
:10EC10006F6C6400444D52536C6F7452583A2076B6
:10EC20006F696365207465726D696E61746F7220BF
:10EC3000666F756E6420736C6F742F706F732F63C3
:10EC4000656E7472652F7468726573686F6C6400AA
:10EC5000444D52536C6F7452583A206373626B2068
:10EC6000666F756E6420736C6F742F706F732F6393
:10EC7000656E7472652F7468726573686F6C64007A
:10EC8000444D52536C6F7452583A20766F696365E5
:10EC90002073796E6320666F756E6420736C6F7479
:10ECA0002F706F732F63656E7472652F7468726551
:10ECB00073686F6C640003FDFDFD03FDFD0303033A
:10ECC000FD03FD03030303FDFD03FDFDFD03804084
:10ECD000201008040201FD030303FD0303FDFDFDF5
:10ECE00003FD03FDFDFDFD0303FD030303FDFD0324
:10ECF000030103FD0103FD01FF0303FF03FD030106
:10ED0000FD0359534652583A20706F732F6E656752
:10ED10002F63656E7472652F7468726573686F6CAB
:10ED2000640059534652583A2073796E6320666FD7
:10ED3000756E6420706F732F63656E7472652F74C7
:10ED400068726573686F6C640059534652583A2074
:10ED500073796E632074696D6564206F75742C20FF
:10ED60006C6F7374206C6F636B008040201008041C
:10ED70000201D471C9634D0FFFFFFFFFFFF007F7DA
:10ED8000D5DD57DFD00D5D7F77FD7570444D524462
:10ED90004D4F52583A206461746120686561646522
:10EDA0007220666F756E6420706F732F63656E746A
:10EDB00072652F7468726573686F6C6400444D529D
:10EDC000444D4F52583A2064617461207061796CEF
:10EDD0006F616420666F756E6420706F732F63655A
:10EDE0006E7472652F7468726573686F6C6400442A
:10EDF0004D52444D4F52583A20766F6963652068F2
:10EE0000656164657220666F756E6420706F732F24
:10EE100063656E7472652F7468726573686F6C6475
:10EE200000444D52444D4F52583A20766F69636505
:10EE30002070692068656164657220666F756E6414
:10EE400020706F732F63656E7472652F74687265BE
:10EE500073686F6C6400444D52444D4F52583A20D1
:10EE6000766F696365207465726D696E61746F7227
:10EE700020666F756E6420706F732F63656E747299
:10EE8000652F7468726573686F6C6400444D5244FA
:10EE90004D4F52583A206373626B20666F756E64F3
:10EEA00020706F732F63656E7472652F746872655E
:10EEB00073686F6C6400444D52444D4F52583A2071
:10EEC000766F6963652073796E6320666F756E6413
:10EED00020706F732F63656E7472652F746872652E
:10EEE00073686F6C640003FDFDFD03FDFD03030308
:10EEF000FD03FD03030303FDFD03FDFDFD03804052
:10EF0000201008040201FD030303FD0303FDFDFDC2
:10EF100003FD03FDFDFDFD0303FD030303FD0000F1
:10EF2000BF090A00B5814E0D1F080C002C87160B77
:10EF300061060F00DF96B508DF0413001892A606DD
:10EF40000F04170096438B05BC03190038421905BE
:10EF500000000300060009000C000F00120015005D
:10EF600018001B001E002100240027002A002D008D
:10EF700030003300360039003C003F0042004500BD
:10EF800048004B004E005100000103010601090139
:10EF90000C010F011201150118011B011E012101B5
:10EFA000240127012A012D013001330136013901E5
:10EFB0003C013F014201450148014B014E01510115
:10EFC00000020302060209020C020F0212021502DD
:10EFD00018021B021E022102240227022A022D020D
:10EFE00030023302360239023C023F02420245023D
:10EFF00048024B024E0251020003030306030903B9
:10F000000C030F031203150318031B031E03210334
:10F01000240327032A032D03300333033603390364
:10F020003C033F034203450348034B034E03510394
:10F0300000040304060409040C040F04120415045C
:10F0400018041B041E042104240427042A042D048C
:10F0500030043304360439043C043F0442044504BC
:10F0600048044B044E045104000503050605090538
:10F070000C050F051205150518051B051E052105B4
:10F08000240527052A052D053005330536053905E4
:10F090003C053F054205450548054B054E05510514
:10F0A00000060306060609060C060F0612061506DC
:10F0B00018061B061E062106240627062A062D060C
:10F0C00030063306360639063C063F06420645063C
:10F0D00048064B064E0651060007030706070907B8
:10F0E0000C070F071207150718071B071E07210734
:10F0F000240727072A072D07300733073607390764
:10F100003C073F074207450748074B074E07510793
:10F110000100040007000A000D0010001300160093
:10F1200019001C001F002200250028002B002E00C3
:10F130003100340037003A003D00400043004600F3
:10F1400049004C004F0052000101040107010A016F
:10F150000D0110011301160119011C011F012201EB
:10F16000250128012B012E013101340137013A011B
:10F170003D0140014301460149014C014F0152014B
:10F180000102040207020A020D0210021302160213
:10F1900019021C021F022202250228022B022E0243
:10F1A0003102340237023A023D0240024302460273
:10F1B00049024C024F0252020103040307030A03EF
:10F1C0000D0310031303160319031C031F0322036B
:10F1D000250328032B032E033103340337033A039B
:10F1E0003D0340034303460349034C034F035203CB
:10F1F0000104040407040A040D0410041304160493
:10F2000019041C041F042204250428042B042E04C2
:10F210003104340437043A043D04400443044604F2
:10F2200049044C044F040105040507050A050D05B2
:10F2300010051305160519051C051F0522052505D2
:10F2400028052B052E053105340537053A053D0502
:10F2500040054305460549054C054F0501060406D2
:10F2600007060A060D0610061306160619061C06E2
:10F270001F062206250628062B062E063106340612
:10F2800037063A063D0640064306460649064C0642
:10F290004F060107040707070A070D0710071307A2
:10F2A000160719071C071F072207250728072B0722
:10F2B0002E073107340737073A073D074007430752
:10F2C000460749074C074F070200050008000B00DE
:10F2D0000E001100140017001A001D00200023006A
:10F2E000260029002C002F003200350038003B009A
:10F2F0003E004100440047004A004D00500002011A
:10F30000050108010B010E011101140117011A0179
:10F310001D0120012301260129012C012F013201A9
:10F32000350138013B013E014101440147014A01D9
:10F330004D0150010202050208020B020E021102E9
:10F34000140217021A021D022002230226022902B9
:10F350002C022F023202350238023B023E024102E9
:10F36000440247024A024D02500202030503080309
:10F370000B030E031103140317031A031D032003C9
:10F380002303260329032C032F03320335033803F9
:10F390003B033E034103440347034A034D03500329
:10F3A0000204050408040B040E04110414041704D9
:10F3B0001A041D0420042304260429042C042F0409
:10F3C0003204350438043B043E0441044404470439
:10F3D0004A044D0450040205050508050B050E05F9
:10F3E0001105140517051A051D0520052305260519
:10F3F00029052C052F053205350538053B053E0549
:10F400004105440547054A054D0550050206050618
:10F4100008060B060E061106140617061A061D0628
:10F4200020062306260629062C062F063206350658
:10F4300038063B063E064106440647064A064D0688
:10F4400050060207050708070B070E0711071407E8
:10F4500017071A071D0720072307260729072C0768
:10F460002F073207350738073B073E074107440798
:10F4700047074A074D075007704F934064746D303B
:10F480002BE72D545F8A1D7FB8A7492032BA3698E2
:10F4900095F316AA2FC58E3FDCD32410195D1BCC23
:10F4A000CA790BD59762C71FEE6912888CAE0D66BC
:10F4B000E5BC85EA4BB1E30FF734094446D706B300
:10F4C00072DE42F5A5D8F1877B9A0422A36B83599B
:10F4D000396F007FBFDFEFF7FBFDFE804020100893
:10F4E000040201FEFDFBF7EFDFBF7F44537461723E
:10F4F00052583A20666F756E64206672616D6520A1
:10F5000073796E6320696E204E6F6E65004453748C
:10F51000617252583A20666F756E6420646174613E
:10F520002073796E6320696E204E6F6E65004453C0
:10F5300074617252583A20466F756E6420656E642D
:10F540002073796E6320696E2044617461004453B6
:10F5500074617252583A20646174612073796E63E9
:10F560002074696D6564206F75742C206C6F7374E2
:10F57000206C6F636B0001020408102040800000C3
:10F58000891112239B322446AD573665BF74488CCF
:10F59000C19D5AAFD3BE6CCAE5DB7EE9F7F8811096
:10F5A000080193331A22A5562C47B7753E64C99CAF
:10F5B000408DDBBF52AEEDDA64CBFFF976E8022175
:10F5C0008B30100299132667AF763444BD554AAD8F
:10F5D000C3BC588ED19F6EEBE7FA7CC8F5D9833156
:10F5E0000A2091121803A7772E66B5543C45CBBD6F
:10F5F00042ACD99E508FEFFB66EAFDD874C9044235
:10F600008D5316619F702004A9153227BB364CCE4E
:10F61000C5DF5EEDD7FC6888E1997AABF3BA855215
:10F620000C4397711E60A1142805B3373A26CDDE2E
:10F6300044CFDFFD56ECE9986089FBBB72AA0663F4
:10F640008F7214409D512225AB343006B9174EEF0E
:10F65000C7FE5CCCD5DD6AA9E3B8788AF19B8773D5
:10F660000E6295501C41A3352A24B1163807CFFFEE
:10F6700046EEDDDC54CDEBB962A8F99A708B0884B4
:10F6800081951AA793B62CC2A5D33EE1B7F04008E6
:10F69000C919522BDB3A644EED5F766DFF7C89947D
:10F6A00000859BB712A6ADD224C3BFF136E0C118C6
:10F6B0004809D33B5A2AE55E6C4FF77D7E6C0AA55C
:10F6C00083B4188691972EE3A7F23CC0B5D14229A6
:10F6D000CB38500AD91B666FEF7E744CFD5D8BB53D
:10F6E00002A499961087AFF326E2BDD034C1C33986
:10F6F0004A28D11A580BE77F6E6EF55C7C4D0CC61C
:10F7000085D71EE597F42880A1913AA3B3B2444A65
:10F71000CD5B5669DF78600CE91D722FFB3E8DD6FC
:10F7200004C79FF516E4A9902081BBB332A2C55A45
:10F730004C4BD7795E68E11C680DF33F7A2E0EE7DB
:10F7400087F61CC495D52AA1A3B03882B193466B25
:10F75000CF7A5448DD59622DEB3C700EF91F8FF7BC
:10F7600006E69DD414C5ABB122A0B9923083C77B05
:10F770004E6AD5585C49E33D6A2CF11E780F9E8D88
:10F780003288261A3F61E8552D160755FD7DF75F33
:10F7900070013000009009100170009000074001D6
:10F7A0007000314007400150A171D170700110000C
:10F7B00000000E2000004F08DC028815782CD014C1
:10F7C000C084ADFF57D75DF5D96524022806200F08
:10F7D000801BC107805C0000200808023815002C3F
:10F7E000A01460846D5D7F77FD757E30300110015F
:10F7F0004003C013C11E806F333AA0300055A65F8E
:10F800005007F7D5DD57DFD0013000009009100117
:10F81000700090000740017000314007400150A186
:10F8200071D1707001100000000E2000004F08DC44
:10F83000028815782CD014C084AD5D7F77FD757972
:10F840006524022806200F801BC107805C00002071
:10F850000808023815002CA01460846DFF57D75D8E
:10F86000F5DE30300110014003C013C11E806F006F
:10F87000CEA8FE83ACC458200ACEA8FE83A0000008
:10F880000000000CC458200ACEA8FE83ACC4582047
:10F890000A0000008EB093E01D50A97027C03A9076
:10F8A000B420DC6052D04F80C1307510FBA0E6F070
:10F8B00068403670B8C0A5902B209F0011B00CE0B6
:10F8C0008250EA1064A079F0F7404360CDD0D08038
:10F8D0005E306CD0E260FF307180C5A04B105640A6
:10F8E000D8F0B0B03E002350ADE019C097708A2028
:10F8F00004905AA0D410C94047F0F3D07D60603026
:10F90000EE8086C0087015209B902FB0A100BC50DF
:10F9100032E0D99057204A70C4C070E0FE50E30036
:10F920006DB005F08B40961018A0AC8022303F607F
:10F93000B1D0EFE061507C00F2B04690C820D570A5
:10F940005BC03380BD30A0602ED09AF01440091007
:10F9500087A0B5403BF026A0A8101C3092808FD025
:10F9600001606920E790FAC07470C0504EE053B057
:10F97000DD0083300D8010D09E602A40A4F0B9A035
:10F9800037105F50D1E0CCB04200F620789065C0CF
:10F99000EB703DA0B310AE4020F094D01A60073059
:10F9A0008980E1C06F707220FC9048B0C600DB50C7
:10F9B00055E00BD0856098301680A2A02C10314005
:10F9C000BFF0D7B059004450CAE07EC0F070ED20BF
:10F9D00063905170DFC0C2904C20F80076B06BE0AD
:10F9E000E5508D1003A01EF090402460AAD0B7808F
:10F9F00039306700E9B0F4E07A50CE7040C05D90D5
:10FA0000D320BB6035D02880A63012109CA081F096
:10FA10000F40E4306A8077D0F9604D40C3F0DEA03B
:10FA200050103850B6E0ABB0250091201F9002C0B6
:10FA30008C70D2405CF041A0CF107B30F580E8D0D4
:10FA400066600E2080909DC01370A75029E034B0EE
:10FA5000BA0088E006501B0095B02190AF20B2702C
:10FA60003CC05480DA30C76049D0FDF073406E105E
:10FA7000E0A0BE9030202D70A3C017E09950840004
:10FA80000AB062F0EC40F1107FA0CB8045305860A6
:10FA9000D6D00000000000000100000002000000BD
:10FAA0000300000004000000050000000600000044
:10FAB0000700000008000000090000000A00000024
:10FAC0000B0000000C0000000D0000000E00000004
:10FAD0002040020010000000110000001200000091
:10FAE00013000000140000001500000016000000C4
:10FAF0001700000018000000190000001A000000A4
:10FB00001B0000001C0000001D00000040800400DD
:10FB100080140000200000002100000022000000EE
:10FB20002300000024000000250000002600000043
:10FB30000840020028000000290000002A00000000
:10FB4000044002002C0000000240020001400200BC
:10FB500000400200300000003100000032000000D0
:10FB60008081000034000000400C000036000000DE
:10FB7000420C000038000000003004003A00000091
:10FB80000230040002290000124002000029000097
:10FB90001040020040000000410000004200000050
:10FBA0004300000044000000450000004600000043
:10FBB0004700000048000000490000004A00000023
:10FBC000002500004C0000004D00000010800400E3
:10FBD000118004005000000051000000520000009D
:10FBE0000012020054000000200C000008800400F5
:10FBF000098004005800000059000000048004003F
:10FC000005800400028004000380040000800400DA
:10FC1000018004006000000061000000620000003C
:10FC20006300000064000000100C000000030100ED
:10FC300000B00000680000006900000080180000AB
:10FC4000811800008101040080010400414002008D
:10FC50004040020070000000040C00007200000030
:10FC6000060C0000010C0000000C0000030C00005A
:10FC7000020C0000045200000C0C00002480040060
:10FC80002580040000520000080C000020800400C1
:10FC9000218004008000000081000000820000003C
:10FCA0008300000084000000850000008600000042
:10FCB0008700000088000000890000008A00000022
:10FCC000000205008C00000000A8000011140000D4
:10FCD000101400009000000091000000920000004D
:10FCE000208100009400000095000000004A000000
:10FCF000081400009800000099000000051400009E
:10FD00000414000003140000021400000114000099
:10FD100000140000A0000000A1000000A2000000EC
:10FD200010810000A4000000A500000000240400D1
:10FD300001240400A8000000A900000040180000F1
:10FD4000411800004101040040010400814002000C
:10FD500080400200B000000002810000018100002C
:10FD600000810000B4000000068100000581000051
:10FD700004810000010A0200000A0200098100005B
:10FD80000881000023140000221400002114000048
:10FD900020140000C0000000C1000000C2000000EC
:10FDA000C3000000C4000000C5000000C600000041
:10FDB000C7000000C8000000C900000020180000B3
:10FDC000211800000006020020010400006001006C
:10FDD00001600100D0000000D100000001280400F3
:10FDE0000028040000310000008201000231000000
:10FDF00002820100D8000000D900000084800400C5
:10FE0000441400008280040042140000808004003A
:10FE100040140000E000000000200300081800006B
:10FE20000046000009010400080104000C1800004D
:10FE30000A01040002180000040104000018000078
:10FE40000118000001010400000104000418000072
:10FE50000201040008A4000042810000418100006A
:10FE600040810000810C0000800C0000830C000029
:10FE7000820C000000A4000001A400001018000083
:10FE800011180000110104001001040014180000F2
:10FE90001201040000010000010100000201000045
:10FEA000030100000401000005010000060100003C
:10FEB0000018040008010000090100000A01000008
:10FEC000402400000C0100000D0100000E010000A4
:10FED0004424000010010000110100001201000084
:10FEE000A0800000140100001501000016010000B0
:10FEF000A48000001801000019010000005001005A
:10FF000001500100222800002328000020280000C2
:10FF10002128000020010000210100002201000032
:10FF20009080000024010000250100004002010033
:10FF30004102010028010000290100002A010000FF
:10FF40000441020000940000C000040010280000DA
:10FF5000004102003001000082800000818000002A
:10FF6000808000000110030000100300082800003A
:10FF700084800000062800008A8000000428000019
:10FF800088800000022800000328000000280000EC
:10FF90000128000040010000410100004201000072
:10FFA0000824000044010000450100002002010077
:10FFB0002102010048010000022400000124000089
:10FFC00000240000A1000400A0000400052400009B
:10FFD0000424000050010000510100005201000003
:10FFE00018240000803000008130000082300000C2
:10FFF00083300000019800000098000011240000E8
:020000040801F1
:100000001024000002810400049800000081040014
:100010000181040060010000610100000402010090
:100020000502010002020100880004000002010034
:100030000102010085000400840004002124000066
:100040002024000081000400800004000802010058
:100050008200040002140400C280000000140400A6
:10006000C0800000010D0000000D00001002010022
:1000700011020100950004009400040044280000CF
:10008000C880000091000400900004004028000097
:100090004128000080010000810100008201000071
:1000A00030800000840100000044010001220200B1
:1000B0000022020088010000890100008A0100007E
:1000C0003880000061000400600004006300040048
:1000D00062000400900100002280000021800000E6
:1000E00020800000403000004130000025800000EA
:1000F00024800000000C0400010C04002980000092
:100100002880000000C0020001C0020001150000AC
:1001100000150000A0010000128000001180000006
:100120001080000049000400480004001580000011
:10013000148000000062000044000400000403007A
:100140001880000041000400400004004300040047
:1001500042000400038000000280000001800000D3
:10016000008000000780000006800000058000007D
:10017000048000000B8000000A800000098000005D
:100180000880000051000400500004008028000096
:100190000C800000C0010000C1010000004006000A
:1001A000014006001030000028000400008C000010
:1001B000018C0000250004002400040081240000BC
:1001C000802400002100040020000400230004001B
:1001D00022000400043000000530000061800000AF
:1001E000608000000030000001300000023000009C
:1001F000033000000C300000340004000508030048
:100200000408030008300000300004000108030067
:10021000000803000D0004000C00040051800000E1
:100220005080000009000400080004008002010062
:100230000A00040005000400040004000019000086
:100240000600040001000400000004000300040094
:1002500002000400004801004280000041800000CC
:10026000408000002030000018000400458000009D
:1002700044800000150004001400040049800000C0
:100280004880000011000400100004001300040066
:10029000120004000002000001020000020200003F
:1002A0000302000004020000050200000602000034
:1002B0000702000008020000090200000A02000014
:1002C000800005000C0200000D0200000E0200007C
:1002D000840005001002000011020000120200005C
:1002E00040100200140200001502000080480000C7
:1002F00081480000180200001902000001E000001F
:1003000000E000001C0200001D0200008848000000
:1003100004E0000020020000210200002202000090
:100320002302000024020000250200004001010019
:100330004101010028020000290200002A020000F9
:1003400004420200012401000024010001420200D5
:1003500000420200300200003102000032020000C0
:100360006010020000A0020001A0020002A0020032
:1003700003A0020081080200800802008308020036
:10038000820802004050000041500000425000002E
:100390001042020040020000410200004202000040
:1003A000101002004402000000600400200101005F
:1003B0002101010048020000490200004A02000039
:1003C000181002008004020081040200820402006E
:1003D000830402005002000002100200011002001B
:1003E00000100200818001008080010005100200E1
:1003F0000410020000280100012801000910020079
:10040000081002002050000021500000008204006B
:10041000018204006002000061020000040101008A
:1004200080440000020101000301010000010100FD
:100430000101010002200600032006000020060042
:1004400001200600105000001150000008010100BA
:10045000090101000C5000002210020021100200CE
:100460002010020008500000000E000010010100E2
:10047000110101000450000005500000065000006A
:10048000281002000050000001500000025000003F
:100490000350000080020000810200008202000080
:1004A00008000500840200008502000010480000DA
:1004B0000021020088020000020005000100050082
:1004C0000000050040040200410402000500050090
:1004D00004000500900200009102000004480000A2
:1004E000054800000248000040800100004800006C
:1004F0000148000021080200200802001100050048
:10050000100005000A48000002160000084800001C
:1005100000160000A0020000A102000041440000FB
:1005200040440000A4020000A50200003048000082
:100530004444000000610000100802002100050092
:1005400020000500046100001408020025000500D9
:10055000240005000908020008080200003001001C
:1005600000830000224800000C0802002048000020
:1005700021480000010802000008020003080200F0
:1005800002080200050802000408020028480000D2
:1005900006080200C0020000C10200002144000061
:1005A0002044000008040200108001000A04020038
:1005B000128001000404020005040200410005004D
:1005C00040000500000402000104020002040200D1
:1005D0000304020005800100048001008110020074
:1005E00080100200018001000080010040480000EE
:1005F00002800100140402000C8001008910020036
:100600008810020010040200088001001204020099
:100610000A8001000344000002440000014400007D
:100620000044000082010100064400008001010036
:1006300004440000021A00000A440000001A0000EE
:100640000844000020040200000304002204020009
:10065000020304001344000012440000114400008F
:100660001044000021800100208001009001010061
:10067000228001004108020040080200101A000018
:1006800042080200805000008150000082500000AB
:10069000835000000003000001030000020300007B
:1006A00003030000040300000503000060000100D4
:1006B00080200200080300000903000000880200F7
:1006C00001880200024404000344040000440400C2
:1006D000014404001003000011030000010C01009C
:1006E000000C01001403000015030000700001005D
:1006F000040C010018030000190300001088020018
:10070000080C010012440400000000001044040022
:10071000114404002003000000040600440001000E
:10072000450001004200010000C800004000010037
:1007300041000100806000008160000082600000D4
:10074000836000004A00010008C800004800010062
:1007500049000100088005008282000081820000BB
:10076000808200005200010010C80000500001000B
:100770005100010000800500018005000280050095
:1007800088820000022A0000032A0000002A0000DC
:10079000012A000040030000410300002400010082
:1007A00025000100220001002300010020000100BB
:1007B0002100010001400300004003000126000069
:1007C000002600002A000100044003002800010068
:1007D0002900010000C4000001C400000111020052
:1007E00000110200000806000108060030000100A8
:1007F0003100010008C4000010400300091102008C
:100800000811020008080600090806003800010067
:10081000208402000600010007000100040001001E
:1008200005000100020001000300010000000100BA
:10083000010001000E000100840204000C00010010
:100840000D0001000A000100800204000800010000
:10085000090001001600010017000100140001004A
:10086000150001001200010013000100100001003A
:100870001100010004510000024804000148040076
:100880000048040000510000015100001800010060
:1008900000840200800300008103000005200200A4
:1008A00004200200032002000220020001200200B6
:1008B000002002002060000021600000010105000E
:1008C00000010500001801000118010009200200C4
:1008D00008200200015004000050040021820000A2
:1008E000208200000249000012200200004900009E
:1008F000102002003060000008500400298200002F
:100900002882000010180100111801000849000099
:100910001820020008600000096000001182000039
:1009200010820000C200010022200200C00001006D
:100930002020020000600000016000000260000052
:100940000360000004600000400204000660000034
:1009500042020400038200000282000001820000C3
:10096000008200000782000006820000058200006D
:1009700004820000106000000009020009820000EB
:1009800008820000021006000409020000100600A0
:10099000011006002090020021900200A400010036
:1009A00044200200A200010042200200A000010039
:1009B00040200200040502002402040005D00000CB
:1009C00004D00000000502002002040001D0000055
:1009D00000D00000043200000481010061820000A8
:1009E000608200000032000000810100023200003D
:1009F0000281010021140100201401000000000008
:100A000022140100083200000881010011D000000A
:100A100010D000000090020001900200840001004C
:100A2000004500008200010008020400800001006F
:100A300081000100406000000402040042600000E8
:100A40000602040001020400000204008800010004
:100A50000202040010900200428200004182000065
:100A60004082000092000100180204009000010082
:100A700091000100011401000014010003140100A1
:100A80000214010011020400100204009800010089
:100A9000120204000004000001040000020400002F
:100AA0000304000004040000050400000604000024
:100AB0000704000008040000090400000A04000004
:100AC000402100000C0400000D0400009110000003
:100AD0009010000010040000110400001204000037
:100AE00013040000140400006008000089100000D6
:100AF000881000001804000000800300851000002A
:100B0000841000008310000082100000811000009B
:100B100080100000200400002104000022040000D6
:100B2000230400002404000050080000802004007A
:100B3000812004002804000029040000018804002A
:100B4000008804000091000000220100014402001E
:100B50000044020030040000440800003204000099
:100B600046080000410800004008000000C00100E5
:100B700042080000380400004C080000A5100000E6
:100B8000A41000004908000048080000A11000005F
:100B9000A0100000400400004104000042040000D6
:100BA0000821000044040000300800000100070094
:100BB000000007004804000002210000012100009D
:100BC00000210000800202008102020005210000D5
:100BD000042100005004000024080000520400001A
:100BE000260800002108000020080000230800005B
:100BF0002208000002480200122100000048020002
:100C000010210000290800002808000000840400CA
:100C1000C0100000600400001408000081420000C1
:100C200080420000110800001008000013080000B6
:100C300012080000004005000140050021210000CD
:100C40002021000019080000180800001B080000FF
:100C50001A08000005080000040800000011040044
:100C6000060800000108000000080000030800005A
:100C70000208000080A000000C08000082A0000014
:100C80000E08000009080000080800000B0800001A
:100C90000A080000800400008104000082040000B3
:100CA00083040000840400000041010020200400AF
:100CB00018100000880400008904000015100000CE
:100CC0001410000040020200121000001110000079
:100CD0001010000090040000910400000D100000AE
:100CE0000C1000000B1000000A100000091000009A
:100CF00008100000000904000610000005100000A4
:100D00000410000003100000021000000110000099
:100D100000100000A0040000A10400000420040052
:100D200040420000022004000320040000200400D0
:100D3000012004000201030003010300000103007D
:100D4000010103000A200400321000000820040002
:100D50003010000000500200015002000185000028
:100D600000850000C1080000C00800001020040039
:100D70002810000040A0000041A000002510000045
:100D80002410000023100000221000002110000099
:100D900020100000C0040000009004002142000068
:100DA000204200000802020009020200008900003F
:100DB00001890000040202000502020081210000F6
:100DC0008021000000020200010202000202020073
:100DD0005010000028A00000A40800004D100000E2
:100DE0004C100000A1080000A008000049100000FD
:100DF0004810000020A0000021A0000045100000C5
:100E000044100000100202004210000041100000D7
:100E100040100000034200000242000001420000B6
:100E200000420000910800009008000040200400EB
:100E30000442000010A0000011A00000001C0000EF
:100E40000842000020020200000504002202020005
:100E50000205040008A00000840800001142000000
:100E60001042000081080000800800008308000094
:100E70008208000000A0000001A0000002A0000005
:100E800003A0000004A0000088080000611000001A
:100E900060100000000500000105000002050000D0
:100EA0004820000004050000804001000605000005
:100EB000824001000805000042200000412000009F
:100EC000402000002090000021900000004204001B
:100ED000442000001005000011050000010A010077
:100EE000000A010001A0040000A0040003A0040007
:100EF00002A00400800804008108040051200000C2
:100F000050200000840804008211000081110000BC
:100F100080110000200500000002060022050000EC
:100F20000202060008900000099000000A900000EC
:100F30000B9000000490000005900000800003006A
:100F4000602000000090000001900000029000006E
:100F5000039000004210040082840000401004004E
:100F60008084000041090000400900004410040092
:100F7000420900001490000015900000042C0000AD
:100F8000888400001090000011900000002C0000E8
:100F9000012C0000400500000A200000092000008C
:100FA00008200000828800000E20000080880000D9
:100FB0000C2000000320000002200000012000009F
:100FC000002000000720000006200000052000008F
:100FD0000420000000C2000001C200002010040034
:100FE000182000002109000020090000241004003E
:100FF0002209000013200000122000001120000030
:10100000102000001720000016200000152000000E
:1010100014200000121004002A2000001010040008
:1010200028200000006002001009000000060100F6
:1010300001060100232000002220000021200000E2
:1010400020200000409000008004040025200000C3
:101050002420000002100400040900000010040015
:101060000110040001090000000900000410040040
:10107000020900000A1004003220000008100400D9
:101080003020000009090000080900000182020068
:10109000008202008005000004400100820500007B
:1010A00006400100014001000040010040880000AE
:1010B0000240010010080400110804002000030091
:1010C000C02000000940010008400100111100008B
:1010D0001011000008080400090804002184000021
:1010E000208400001140010010400100091100009F
:1010F00008110000000804000108040002080400B0
:101100000411000004080400021100000111000095
:101110000011000001380000003800000800030042
:101120001084000021400100204001000021040043
:10113000012104000200030003000300000003007B
:10114000010003008090000040040400040003003C
:1011500005000300038400000284000001840000F5
:10116000008400000784000006840000058400005D
:10117000048400002008040021080400100003007B
:10118000088400002408040022110000211100003E
:1011900020110000068800008A200000048800005A
:1011A0008820000002880000404001000088000004
:1011B00001880000832000008220000081200000C0
:1011C00080200000000302002004040008880000C2
:1011D000842000000434000005340000148800005E
:1011E0009820000000340000013400001088000046
:1011F000118800004008040041080400912000000C
:101200009020000044080400421100004111000039
:1012100040110000034300000243000001430000AE
:1012200000430000090404000804040020880000B2
:1012300021880000050404000404040040000300A9
:10124000A0200000010404000004040003040400C2
:101250000204040082100400428400008010040094
:10126000408400008109000080090000841004000F
:101270008209000000A100000012010002A100008C
:1012800002120100110404001004040013040400FD
:10129000120404000006000001060000020600001F
:1012A0000306000004060000050600000606000014
:1012B0000706000008060000005800000A060000AB
:1012C00002580000C000020020200100004104007C
:1012D0000141040010060000110600000109010090
:1012E00000090100001005000110050002100500B2
:1012F00004090100180600001058000085120000C3
:101300008412000008100500821200008112000003
:10131000801200002006000000010600C14000000D
:10132000C040000009200100082001000018020050
:10133000011802000520010004200100072001001F
:10134000062001000120010000200100032001000F
:101350000220010030060000440A0000D1400000D5
:10136000D0400000410A0000400A000010180200AE
:10137000420A0000152001001420010000000000B6
:10138000162001001120010010200100132001008F
:10139000122001004006000041060000A1400000AC
:1013A000A040000088000200890002008A000200BC
:1013B000A4400000840002008500020000900100AB
:1013C0000023000080000200810002008200020071
:1013D0008300020000C1000001C1000001140200EE
:1013E00000140200210A0000200A0000230A000065
:1013F000220A0000940002009500020010900100F3
:101400000814020090000200910002009200020005
:1014100020810200834000008240000081400000E3
:1014200080400000110A0000100A000000050100C1
:1014300084400000A40002008A40000089400000AF
:1014400088400000A000020040200100A20002002D
:1014500042200100050A0000040A0000914000003B
:1014600090400000010A0000000A0000030A00008A
:10147000020A0000045400000C0A0000058102006A
:101480000481020000540000080A000001810200EB
:10149000008102008006000081060000614000001B
:1014A0006040000048000200490002004A000200BB
:1014B00064400000440002004500020001040500F1
:1014C000000405004000020041000200420002004A
:1014D0001012000002800600038006000080060053
:1014E00001800600024C00000A120000004C0000BF
:1014F000081200005400020006120000051200004D
:10150000041200005000020002120000011200004C
:10151000001200000088010042400000414000002D
:101520004040000002220400464000000022040067
:1015300044400000640002004A40000049400000AE
:1015400048400000600002008020010062000200AC
:10155000822001001088010052400000514000002C
:101560005040000009C0040008C00400102204001C
:1015700054400000010C0200000C0200030C0200A9
:10158000020C020001C0040000C00400211200008F
:10159000201200000C000200224000002140000048
:1015A0002040000008000200090002000A000200BA
:1015B00024400000040002000500020006000200B2
:1015C00028400000000002000100020002000200AA
:1015D000030002001C000200324000003140000005
:1015E0003040000018000200008401001A000200D0
:1015F000028401001400020015000200160002001F
:10160000441200001000020011000200120002004B
:1016100040120000034000000240000001400000B2
:1016200000400000280002000640000005400000C5
:1016300004400000240002000A40000009400000AD
:1016400008400000200002002100020022000200E9
:101650000C40000013400000124000001140000048
:1016600010400000810A0000800A000015400000C0
:101670001440000000A20000001101001940000009
:101680001840000030000200310002000008050090
:1016900001080500000700002000060011080100F5
:1016A000100801000A40040024000600084004005D
:1016B00009400400064004004222000004400400E7
:1016C00040220000024004000340040000400400E7
:1016D0000140040040C000000208010001080100B0
:1016E0000008010044C000000608010005080100D0
:1016F0000408010000300200013002000908010066
:1017000008080100124004001340040010400400C7
:10171000114004000100060000000600030006005E
:101720000200060005000600040006004004010057
:1017300041040100090006000800060024400400DE
:101740000A00060000920000002101002040040071
:1017500021400400110006001000060021080100CD
:1017600020080100037000000270000001700000FA
:1017700000700000203002001800060045800200C2
:10178000448002001092000042800200418002006A
:101790004080020010C0000011C0000009220000BB
:1017A000082200002204010023040100200401009B
:1017B0002104010003220000022200000122000097
:1017C000002200008001020081010200404004006C
:1017D0000422000000C0000001C0000002C00000A0
:1017E0004008010004C0000005C0000006C0000061
:1017F0004408010008C0000009C0000011220000D8
:10180000102200000CC00000228002002180020093
:101810002080020041000600400006000404010090
:1018200080410000020401000304010000040100E3
:1018300001040100232200002222000021220000D6
:10184000202200000A0401001280020008040100A6
:101850001080020020C0000021C00000001204001F
:1018600001120400010B0000000B00001004010035
:101870000880020081100100801001000580020034
:101880000480020003800200028002000180020046
:1018900000800200402005000442010005240200EF
:1018A0000424020001420100004201000124020060
:1018B00000240200440102004501020084400400AB
:1018C000C0220000400102004101020080400400EB
:1018D00081400400080A0400820801008108010018
:1018E00080080100114201001042010008A001001F
:1018F00084080100000A0400010A0400020A04002E
:101900000413000002A001000213000000A0010067
:101910000013000081000600800006004141000025
:10192000404100008500060084000600C00401005C
:101930004441000000640000016400000002030054
:1019400001020300046400004006040004020300D6
:1019500005020300038600000286000001860000E5
:1019600000860000000000000686000005860000DA
:101970000486000041100100401001001002030025
:1019800042100100451001004410010020A0010098
:101990002013000000200500012005002141000067
:1019A000204100000801020009010200008A000035
:1019B000018A0000040102000501020081220000EA
:1019C0008022000000010200010102000201020069
:1019D0000301020080C0000081C0000082C000003E
:1019E0003041000084C0000008680000108A000038
:1019F000118A0000211001002010010023100100B5
:101A00002210010010010200006800001201020013
:101A10000268000003410000024100000141000093
:101A20000041000082040100064100008004010022
:101A300004410000111001001010010009410000D4
:101A400008410000200102000006040022010200FB
:101A5000020604000910010008100100002802001D
:101A6000104100000D1001000C10010004280200BC
:101A700014410000011001000010010003100100DA
:101A80000210010005100100041001008180020015
:101A90008080020000000044495245435420204405
:101AA0004952454354202043514351435120204D36
:101AB0004D44564D20202054455354A96A9E8D32E2
:101AC00088261A3F61E8552D164D65737361676569
:101AD00020637265617465642077697468206C6541
:101AE0006E6774680000000041000000000000B84C
:101AF0000800000042000000000080EA0C00000026
:101B0000430000000000A0EB0E00000044000000B5
:101B1000000000EA0A00000045000000000000800C
:101B20000400000046000000000080AE0C00000031
:101B300047000000000080EE0C000000480000009C
:101B4000000000AA0A00000049000000000000A0F8
:101B5000060000004A0000000000B8BB10000000B2
:101B60004B000000000080EB0C0000004C00000067
:101B7000000080BA0C0000004D000000000000EEE4
:101B80000A0000004E000000000000E8080000000D
:101B90004F0000000000E0EE0E00000050000000CA
:101BA0000000A0BB0E000000510000000000B8EED5
:101BB0001000000052000000000000BA0A000000FF
:101BC00053000000000000A80800000054000000BE
:101BD000000000E00600000055000000000000AE1C
:101BE0000A00000056000000000080AB0C0000005E
:101BF00057000000000080BB0C00000058000000EF
